:100000000C943A1B0C946B1B0C946B1B0C946B1B89
:100010000C946B1B0C946B1B0C946B1B0C946B1B48
:100020000C946B1B0C946B1B0C946B1B0C946B1B38
:100030000C946B1B0C946B1B0C946B1B0C946B1B28
:100040000C946B1B0C94E59C0C946B1B0C946B1B1D
:100050000C946B1B0C946B1B0C9411BD0D94F5054B
:100060000C946B1B0C9450560C9446560C946B1BC2
:100070000C946B1B0C946B1B0C946B1B0C946B1BE8
:100080000C946B1B0C946B1B0C946B1B0C946B1BD8
:100090000C946B1B0C946B1B0C946B1B0C946B1BC8
:1000A0000C946B1B0C946B1B0C946B1B0C946B1BB8
:1000B0000C946B1B0C946B1B0C946B1B0C946B1BA8
:1000C0000C946B1B0C946B1B0C946B1B0C94F558D1
:1000D0000C94CB580C946B1B0C946B1B0C946B1BEB
:1000E0000C946B1B1A1D601D661D8D1D9A1DA31D92
:1000F000AE1D722592266E27A127FE32FE32BC2845
:100100005F296E26FE32FE32FC2A952CCD2CFE3263
:10011000CB2EFE32FE321C30FE32FE32A630D930FB
:10012000FE3255311132DC2CE42C082D2C2D602DA3
:10013000032E172E302E3D2E4A2E5E2E83568956C4
:100140009B56AB56B356E056B756E056BB56BF5615
:10015000E056C356C756CB56D356E056DD564BE84D
:100160004EE83DE841E847E885E852E856E85CE8B3
:1001700060E864E86AE86EE872E885E878E87CE8B8
:1001800080E888ED8DED92ED9CEDA6ED1FEEB0EDD3
:10019000B8EDC0EDCAEDD4EDDEEDEDEDF7ED1FEEFF
:1001A00001EE0BEE15EEB0F5B3F5B7F5BAF5BDF50A
:1001B000E7F5C1F5C4F5C8F5CBF5CEF5D2F5D5F523
:1001C000D8F5E7F5DCF5DFF5E2F532F654F674F62E
:1001D00099F6BEF675F8E3F606F729F74EF773F7CA
:1001E00098F7BDF7E2F775F807F82CF851F8084AC8
:1001F000D73B3BCE016E84BCBFFDC12F3D6C74313B
:100200009ABD56833DDA3D00C77F11BED9E4BB4C91
:100210003E916BAAAABE000000803F05A84CCDB25B
:10022000D44EB93836A9020C50B9918688083CA63C
:10023000AAAA2ABE000000803F000C94CAED0C94CC
:100240004EE80C94DD570C94CD2C0C9411320C9488
:10025000B0F50C9489560C944EF70C9499F60C94C6
:100260005E2E0C9483560C9474F60C94C0ED0C9492
:100270001FEE0C943DE80C94602D0C94B3560C9436
:100280008D1D0C940BEE0C948DED0C9451F80C9488
:100290002CF80C9407F80C94DEED0C94302E0C9492
:1002A000CB560C9415EE0C9441E80C9488ED0C940C
:1002B00032F60D94490F0C94082D0C9483570C942E
:1002C000BAF50C94C3560C9475F80C9456E80C943B
:1002D00060E80C94FC2A0C94BC280C949A1D0C9495
:1002E00078E80C9401EE0C94D9300C94E2F70C945D
:1002F00006F70C9447E80C9472250C94E42C0C94AB
:10030000BDF50C94AE1D0C949B560C9492ED0C9480
:10031000C1F50C94B7F50C94A6300C9473F70C94BB
:10032000C7560D94A40E0C9454F60C9498F70C94A4
:10033000AB560C946EE80C9492260C941A1D0C94F7
:1003400097570C94DFF50C94601D0C94CB2E0C94F5
:100350006E260C9480E80C945CE80C94B0ED0C9440
:10036000DD560C94E0560C94E2F50C944BE80C949A
:10037000CEF50C94B3F50C94661D0C94C4F50C9456
:100380007CE80C94C8F50C9455310C94032E0C9415
:100390002C2D0C9446570C94D2F50C94EDED0C9446
:1003A0001C300C9474570C94BEF60C946E270C946D
:1003B0006AE80C94CBF50C94E3F60C943D2E0C9467
:1003C0009CED0C94BDF70C942A580C94DCF50C941D
:1003D000B8ED0C94BF560C94D4ED0C94D3560C94F9
:1003E000A31D0C94D5F50C944A2E0C94172E0C9446
:1003F000F7ED0C94DC2C0C94A6ED0C94E7F50C9422
:1004000064E80C9472E80C94BB560C9485E80C9448
:1004100029F70C94FE320C94952C0C9452E80C9411
:10042000D8F50C94A1270C94A5570C945F290C9433
:10043000B7564E414E494E495459494E46CDCCCC03
:100440003D0AD7233C17B7D13877CC2B329595E6A8
:10045000241FB14F0A000020410000C84200401C88
:100460004620BCBE4CCA1B0E5AAEC59D7400407AD5
:1004700010F35A00A0724E18090010A5D4E800002D
:10048000E87648170000E40B54020000CA9A3B00CB
:100490000000E1F505000080969800000040420F42
:1004A000000000A08601000000102700000000E806
:1004B00003000000006400000000000A00000000CB
:1004C000000100000000002C76D888DC674F08236C
:1004D000DFC1DFAE59E1B1B796E5E3E453C63AE6D2
:1004E00051997696E8E6C28426EB898C9B62ED40B2
:1004F0007C6FFCEFBC9C9F40F2BAA56FA5F4900501
:100500005A2AF75C936B6CF9676DC11BFCE0E40D34
:1005100047FEF520E6B500D0ED902E030094357728
:10052000050080841E080000204E0A000000C80C50
:10053000333333330F986E12831141EF8D211489B9
:100540003BE65516CFFEE6DB18D1844B381BF77C13
:100550001D901DA4BBE424203284725E228100C958
:10056000F124ECA1E53D274D323520500A4D3234BF
:10057000005072696E742050617573656400526535
:1005800073756D65005549205061757365004E6F38
:10059000204D61746368203A004D333033452D316E
:1005A000533635433455004D393939004D353032E5
:1005B0000A4D353030004D3330334530533231350C
:1005C000433855000A202A2A2A7265636461742E12
:1005D000646174615B305D203D004732380A473109
:1005E000204631303030205A313000556E737570EE
:1005F000706F72746564204F7074696F6E205365FC
:100600006C6563746564004D3139305335350A4784
:1006100032380A4732390A4D3430300A4D313034DD
:10062000533231350A4732380A4D3130395332317D
:10063000350A4D34323053310A4731583130305950
:1006400031303046353030300A47315A300A4D3576
:1006500030300A4D31313720536574205A204F66AF
:1006600066736574004731204631303030205A308F
:100670002E30004732380A473120463130303020A2
:100680005A302E30004D353030005A204F66667398
:100690006574203A202573004D353030005A204FC4
:1006A0006666736574203A202573004732385A0A0B
:1006B000473146313530305A302E30004732380A13
:1006C000473146313530305A302E30004D38340005
:1006D000473146313030305A302E30004732380AF8
:1006E000473146313030305A302E30005A204F6674
:1006F00066736574203A202573004D353030004D07
:10070000383400426567696E5377697463680072B4
:1007100065636461742E61646472203D3D0072659E
:10072000636461742E646174615B305D203D3D00E3
:1007300077616974776179203D3D000A202A2A2A71
:100740004E6F7A7A6C6554656D705374617475730D
:100750005B325D203D00434F4D4D554E4943415462
:10076000494F4E0044525952554E004552524F5235
:100770005300494E464F004543484F0047322F47EC
:10078000332062616420706172616D65746572739B
:100790000A00536C6565702E2E2E005A2050726F21
:1007A00062652050617374204265640A005A2050CB
:1007B000726F626520506173742042656400486FF7
:1007C0006D652058592046697273740A00486F6D30
:1007D00065205859204669727374004D31313720B5
:1007E00050726F6265206661696C65642E0A4732DB
:1007F000380A0070726F62655F72657769706500B4
:10080000473239205265747279696E670050726F91
:1008100062696E67204661696C6564004D313137ED
:1008200020426564206C6576656C696E6720666140
:10083000696C65642E0A4730205A31300A4D3330D6
:10084000302050323520533838300A4D3330302084
:100850005035302053300A4D33303020503235205F
:10086000533838300A4D3330302050353020533033
:100870000A4D3330302050323520533838300A4D4D
:10088000333030205035302053300A473420533134
:100890000070726F62655F6661696C6564004D31FE
:1008A000313720426564206C6576656C696E67201F
:1008B000646F6E652E00205A3A200020593A2000BD
:1008C00042656420583A20004D65736820706F6956
:1008D0006E742063616E6E6F742062652072657342
:1008E0006F6C7665640A004D302F3120427265616D
:1008F0006B2043616C6C656400436F6E74696E7548
:1009000065004D302F3120427265616B2043616C70
:100910006C6564004E6F204D6F76652E00456E64E9
:100920002066696C65206C6973740A0042656769AA
:100930006E2066696C65206C6973740A0052657379
:10094000756D6520534400286E6F2066696C6529BB
:100950000043757272656E742066696C653A20009A
:100960002E0A0044656C6574696F6E206661696C5F
:1009700065642C2046696C653A200046696C6520E8
:1009800064656C657465643A005072696E742074B5
:10099000696D653A20000A53746174733A204669A0
:1009A0006C616D656E7420757365643A20002C204F
:1009B0004C6F6E67657374206A6F623A2000546FE3
:1009C00074616C2074696D653A20005374617473AE
:1009D0003A20002C204661696C65643A20002C2086
:1009E00046696E69736865643A20005072696E7476
:1009F000733A200053746174733A20004520436FAA
:100A00006F6C696E672E2E2E0045204865617469F3
:100A10006E672E2E2E006F666600770772076B07D3
:100A20006407560744454255473A004D313133205B
:100A3000530042656420436F6F6C696E672E2E2EE3
:100A4000004265642048656174696E672E2E2E0031
:100A50006F6B004348414D4245525F54454D5045F0
:100A6000524154555245004D4F54494F4E5F4D4FE2
:100A700044455300544845524D414C5F50524F54E9
:100A8000454354494F4E004155544F5245504F52E3
:100A9000545F53445F5354415455530050524F4D8B
:100AA00050545F535550504F525400454D45524796
:100AB000454E43595F5041525345520043415345BF
:100AC0005F4C494748545F4252494748544E45534A
:100AD0005300544F47474C455F4C494748545300D7
:100AE000534F4654574152455F504F57455200426D
:100AF00055494C445F50455243454E54004C455671
:100B0000454C494E475F44415441005A5F50524F53
:100B10004245004155544F4C4556454C00505249B2
:100B20004E545F4A4F420050524F47524553530074
:100B30004155544F5245504F52545F54454D50000B
:100B4000564F4C554D455452494300454550524F20
:100B50004D0042494E4152595F46494C455F5452FF
:100B6000414E534645520053455249414C5F584F00
:100B70004E5F584F4646004649524D574152455FD9
:100B80004E414D453A4D61726C696E20322E305F98
:100B900044573320544D33442053534D444E422048
:100BA000534F555243455F434F44455F55524C3A6E
:100BB00068747470733A2F2F6769746875622E6356
:100BC0006F6D2F496E73616E6974794175746F6DC5
:100BD0006174696F6E2F4D61726C696E2F747265EE
:100BE000652F437265616C6974795F4D61726C69E0
:100BF0006E322E302E782050524F544F434F4C5F60
:100C000056455253494F4E3A312E30204D414348BC
:100C1000494E455F545950453A544D334420313084
:100C2000532050726F2045585452554445525F43EB
:100C30004F554E543A3120555549443A63656465E1
:100C4000326132662D343161322D343734382D39EA
:100C50006231322D63353563363266333637666638
:100C60000A002F2F20003F4A206F7574206F6620E6
:100C700072616E67652028302E303120746F20300D
:100C80002E33290A0020466C6F773A200050726F8D
:100C90007465637465642050696E0A0050726F62F7
:100CA00065205A204F66667365743A2000496E7657
:100CB000616C69642065787472756465720A0020DD
:100CC000643A0020693A0020703A0020643A00201B
:100CD000693A0020703A0064697300656E00432928
:100CE0000A0061626C656420286D696E2074656D10
:100CF000702000436F6C642065787472756465734E
:100D00002061726520004F4646004F4E0046696CD8
:100D1000616D656E742072756E6F75742064697391
:100D200074616E636520286D6D293A200046696CF8
:100D3000616D656E742072756E6F757420004D65FF
:100D4000736820706F696E742063616E6E6F7420BB
:100D50006265207265736F6C7665640A004D34328B
:100D60003120696E636F72726563742070617261A5
:100D70006D657465722075736167650A004F6666FC
:100D800073657473204170706C696564004572729C
:100D90003A20546F6F206661722100546F6F206695
:100DA00061722066726F6D207265666572656E6332
:100DB0006520706F696E740A00454550524F4D2092
:100DC0004F4B0A004572726F722077726974696EB8
:100DD0006720746F20454550524F4D210A00363729
:100DE00026033C3D380E2E303E121A1C1808440AC9
:100DF000FF430809070001627573793A2070617535
:100E000073656420666F7220696E7075740A006283
:100E10007573793A2070617573656420666F72200E
:100E2000757365720A00627573793A2070726F6328
:100E3000657373696E670A007061757365004D367E
:100E40003030200A204D313137200A002066696C8D
:100E5000616D656E745F72756E6F75742000666982
:100E60006C616D656E745F72756E6F757420540081
:100E700046696C616D656E7452756E6F7574205441
:100E80000053544F505045442E20005072696E74E8
:100E900065722073746F707065642064756520746A
:100EA0006F206572726F72732E20466978207468A5
:100EB00065206572726F7220616E642075736520A3
:100EC0004D39393920746F20726573746172742ED4
:100ED000202854656D706572617475726520697340
:100EE0002072657365742E205365742069742061C7
:100EF000667465722072657374617274696E6729B5
:100F00000A004E6F20436865636B73756D207769C7
:100F10007468206C696E65206E756D6265722C2038
:100F20004C617374204C696E653A20004E6F20430B
:100F30006865636B73756D2077697468206C696E82
:100F400065206E756D6265722C204C617374204C47
:100F5000696E653A2000636865636B73756D206D1B
:100F600069736D617463682C204C617374204C69E3
:100F70006E653A20004C696E65204E756D62657233
:100F8000206973206E6F74204C617374204C696EFD
:100F900065204E756D6265722B312C204C61737427
:100FA000204C696E653A20004D313130007761691F
:100FB000740A004D313137004D33310053442072F3
:100FC000656164206572726F720A00446F6E6520FD
:100FD0007072696E74696E672066696C650A004B91
:100FE000494C4C2063617573656420627920746F8D
:100FF0006F206D75636820696E6163746976652022
:1010000074696D65202D2063757272656E7420633E
:101010006F6D6D616E643A20002020506C616E6EC1
:10102000657242756666657242797465733A20002E
:101030002046726565204D656D6F72793A200043D8
:101040006F6D70696C65643A20536570202038209C
:10105000323031390A00207C20417574686F723A51
:101060002054696E794D616368696E657333440A13
:1010700000323031392D30372D333000204C617340
:101080007420557064617465643A2000322E305FBC
:101090004457330A004D61726C696E0020536F66CD
:1010A00074776172652052657365740A0020576118
:1010B000746368646F672052657365740A00204228
:1010C000726F776E206F75742052657365740A00B5
:1010D0002045787465726E616C2052657365740A80
:1010E00000506F77657255700A0073746172740AEC
:1010F000006175746F25632E67006572726F7220D0
:1011000077726974696E6720746F2066696C650A0E
:1011100000446F6E6520736176696E672066696C46
:10112000652E0A004D323900205A3A0020593A0003
:1011300020583A00656E6473746F70732068697428
:101140003A200047323858590043616E6E6F742060
:101150006F70656E2073756264697220005344205D
:1011600063617264206F6B0A006F70656E526F6FFF
:1011700074206661696C65640A00766F6C756D65D4
:101180002E696E6974206661696C65640A00534457
:1011900020696E6974206661696C0A004D32340002
:1011A0004D32332025730057726974696E6720745D
:1011B0006F2066696C653A20002E0A006F70656EBC
:1011C000206661696C65642C2046696C653A200074
:1011D0002E0A006F70656E206661696C65642C2054
:1011E00046696C653A200046696C652073656C65DC
:1011F000637465640A002053697A653A2000466981
:101200006C65206F70656E65643A20006672657368
:101210006800646F696E67002066696C653A20003B
:101220004E6F772000454E4420535542524F55543F
:10123000494E450A002220706F73002220706172AF
:10124000656E743A2200535542524F5554494E45EB
:101250002043414C4C207461726765743A220074DB
:101260007279696E6720746F2063616C6C2073758E
:10127000622D67636F64652066696C6573207769AA
:10128000746820746F6F206D616E79206C6576656F
:101290006C732E204D4158206C6576656C20697307
:1012A0003A310A005344207072696E74696E672087
:1012B0006279746520004E6F742053442070726907
:1012C0006E74696E670A00496E76616C69642065A8
:1012D000787472756465720A007C3C3E5E2B3D3FFB
:1012E0002F5B5D3B2C2A225C000050726F62696E9E
:1012F0006720506F696E742025692F2569002E0ABA
:10130000002F0050726F62696E67206D65736820F0
:10131000706F696E742000202844525952554E292E
:1013200000473239204175746F20426564204C6556
:1013300076656C696E67003F20284C2C522C462C39
:101340004229206F7574206F6620626F756E64731A
:101350002E0A003F2856296572626F7365206C65FE
:1013600076656C20697320696D706C617573696254
:101370006C652028302D34292E0A00426164205AE1
:101380002076616C75650A004E6F2062696C696E2B
:1013900065617220677269640A0046696E697368E4
:1013A0006564210A00206F662000205A0020590041
:1013B000476F696E6720746F3A20580043570A00E0
:1013C000206469723A0020616E676C653A0053745C
:1013D000617274207261646975733A00506F736949
:1013E00074696F6E696E67207468652070726F62D1
:1013F000652E2E2E0A003F4E756D626572206F6657
:10140000206C65677320696E206D6F76656D656E03
:1014100074206E6F7420706C61757369626C6520E6
:1014200028302D3135292E0A003F2028582C5929E3
:10143000206F7574206F6620626F756E64732E0A5C
:10144000003F53616D706C652073697A65206E6F23
:101450007420706C61757369626C652028342D3559
:1014600030292E0A004D3438205A2D50726F626593
:10147000205265706561746162696C697479205489
:101480006573740A003F2856296572626F73652080
:101490006C6576656C20697320696D706C6175731D
:1014A00069626C652028302D34292E0A00486F6D42
:1014B0006520257325732573204669727374002097
:1014C00046697273740A00486F6D652000220A0035
:1014D000556E6B6E6F776E20636F6D6D616E643AE3
:1014E00020220020746F6F206C6F6E672065787407
:1014F000727573696F6E2070726576656E7465645F
:101500000A0020636F6C6420657874727573696F6C
:101510006E2070726576656E7465640A0024F4D47A
:101520003050C38E20C2A24017828B7011127A9164
:101530000D816CD90AA861E108C75866076151435B
:10154000061E4B5D05C145A7041A411104093D98CB
:1015500003713931034036DB0265339102D43054D4
:1015600002802E1D02632CEE01752AC501B028A051
:1015700001102781018F2564012B244B01E02234C7
:1015800001AC211F018D200D01801FFC00841EED88
:1015900000971DDF00B81CD200E61BC600201BBC54
:1015A00000641AB200B219A8000A19A0006A1899BA
:1015B00000D117910040178B00B516840031167EBC
:1015C00000B31579003A157300C7146F0058146AF8
:1015D00000EE1366008813630025135E00C7125BDC
:1015E000006C12570015125400C111510070114FB8
:1015F0000021114B00D61049008D104700461044C1
:101600000002104200C00F4000800F3E00420F3C1D
:1016100000060F3B00CB0E3800930E37005C0E35F2
:1016200000270E3400F30D3200C10D3100900D3053
:1016300000600D2E00320D2D00050D2C00D90C2B55
:1016400000AE0C2900850C29005C0C2700350C2706
:10165000000E0C2600E80B2400C40B2400A00B2372
:10166000007D0B23005A0B2100390B2100180B20A1
:1016700000F80A1F00D90A1E00BB0A1E009D0A1DA1
:1016800000800A1D00630A1C00470A1B002C0A1B6D
:1016900000110A1A00F7091A00DD091900C4091916
:1016A00000AB091900920917007B0918006309179C
:1016B000004C09160036091600200916000A091503
:1016C00000F5081500E0081400CC081400B8081450
:1016D00000A4081400900813007D0812006B081382
:1016E000005808120046081200340811002308119F
:1016F000001208110001081100F0071000E00710A7
:1017000000D0071000C0071000B0070F00A107109D
:101710000091070E0083070F0074070F0065070E86
:101720000057070E0049070E003B070D002E070E5D
:101730000020070D0013070D0006070D00F9060C29
:1017400000ED060D00E0060C00D4060C00C8060CE7
:1017500000BC060C00B0060C00A4060B0099060C99
:10176000008D060B0082060B0077060B006C060B43
:101770000061060A0057060B004C060A0042060AE2
:101780000038060A002E060A0024060A001A060A75
:10179000001006090007060A00FD050900F4050906
:1017A00000EB050900E2050900D9050900D005098B
:1017B00000C7050900BE050900B5050800AD05080C
:1017C00000A50509009C050800940508008C050883
:1017D00000840508007C050800740508006C0507F6
:1017E00000650508005D050700560508004E050761
:1017F00000470507004005080038050700310507C8
:10180000002A050700230507001C0506001605072A
:10181000000F0507000805060002050700FB040687
:1018200000F5040700EE040600E8040600E20407E1
:1018300000DB040600D5040600CF040600C9040638
:1018400000C3040600BD040600B7040600B1040589
:1018500000AC040600A6040600A00405009B0406D4
:101860000095040500900406008A0405008504051F
:1018700000800406007A0405007504050070040564
:10188000006B04050066040500610405005C0405A6
:101890000057040500520405004D040500480405E6
:1018A00000430405003E0404003A04050035040525
:1018B00000300404002C0405002704040023040560
:1018C000001E0404001A0404001604050011040498
:1018D000000D0404000904050004040400000404CD
:1018E00000FC030400F8030400F4030400F0030404
:1018F00000EC030400E8030400E4030400E0030434
:1019000000DC030400D8030400D4030400D0030463
:1019100000CC030400C8030300C503030024F4043F
:10192000D9201BC40C5C0E9804C4095F02650771C2
:1019300001F405F900FB04B30048048700C1036902
:10194000005803550003034500BE023A00840231EB
:101950000053022A002902250004022000E4011C91
:1019600000C8011900AF0117009801140084011389
:1019700000710110006101100051010E0043010DC2
:101980000036010B002B010B0020010B0015010993
:10199000000C01090003010800FB000800F3000827
:1019A00000EB000700E4000600DE000600D8000699
:1019B00000D2000600CC000500C7000500C20005EB
:1019C00000BD000400B9000400B5000400B100042B
:1019D00000AD000400A9000400A5000300A200035C
:1019E000009F0004009B0003009800030095000284
:1019F0000093000300900003008D0002008B0003A1
:101A000000880002008600020084000300810002BA
:101A1000007F0002007D0002007B000200790002CE
:101A200000770001007600020074000200720001DD
:101A300000710002006F0002006D0001006C0002E6
:101A4000006A0001006900020067000100660001F1
:101A500000650001006400020062000100610001F5
:101A600000600001005F0002005D0001005C0001F9
:101A7000005B0001005A00010059000100580001FC
:101A800000570001005600010055000100540001FC
:101A900000530000005300010052000100510001FA
:101AA00000500001004F0001004E0000004E0001F8
:101AB000004D0001004C0001004B0000004B0001F4
:101AC000004A0001004900010048000000480001F0
:101AD00000470001004600000046000100450000EC
:101AE00000450001004400010043000000430001E4
:101AF00000420000004200010041000000410001DE
:101B000000400001003F0000003F0001003E0000D7
:101B1000003E0001003D0000003D0001003C0000CF
:101B2000003C0000003C0001003B0000003B0001C5
:101B3000003A0000003A00010039000000390001BD
:101B400000380000003800000038000100370000B5
:101B500000370001003600000036000000360001AA
:101B600000350000003500000035000100340000A1
:101B70000034000000340001003300000033000096
:101B8000003300010032000000320000003200018A
:101B90000031000000310000003100010030000081
:101BA0000030000000300001002F0000002F000076
:101BB000002F0000002F0001002E0000002E00006A
:101BC000002E0001002D0000002D0000002D00005F
:101BD000002D0001002C0000002C0000002C000053
:101BE000002C0001002B0000002B0000002B000047
:101BF000002B0001002A0000002A0000002A00003B
:101C0000002A00010029000000290000002900002E
:101C10000029000000290001002800000028000021
:101C20000028000000280000002800010027000014
:101C30000027000000270000002700000027000107
:101C400000260000002600000026000000260000FC
:101C500000260001002500000025000000250000EE
:101C600000250000002500000025000100240000E0
:101C700000240000002400000024000000240001D3
:101C800000230000002300000023000000230000C8
:101C900000230000002300000023000100220000B8
:101CA00000220000002200000022000000220000AC
:101CB000002200010021000000210000002100009E
:101CC000002100000021000000210000002100018F
:101CD0000020000000200000002000000020000084
:101CE0000020000000200000002000000020000173
:101CF000001F0000001F0000001F0000001F000068
:101D0000001F0000001F0000001F0001001E000057
:101D1000001E0000001E0000001E0000000437002E
:101D2000001E290000511B0000581000001009007F
:101D300000CC0400007802000041010000626564EC
:101D4000002C2073797374656D2073746F707065E7
:101D50006421204865617465725F49443A200042FD
:101D600065642048656174696E67204661696C65C9
:101D7000640048656174696E67206661696C6564BA
:101D80000042454420544845524D414C2052554E46
:101D90004157415900546865726D616C2052756EEF
:101DA000617761790045312048656174696E67200B
:101DB0004661696C65640048656174696E67206698
:101DC00061696C656400453120544845524D414C71
:101DD0002052554E4157415900546865726D616CEF
:101DE0002052756E617761790057616974696E6719
:101DF00020666F72206865617475702E0A004C65EC
:101E00006176696E6720473236003F5370656369BB
:101E10006669656420582C5920636F6F7264696E1F
:101E2000617465206F7574206F6620626F756E64D3
:101E3000732E0A003F28522965706561742076610F
:101E40006C7565206E6F7420706C61757369626C5F
:101E5000653B206D757374206265206174206C652C
:101E600061737420312E0A003F2852296570656124
:101E700074206D7573742062652073706563696684
:101E8000696564207768656E206E6F74207573696C
:101E90006E6720616E204C43442E0A003F537065EC
:101EA000636966696564206E6F7A7A6C6520746513
:101EB0006D7065726174757265206E6F7420706CE0
:101EC00061757369626C652E0A003F5370656369C2
:101ED000666965642066696C616D656E74207369FE
:101EE0007A65206E6F7420706C61757369626C65C1
:101EF0002E0A003F537065636966696564207072DD
:101F0000696D65206C656E677468206E6F742070F3
:101F10006C61757369626C652E0A003F5072696D61
:101F200065206C656E677468206D757374206265DA
:101F300020737065636966696564207768656E20E3
:101F40006E6F74207573696E6720616E204C434418
:101F50002E0A003F537065636966696564206E6F81
:101F60007A7A6C652073697A65206E6F7420706C64
:101F700061757369626C652E0A003F526574726107
:101F80006374696F6E204D756C7469706C696572ED
:101F9000206D75737420626520737065636966696E
:101FA00065642E0A003F5370656369666965642045
:101FB00052657472616374696F6E204D756C7469DB
:101FC000706C696572206E6F7420706C61757369D6
:101FD000626C652E0A003F537065636966696564CB
:101FE000206C6179657220686569676874206E6F1E
:101FF0007420706C61757369626C652E0A004329E8
:102000002E0A003F537065636966696564206265E6
:10201000642074656D7065726174757265206E6F91
:102020007420706C61757369626C65202834302D82
:1020300000473236207374617274696E672E2E2EDB
:102040000A004F46460A0046616465204865696794
:1020500068742000426564204C6576656C696E6723
:1020600020004661696C656420746F20656E616252
:102070006C6520426564204C6576656C696E670A04
:1020800000496E76616C6964206D6573682E0A0084
:102090002F2F616374696F6E3A00627574746F6E8E
:1020A00000656E640070726F6D70745F0073686FAE
:1020B00077004D38373620526573706F6E64696EE5
:1020C000672050524F4D50545F00554E4B4E4F5766
:1020D0004E2053544154450047434F44455F494EB9
:1020E000464F004C43445F50415553455F52455362
:1020F000554D450046494C414D454E545F52554E55
:102100004F55545F434F4E54494E55450046494C38
:10211000414D454E545F52554E4F5554004D32344B
:1021200000436F6E74696E75650044697361626C1B
:102130006552756E6F7574005075726765204D6FCE
:1021400072650050617573656400706175736564D4
:1021500000486F74656E6420746F6F20636F6C64E9
:102160000A00506175736500507265737320627563
:1021700074746F6E20286F72204D313038292074AE
:102180006F20726573756D650A00496E73657274B0
:102190002066696C616D656E7420616E642070727A
:1021A00065737320627574746F6E20286F72204D92
:1021B000313038290A00436F6E74696E75650052BC
:1021C000656865617420446F6E650052656865617D
:1021D00074696E672E2E2E00526568656174696E93
:1021E000670048656174657254696D656F75740048
:1021F0005265686561740048656174657254696D03
:10220000656F757400507265737320627574746FB6
:102210006E20286F72204D3130382920746F20686D
:10222000656174206E6F7A7A6C650A004E6F7A7AF7
:102230006C65205061726B656400436F6E74696EEB
:102240007565004E6F7A7A6C65205061726B6564BB
:1022500000486F74656E6420746F6F20636F6C64E8
:102260000A00726573756D656400626567696E006A
:10227000436F6E74696E75650044697361626C6565
:1022800052756E6F75740050757267654D6F72652B
:1022900000506175736564004C6F61642046696C21
:1022A000616D656E7400436F6E74696E7565004C88
:1022B0006F61642046696C616D656E7420540049DD
:1022C0006E736572742066696C616D656E742061F1
:1022D0006E6420707265737320627574746F6E2003
:1022E000286F72204D313038290A00526573756DA0
:1022F0006500526573656E643A200043616E6E6FCF
:1023000074206F70656E2073756264697220002599
:1023100069730025696D202569730025696820258A
:10232000696D202569730025696420256968202569
:10233000696D202569730025697920256964202548
:1023400069682025696D20256973002364656669C5
:102350006E652044454641554C545F0000626564FB
:10236000004B6420004B6920004B70200050494412
:10237000204175746F74756E652066696E69736847
:102380006564212050757420746865206C617374D5
:10239000204B702C204B6920616E64204B642063BD
:1023A0006F6E7374616E74732066726F6D206265F8
:1023B0006C6F7720696E746F20436F6E6669677506
:1023C000726174696F6E2E680A005049442041752D
:1023D000746F74756E65206661696C656421207424
:1023E000696D656F75740A00453120544845524D3A
:1023F000414C2052554E41574159004245442054CA
:102400004845524D414C2052554E41574159005478
:102410006865726D616C2052756E617761790045F7
:10242000312048656174696E67204661696C656436
:10243000004265642048656174696E672046616981
:102440006C65640048656174696E67206661696CDB
:10245000656400504944204175746F74756E652041
:102460006661696C6564212054656D706572617484
:1024700075726520746F6F20686967680A00204B69
:10248000643A2000204B693A2000204B703A20002B
:102490000A20436C617373696320504944200A0029
:1024A000204B643A2000204B693A2000204B703AC0
:1024B00020000A204E6F206F76657273686F6F740C
:1024C0000A002054753A2000204B753A2000206DF8
:1024D00061783A2000206D696E3A200020643A202D
:1024E0000020626961733A200050494420417574AC
:1024F0006F74756E652073746172740A005049447C
:10250000204175746F74756E65206661696C6564D1
:10251000212054656D706572617475726520746FE9
:102520006F20686967680A00504944204175746FDC
:1025300074756E65206661696C6564212042616412
:10254000206578747275646572206E756D6265724F
:102550000A0070012C0190012701B0012201C00185
:102560001D01F00118011002130130020E0160027A
:10257000090190020401C002FF000003FA004003B9
:10258000F5008003F000D003EB002004E6007004A7
:10259000E100E004DC004005D700C005D2004006A1
:1025A000CD00D006C8008007C3003008BE00F00888
:1025B000B900C009B400B00AAF00B00BAA00D00C3B
:1025C000A500000EA000500F9B00C01096005012F6
:1025D000910000148C00C0158700B0178200B0195C
:1025E0007D00D01B7800001E730040206E009022FA
:1025F0006900F024640040275F0090295A00E02B16
:102600005500102E500020304B0010324600E033B1
:10261000410090353C001037370070383200A03947
:102620002D00B03A2800A03B2300603C1E00103D66
:102630001900903D1400103E0F00703E0A00C03E8D
:102640000500003F0000403FFBFF803FF6FFC03F1A
:10265000F1FF202D20496E76616C696420657874E5
:102660007275646572206E756D62657220210A0054
:102670001000C90210012C01400122017001180153
:10268000B0010E01F00104015002FA00B002F000A6
:102690003003E600D003DC009004D2007005C800CF
:1026A000A006BE000008B400B009AA00D00BA0002C
:1026B000600E960060118C000015820020197800D1
:1026C000C01D6E00A0226400B0275A00902C50005C
:1026D00000314600E0343C0010383200903A2800C7
:1026E000603C1E00A03D1400803E0A00203F000018
:1026F000453120544845524D414C2052554E41578A
:1027000041590042454420544845524D414C2052C5
:10271000554E4157415900546865726D616C2052A5
:10272000756E61776179004531204572723A204DAE
:10273000415854454D50004572723A204D4158540D
:10274000454D5020424544004D415854454D502080
:1027500074726967676572656400453120457272FD
:102760003A204D494E54454D50004572723A204D25
:10277000494E54454D5020424544004D494E544524
:102780004D5020747269676765726564000A0A00BB
:1027900020205A5F4D494E3A002020595F4D494E46
:1027A0003A002020585F4D494E3A004D38342058A9
:1027B0002059205A204500202F002042403A002076
:1027C000403A0020573A0020573A005A5F53544F7E
:1027D000505F50494E005A5F535445505F50494E28
:1027E000005A5F4D494E5F50494E005A5F454E4179
:1027F000424C455F50494E005A5F4449525F504930
:102800004E005A5F43535F50494E00595F53544F37
:10281000505F50494E00595F535445505F50494EE8
:1028200000595F4D494E5F50494E00595F454E413A
:10283000424C455F50494E00595F4449525F5049F0
:102840004E00595F43535F50494E00585F53544FF9
:10285000505F50494E00585F535445505F50494EA9
:1028600000585F4D494E5F50494E00585F454E41FC
:10287000424C455F50494E00585F4449525F5049B1
:102880004E00585F43535F50494E0053535F5049C9
:102890004E00534552564F335F50494E00534552F8
:1028A000564F325F50494E00534552564F315F509C
:1028B000494E00534552564F305F50494E005344E5
:1028C00053530053445F4445544543545F50494E6D
:1028D0000053434B5F50494E0052414D50535F44AB
:1028E000395F50494E0052414D50535F44385F505C
:1028F000494E0052414D50535F4431305F50494E74
:10290000004D4F53495F50494E004D4F534645547B
:102910005F445F50494E004D49534F5F50494E0050
:102920004D4158363637355F53535F50494E004C52
:1029300045445F50494E004845415445525F424529
:10294000445F50494E004845415445525F305F5006
:10295000494E0046494C5F52554E4F55545F5049C1
:102960004E0046414E315F50494E0046414E5F5049
:10297000494E0045315F535445505F50494E004524
:10298000315F454E41424C455F50494E0045315FF5
:102990004449525F50494E0045315F43535F5049AF
:1029A0004E0045305F535445505F50494E0045300E
:1029B0005F454E41424C455F50494E0045305F44B3
:1029C00049525F50494E0045305F43535F50494E76
:1029D00000455F4D5558325F50494E00455F4D559B
:1029E00058315F50494E00455F4D5558305F504952
:1029F0004E004156525F53535F50494E004156526C
:102A00005F53434B5F50494E004156525F4D4F5309
:102A1000495F50494E004156525F4D49534F5F50F8
:102A2000494E0054454D505F4245445F50494E0069
:102A300054454D505F315F50494E0054454D505FF5
:102A4000305F50494E0046494C57494454485F5006
:102A5000494E005458440052584400202020002081
:102A60002020416E616C6F6720696E203D20253506
:102A70006C64003C756E757365642F756E6B6E6F5C
:102A8000776E3E002028412532642920200025331E
:102A9000642000257350494E3A20004F75747075BC
:102AA00074203D2000496E70757420203D20004147
:102AB0006E616C6F6720696E203D2025356C640067
:102AC00070726F746563746564200020284125323C
:102AD00064292020002533642000257350494E3A94
:102AE0002000572A0001532A0101462A3B003B2AB5
:102AF0004300302A4500232A4400162A3201092ABD
:102B00003301FD293401F2293501E7292801DC29A7
:102B10002A01D1292C01C7292A01BC291C01AE296F
:102B20001801A2291A0198292C018D2922017F2937
:102B30001E01732924016B29090162290701532908
:102B4000020146290A01372908012F290D012029F0
:102B50004201172932010A29070101293301F3280B
:102B60000A01E6280801D9280901D1283401C3281F
:102B70003101BE283501B3280B01A82806019D2884
:102B80000501922804018B28350182283501782817
:102B900037016B28260161280301562836014B288E
:102BA00003014228310138283D012B283801212812
:102BB0000E0116283C010B280E0102282801F827D7
:102BC0003001EB273E01E1271201D6272E01CB274A
:102BD0001201446F6E652E0A00534552564F206E07
:102BE0006F74207365742075702E0A004D34332085
:102BF000576169742043616C6C656400436F6E7447
:102C0000696E7565004D34332057616974204361E6
:102C10006C6C6564005761746368696E67207069E5
:102C20006E730A0064697300656E0061626C6564AE
:102C30000A00656E6473746F70206D6F6E69746FD7
:102C4000722000204500205A00205900204D3932C2
:102C5000205800205A00205900580020204D61784B
:102C60003A2000205A00205900580020204D696E5B
:102C70003A2000536F667420656E6473746F7073CE
:102C80003A20004732380020496E76616C69642032
:102C90006578747275646572200044696666657251
:102CA0003A200046726F6D5374703A005374657029
:102CB0007065723A00556E4C6576656C3A004C65ED
:102CC00076656C65643A005261773A2020202000D6
:102CD0000A4C6F676963616C3A004361703A005057
:102CE000726F6265205A204F66667365743A2000E1
:102CF00050726F62652059204F66667365743A2082
:102D00000050726F62652058204F66667365743A92
:102D100020003F59206F7574206F662072616E67C6
:102D2000652028302D33313020746F203331302925
:102D30000A003F58206F7574206F662072616E67BD
:102D4000652028302D33313520746F2033313529FB
:102D50000A003F5A206F7574206F662072616E679B
:102D60006520282D323020746F203230290A00224D
:102D70000A00656E7175657565696E6720220020B1
:102D800042002050006F6B006F70656E0054524916
:102D9000474745524544003A200066696C616D65BD
:102DA0006E74007A5F6D696E00795F6D696E007890
:102DB0005F6D696E005265706F7274696E67206531
:102DC0006E6473746F70207374617475730A00207D
:102DD0005A3A0020593A0020436F756E7420583AD1
:102DE0000020453A00205A3A0020593A00583A004B
:102DF00020746F6F206C6F6E6720657874727573C6
:102E0000696F6E2070726576656E7465640A002065
:102E1000636F6C6420657874727573696F6E20706F
:102E2000726576656E7465640A000000000000003B
:102E3000000000000000000048420000484200007E
:102E400080405761726E696E673A20486F6D696E97
:102E5000672042756D702044697669736F72203CFB
:102E600020310A000202040000A0400000A040003F
:102E700000004000809D4300009B430000C843FFCA
:102E8000FFFF544D3344203130532050726F205295
:102E9000656164792E005072696E74696E672E2EBA
:102EA0002E005072696E7420506175736564006302
:102EB000616E63656C005072696E742041626F725E
:102EC0007465640055492041626F727400726573C5
:102ED000756D65004D32340000809D4300009B43BA
:102EE0000000C843000000000000000000000000D7
:102EF000290A002062797465733B206372632000A5
:102F000053657474696E67732053746F72656420BF
:102F10002800454550524F4D206461746173697AB1
:102F200065206572726F722E0A00290A002062798C
:102F30007465733B2063726320002073746F726545
:102F4000642073657474696E677320726574726946
:102F500065766564202800202863616C63756C6168
:102F600074656429210A0020213D20004545505206
:102F70004F4D20435243206D69736D617463682027
:102F80002D202873746F7265642920002053697A9C
:102F9000653A2000496E6465783A2000204D6172E0
:102FA0006C696E3D563730290A00454550524F4DE9
:102FB0002076657273696F6E206D69736D617463DD
:102FC000682028454550524F4D3D00000021002407
:102FD0000027002A002D003000330001010000040A
:102FE0000107010A0100002200250028002B002E05
:102FF000003100340002010000050108010B01004E
:103000000020002300260029002C002F00320000A1
:103010000100000301060109010505050507050872
:10302000080808020202020A0A080804040404014B
:10303000010101010101010303030303030303046D
:103040000707070C0C0C0C0C0C0C0C0202020206FD
:10305000060606060606060B0B0B0B0B0B0B0B01ED
:103060000210202008081020401020408002010299
:103070000108040201010204081020408080402061
:10308000100804020180040201804020100804029C
:10309000010804020101020408102040800102041A
:1030A000081020408000000A0B02090C0D0E0807D2
:1030B0000304010000000000000000000000000008
:1030C0000000000000000000000000000000000000
:1030D00000121110000000000000000000000000BD
:1030E000000000000000000000000050726F6269E4
:1030F0006E67204661696C65640A0050726F626990
:103100006E67204661696C6564000A20696E6974A7
:10311000207A70726F62655F7A6F6666736574207D
:103120003D2000454550524F4D20496E69746961FC
:103130006C697A65640A0048617264636F646564EF
:103140002044656661756C742053657474696E679C
:1031500073204C6F616465640A00EE020000EE02A9
:103160000000640000003C0000000000FA43000082
:10317000FA430000204100008C420000A042000001
:10318000A0420000C84300000C433A0A0020204D32
:10319000363033200020440020204D34313220537B
:1031A0000046696C616D656E742072756E6F757422
:1031B0002073656E736F723A0A002055004C00460A
:1031C000696C616D656E74206C6F61642F756E6CD7
:1031D0006F6164206C656E677468733A0A00202022
:1031E0004D383531205A0020204D383531205900D6
:1031F00020204D3835312058005A2D50726F6265AD
:10320000204F66667365740020440020490020202A
:103210004D33303420500020440020490020204D00
:103220003330312050005049442073657474696E06
:1032300067733A0A00204A0020204732392057207D
:103240004900205A0020204D34323020530041756F
:10325000746F20426564204C6576656C696E673AD0
:103260000A00205A0020590020204D3230362058C4
:1032700000486F6D65206F66667365743A0A0020BA
:103280004A0020540020530020204D323035204287
:1032900000204A3C6A756E635F6465763E00416457
:1032A00076616E6365643A20423C6D696E5F73655A
:1032B000676D656E745F74696D655F75733E2053ED
:1032C0003C6D696E5F66656564726174653E20542D
:1032D0003C6D696E5F74726176656C5F666565648E
:1032E000726174653E0020540020520020204D324F
:1032F0003034205000416363656C65726174696F9E
:103300006E2028756E6974732F7332293A20503CF1
:103310007072696E745F616363656C3E20523C72CB
:103320006574726163745F616363656C3E20543CD5
:1033300074726176656C5F616363656C3E0A002040
:103340004500205A0020590020204D3230312058AD
:10335000004D6178696D756D20416363656C6572C0
:103360006174696F6E2028756E6974732F733229CA
:103370003A0A00204500205A0020590020204D32F2
:1033800030332058004D6178696D756D2066656534
:103390006472617465732028756E6974732F732964
:1033A0003A0A0053746570732070657220756E69F7
:1033B000743A0A0020204D3230302044300A002078
:1033C000204D3230302044002044697361626C65C6
:1033D000640A0046696C616D656E7420736574746F
:1033E000696E67733A0020286D6D290020204732EE
:1033F00031202020203B20556E69747320696E2097
:103400006D6D00486F6D696E67204661696C65641B
:1034100000205400205200416363656C6572617442
:10342000696F6E3A20500050574D3A202025346481
:103430000050574D3A20202534640050574D3A2013
:10344000202534640050574D3A2020253464005024
:10345000574D3A20202534640050574D3A202025FE
:1034600034640050574D3A20202534640050574DA5
:103470003A20202534640050574D3A2020253464EA
:103480000050574D3A20202534640050574D3A20C3
:10349000202534640050574D3A20202534640050D4
:1034A000574D3A20202534640050574D3A202025AE
:1034B00034640050574D3A20202534640050574D55
:1034C0003A202025346400433A2000423A2000414B
:1034D0003A200020202020434F4D002020206E6FF6
:1034E0006E2D7374616E646172642050574D206D4F
:1034F0006F646500202020636F6D706172652069C4
:103500006E7465727275707420656E61626C65644C
:10351000002020206F766572666C6F7720696E746C
:1035200065727275707420656E61626C6564003AD4
:1035300020002020202054494D534B00423A2000C7
:10354000202020205443435200413A2000202020D4
:103550002054434352002020202043533A2000208F
:1035600020202057474D3A200050574D3A20202523
:1035700034640050574D3A202025346400470048F9
:1035800000000088008A008C00B300B4000000989E
:10359000009A009C00A800AA00AC0028012A012C77
:1035A000012020202054494D455200440045006E22
:1035B00000800081006F00B000B1007000900091A9
:1035C000007100A000A10072002001210173002001
:1035D000697320616C736F207469656420746F2057
:1035E000746869732070696E0054494D45523143C7
:1035F000000A202E002020002020506F72743A20F4
:10360000002E0A006F70656E206661696C65642C1F
:103610002046696C653A2000706F7765726F666648
:10362000004B494C4C45442E20005072696E746525
:10363000722068616C7465642E206B696C6C28293B
:103640002063616C6C6564210A006563686F3A00F1
:103650004572726F723A0042696C696E65617220E0
:103660004C6576656C696E6720477269643A0A003A
:103670005901910111241FBECFEFD1E2DEBFCDBFB2
:1036800000E00CBF18E0A0E0B2E0E6EDFFE302E0EE
:103690000BBF02C007900D92A434B107D9F72CE1FB
:1036A000A4E4B8E001C01D92A43EB207E1F71BE11B
:1036B000C9E3DBE100E006C021970109802FFE018C
:1036C0000F94141CC833D10780E00807A9F70F94A2
:1036D0003F060D94D91F0C9400002F923F924F92F9
:1036E0005F926F927F928F929F92AF92BF92CF9292
:1036F000DF92EF92FF920F931F93CF93DF93CDB79B
:10370000DEB7E3970FB6F894DEBF0FBECDBF809152
:103710000901817091E0982720916308921781F147
:1037200090936308811116C00E94CD598091CE16E6
:1037300083FF09C08FE993E00E943A4F61E080E087
:103740000F9400021DC060E081E00F94000288EB3E
:1037500093E014C00091CE1603FB002700F90E94ED
:103760005C598091CE16877F8093CE16002341F05E
:1037700060E081E00F94000281ED93E00E943A4FF7
:103780008091BB1381FF11C18091D0149091D1140D
:10379000891B8F70843008F008C18CE0E1E1F3E10F
:1037A000DE01119601900D928A95E1F78091431701
:1037B00090914417A0914517B091461788A799A7F3
:1037C000AAA7BBA79C01AD016091111370911213C0
:1037D00080911313909114130F941C1C6B017C01A6
:1037E0006093111370931213809313139093141317
:1037F0008091471790914817A0914917B0914A17A7
:103800008CA79DA7AEA7BFA79C01AD016091151322
:103810007091161380911713909118130F941C1C1C
:1038200068A379A38AA39BA36093151370931613BF
:10383000809317139093181380914B1790914C1706
:10384000A0914D17B0914E1788AB99ABAAABBBAB0B
:103850009C01AD016091191370911A1380911B1393
:1038600090911C130F941C1C4B015C016093191365
:1038700070931A1380931B1390931C13A701960146
:10388000C701B6010F9499152B013C0128A139A15C
:103890004AA15BA1CA01B9010F9499159B01AC0122
:1038A000C301B2010F941D1C2B013C01A501940121
:1038B000C501B4010F9499159B01AC01C301B2017C
:1038C0000F941D1C0F94CB1E9B01AC0160E070E0B7
:1038D00080E89FE30F94171D20915F0230916002F2
:1038E00040916102509162020F9499152DEC3CECCD
:1038F0004CEC5DE30F94991520E030E040E85EE386
:103900000F9499152B013C0120E030E040E85FE383
:103910000F94331587FFF1C3A3019201C701B601CC
:103920000F94991528A539A54AA55BA50F941D1CD0
:1039300060931113709312138093131390931413C5
:10394000A301920168A179A18AA19BA10F94991565
:103950002CA53DA54EA55FA50F941D1C60931513C6
:10396000709316138093171390931813A301920169
:10397000C501B4010F94991528A939A94AA95BA9D1
:103980000F941D1C6093191370931A1380931B13CB
:1039900090931C130E9478D38CE0FE013196A1E134
:1039A000B3E101900D928A95E1F78091620881114F
:1039B0000C94503780916008909161089C012F5FB2
:1039C0003F4F3093610820936008883E934010F485
:1039D0000C94503781E08093620810926108109235
:1039E00060088091CE11882309F498C30E94A1AD8C
:1039F000811194C380915F088F5F80935F088091ED
:103A00005F08853620F010925F081092CE11E09189
:103A1000CE118E2FEE0F990BAA0BBB0BFC01319729
:103A2000E730F10508F0A0C08827EE58FF4F8F4F10
:103A30000D94141C0E9499AD882309F495C081E06F
:103A40008093340284EE93E00E943A4F80E190E04C
:103A5000909353158093521585E08093461502E8A4
:103A60000093491584E190E1A0E0B0E080934A150D
:103A700090934B15A0934C15B0934D150E948DF962
:103A800081E09AE5909353158093521586E390E078
:103A9000909355158093541587E0809346150093B5
:103AA000491584E890E0A0E0B0E080934A15909337
:103AB0004B15A0934C15B0934D150E948DF952C033
:103AC0000E9499AD882309F44FC048C082EF93E06B
:103AD0000E943A4F81E09AE59093531580935215D6
:103AE00080E490E0909355158093541507E000937F
:103AF000461582E88093491584E890E0A0E0B0E0A4
:103B000080934A1590934B15A0934C15B0934D1587
:103B10000E948DF90093CE1127C080915E08882302
:103B200019F10E9499AD8823F9F00E94A1AD81118D
:103B30001BC0F7C20E9499AD8823B1F00E94A1ADCD
:103B4000811112C01CC30E94A1AD81110DC042E0C1
:103B500060E070E0CB010E94B7AD04C00E94A1AD4F
:103B6000811102C01092CE1180913402882309F491
:103B7000ACC28091CA119091CB11892B09F08FC1F1
:103B800080915B0890915C08892B09F01EC184E04C
:103B900096E0909353158093521580EA90E89093A5
:103BA00055158093541517E01093461502E80093BD
:103BB000491580EA90E0A0E0B0E080934A15909328
:103BC0004B15A0934C15B0934D150E948DF9809123
:103BD000060290910702A0910802B0910902009795
:103BE000A105B10511F5109253151092521515E06B
:103BF00010934615009349158AE890E1A0E0B0E0E3
:103C000080934A1590934B15A0934C15B0934D1586
:103C10000E948DF989E090E090935315809352159E
:103C2000109346150093491540C00196A11DB11D82
:103C3000F5E0B695A79597958795FA95D1F70197F1
:103C4000A109B109009731E0A307B10558F0B0937D
:103C50005315A093521590935515809354151093B6
:103C6000461507C0909353158093521585E08093B5
:103C7000461512E8109349158AE890E1A0E0B0E0FB
:103C800080934A1590934B15A0934C15B0934D1506
:103C90000E948DF988E090E090935315809352151F
:103CA00085E080934615109349158CE890E1A0E0DB
:103CB000B0E080934A1590934B15A0934C15B093A8
:103CC0004D150E948DF98091060290910702A091F6
:103CD0000802B09109020097E1E0AE07B10550F08B
:103CE000B0935315A0935215909355158093541586
:103CF00087E005C0909353158093521585E080931B
:103D0000461582E88093491588E890E1A0E0B0E08C
:103D100080934A1590934B15A0934C15B0934D1575
:103D20000E948DF98091060290910702A0910802ED
:103D3000B0910902BA2FA92F982F88270097F1E098
:103D4000AF07B10550F0B0935315A093521590935F
:103D500055158093541587E005C0909353158093B3
:103D6000521585E08093461512E81093491581EAB3
:103D700090E0A0E0B0E080934A1590934B15A0939B
:103D80004C15B0934D150E948DF980915B178823D7
:103D900019F082E090E002C083E090E09093531528
:103DA0008093521585E0809346151093491585E45C
:103DB00090E1A0E0B0E080934A1590934B15A0935A
:103DC0004C15B0934D150E948DF900915B08109130
:103DD0005C08053611057CF41093531500935215B9
:103DE00085E08093461582E88093491580E090E154
:103DF000A0E0B0E011C0C80184569109909353151A
:103E00008093521585E08093461582E8809349158A
:103E100081E090E1A0E0B0E080934A1590934B15CB
:103E2000A0934C15B0934D150E948DF90F5F1F4F55
:103E300010935C0800935B08093C110564F180E075
:103E400094E00E943A4F81E090E09093CB118093F0
:103E5000CA118093340281E09AE5909353158093C0
:103E600052158DE290E0909355158093541587E09C
:103E70008093461582E88093491584E890E0A0E09D
:103E8000B0E080934A1590934B15A0934C15B093D6
:103E90004D150E948DF9109262080C945037809154
:103EA000D0149091D114891B8F7009F092C10E9497
:103EB0003EB781118EC18091CE1682FD8AC112C398
:103EC00084E690E090935315809352151093461515
:103ED000009349158EE090E1A0E0B0E080934A1590
:103EE00090934B15A0934C15B0934D150E948DF9EE
:103EF000C60182539048880F991F90935315809361
:103F0000521510934615009349158FE090E1A0E0FB
:103F1000B0E080934A1590934B15A0934C15B09345
:103F20004D150E948DF90E947BE090E0909353150F
:103F30008093521585E08093461582E88093491559
:103F400086E190E1A0E0B0E080934A1590934B1594
:103F5000A0934C15B0934D150E948DF920E030E0F0
:103F600048EC52E460913613709137138091381306
:103F7000909139130F9499150F94891D70935315CF
:103F80006093521515E01093461502E80093491509
:103F900086E290E1A0E0B0E080934A1590934B1543
:103FA000A0934C15B0934D150E948DF96091B20B02
:103FB0007091B30B8091B40B9091B50B0F94891D48
:103FC000709353156093521510934615009349153D
:103FD00086E390E1A0E0B0E080934A1590934B1502
:103FE000A0934C15B0934D150E948DF960910D0969
:103FF00070910E0980910F09909110090F94891DFD
:1040000070935315609352151093461500934915FC
:104010008CE390E1A0E0B0E080934A1590934B15BB
:10402000A0934C15B0934D150E948DF98091B60B5D
:104030009091B70B9093531580935215109346159A
:104040000093491584E390E1A0E0B0E080934A1525
:1040500090934B15A0934C15B0934D150E948DF97C
:1040600080911109909112099093531580935215E4
:1040700010934615009349158AE390E1A0E0B0E063
:1040800080934A1590934B15A0934C15B0934D1502
:104090000E948DF90091570801113CC18091590887
:1040A000811138C180915E0881118BC18091FA1411
:1040B0009091FB14A091FC14B091FD148C3420E17C
:1040C0009207A105B10509F0A1C136E9C32E35E17A
:1040D000D32E0AE18CEB93E10E94A557E0904C08A7
:1040E000F0904D08181619060CF085C38AE1E81601
:1040F000F10414F40C9411337EC38CE0FE0131966C
:10410000A1E1B3E101900D928A95E1F70E9478D385
:104110008091BB138D7F8093BB1347CC10925F08B7
:104120006ECC82EB95E00E943A4F80915D0890E062
:10413000A0E0B0E0895B9F4FAE4FB54A21E03AE581
:104140003093531520935215909355158093541521
:1041500087E08093461582E88093491584E890E0D3
:10416000A0E0B0E080934A1590934B15A0934C15B6
:10417000B0934D150E948DF910925E08F3CC81E04A
:10418000809334021092CE1180EC95E00E943A4F59
:1041900081E09AE590935315809352158EE490E058
:1041A000909355158093541587E08093461582E8C7
:1041B0008093491584E890E0A0E0B0E080934A1530
:1041C00090934B15A0934C15B0934D150E948DF90B
:1041D000CBCC8CE090E0909353158093521505E082
:1041E0000093461582E88093491584E190E1A0E0B0
:1041F000B0E080934A1590934B15A0934C15B09363
:104200004D150E948DF90E945DDF20E13EE040E007
:1042100050E00F94891B2115310591E049075105A4
:1042200060F05093531540935215309355152093D9
:10423000541587E08093461506C03093531520939C
:1042400052150093461502E80093491580E190E16C
:10425000A0E0B0E080934A1590934B15A0934C15C5
:10426000B0934D150E948DF90E945DDF20E13EE084
:1042700040E050E00F94891B2CE330E040E050E038
:104280000F94891B309353152093521515E010930A
:1042900046150093491582E190E1A0E0B0E08093DB
:1042A0004A1590934B15A0934C15B0934D150E9451
:1042B0008DF90E947BE0882391F00E947BE08F5F64
:1042C00080935A08C82ED12C833308F0F9CDC6014B
:1042D000880F991F909353158093521504C0109224
:1042E00053151092521510934615009349158EE000
:1042F00090E1A0E0B0E080934A1590934B15A09315
:104300004C15B0934D150E948DF9109253151092D3
:104310005215F7CD20E030E048EC52E46091B20B4A
:104320007091B30B8091B40B9091B50B0F949915CC
:104330006B017C016091B60B7091B70B072E000CDE
:10434000880B990B0F943A159B01AC01C701B6017C
:104350000F94171D0F94901D6436710510F064E6DC
:1043600070E0709353156093521545E0A42EA0920F
:10437000461552E8B52EB092491584E290E1A0E0CE
:10438000B0E080934A1590934B15A0934C15B093D1
:104390004D150E948DF9C090B20BD090B30BE090F8
:1043A000B40BF090B50B20E030E040E253E4C701DD
:1043B000B6010F947D1E18160CF03AC1011188C188
:1043C00037C180914E0801E0080F00934E0890E03D
:1043D000909353158093521585E08093461582E89B
:1043E0008093491582E490E1A0E0B0E080934A1503
:1043F00090934B15A0934C15B0934D150E948DF9D9
:104400000A3008F453CE10924E0850CE8A349041B0
:10441000A105B10509F459CE80E00E9495AE20E0D7
:1044200030E040E251E40F9499150F94891D709388
:1044300053156093521515E01093461502E800934A
:10444000491588E490E1A0E0B0E080934A1590938C
:104450004B15A0934C15B0934D150E948DF981E03A
:104460000E9495AE20E030E040E251E40F949915AF
:104470000F94891D70935315609352151093461530
:10448000009349158AE490E1A0E0B0E080934A15DA
:1044900090934B15A0934C15B0934D150E948DF938
:1044A00082E00E9495AE20E030E040E251E40F94BB
:1044B00099150F94891D709353156093521510939D
:1044C0004615009349158CE490E1A0E0B0E080939C
:1044D0004A1590934B15A0934C15B0934D150E941F
:1044E0008DF9F3CD80910D0990910E09A0910F09DE
:1044F000B091100988A399A3AAA3BBA36091110945
:1045000070911209072E000C880B990B0F943A1525
:104510006B017C0120E030E040E050E40F941C1C73
:1045200028A139A14AA15BA10F947D1E181604F1A0
:104530004090B20B5090B30B6090B40B7090B50BE1
:104540006091B60B7091B70B072E000C880B990B7E
:104550000F943A154B015C0120E030E040E251E459
:104560000F941C1CA30192010F947D1E181604F5D4
:104570008DE090E0909353158093521585E08093E1
:10458000461582E88093491584E190E1A0E0B0E00F
:1045900080934A1590934B15A0934C15B0934D15ED
:1045A0000E948DF98091CD1181113FC081E03DC005
:1045B00020E030E040E050E4C701B6010F941D1C3C
:1045C00028A139A14AA15BA10F94331587FD0EC024
:1045D00020E030E040E251E4C501B4010F941D1C1D
:1045E000A30192010F94331587FFB8CC84E190E0CA
:1045F000909353158093521585E08093461582E879
:104600008093491584E190E1A0E0B0E080934A15E1
:1046100090934B15A0934C15B0934D150E948DF9B6
:104620008091CD11811101C082E08093CD1196CC93
:104630006091B60B7091B70B072E000C880B990B8D
:104640000F943A159B01AC01C701B6010F947D1E72
:104650006091590887FDAEC0662309F423CD062E6C
:10466000000C770B8BE397E00F94D8011092590858
:1046700010925C0810925B0884E090E090935315D0
:104680008093521585E08093461502E80093491502
:104690008EE890E1A0E0B0E080934A1590934B152E
:1046A000A0934C15B0934D150E948DF981E09AE5C9
:1046B000909353158093521583E590E09093551590
:1046C0008093541587E0809346150093491563C085
:1046D0001092570820E030E040E251E460914F082A
:1046E0007091500880915108909152080F9499153B
:1046F0000F94891D7093531560935215A09246151F
:10470000B092491584E590E1A0E0B0E080934A15AD
:1047100090934B15A0934C15B0934D150E948DF9B5
:1047200020E030E040E251E4609153087091540879
:1047300080915508909156080F9499150F94891DF2
:104740007093531560935215A0924615B092491577
:1047500088E590E1A0E0B0E080934A1590934B1576
:10476000A0934C15B0934D150E948DF98EEC95E0F9
:104770000E943A4F81E09AE5909353158093521529
:1047800081E490E0909355158093541587E08093D1
:104790004615B092491584E890E0A0E0B0E080931F
:1047A0004A1590934B15A0934C15B0934D150E944C
:1047B0008DF978CC662309F475CC80915B089091D3
:1047C0005C089C012F5F3F4F30935C0820935B088F
:1047D00065E070E00F94001C909353158093521580
:1047E00085E08093461582E8809349158EE890E134
:1047F000A0E0B0E0D4CF1E141F040CF04CCB90917D
:10480000F71480919615981322C09091F814809116
:10481000971598131CC023E0E216F104C4F09091A0
:1048200098159093F614809199158093F91493300C
:10483000D1F4982F9D7F9038B1F490919A159F34C0
:1048400009F059C090919B159B3409F054C08AE13E
:10485000E6E9F5E1DF011D928A95E9F710924D082E
:1048600010924C0818CB833809F045C080919A15F6
:1048700090919B15982789279827A0E0B0E0809316
:10488000FA149093FB14A093FC14B093FD14C09001
:104890009C15D12CE12CF12CC092FE14D092FF1467
:1048A000E0920015F0920115ADE9B5E140E050E06D
:1048B000BA014C155D056E057F0508F04AC04A0136
:1048C0005B01B694A79497948794F4013696EE0F03
:1048D000FF1FEA50FB4E8C9190E0982F882711968D
:1048E0002C911197822B918380834E5F5F4F6F4F86
:1048F0007F4F1296DECF813861F580919A1590E056
:10490000A0E0B0E08093FA149093FB14A093FC1401
:10491000B093FD1480919B15482F50E060E070E04B
:104920004093FE145093FF1460930015709301158B
:10493000ACE9B5E1E2E0F5E190E020E030E02817F5
:10494000390739F04D9150E0419351932F5F3F4F1C
:10495000F6CF8AE1E6E9F5E1DF011D928A95E9F7F4
:1049600010924D0810924C0881E194E00E943A4F59
:104970006091CE11161664F4062E000C770B80E3BE
:1049800097E00F94D8018AE00E942F4E0C940233D6
:1049900060910215709103158EE197E00F94BA01B2
:1049A0008AE00E942F4E4091FA145091FB146091BE
:1049B000FC147091FD148FE097E00F94A9018AE038
:1049C0000E942F4E8091FA149091FB14A091FC1438
:1049D000B091FD14E5E7F2E000E010E04191519163
:1049E000619171914115510561057105D1F148172A
:1049F00059076A077B0791F5AC01BD01485050414A
:104A000061097109453051056105710568F1AC0115
:104A1000BD01477F423350416105710541F1843347
:104A2000F0E19F07A105B10511F1AC01BD014654AC
:104A30005041610971094730510561057105D0F098
:104A4000AC01BD0144555041610971094530510522
:104A50006105710588F402E110E00EC00F5F1F4F81
:104A6000BDCF0FEF1FEF08C003E010E005C008E066
:104A700010E002C00FE010E08A509042A109B10995
:104A8000833D9105A105B10530F00F3F2FEF1207CF
:104A900021F40C94023309E110E0F2E3CF2EF4E0AC
:104AA000DF2EF60181916F01882319F00E942F4EAD
:104AB000F8CFB801012E000C880B990B0E94A34E71
:104AC0000E94344F83E097E00E943A4F0A3111056B
:104AD00010F00C94FE32F8018827E758FF4F8F4FF3
:104AE0000D94141C8091021590910315813091054D
:104AF000E1F4109234028FEF8093BA1960E080E005
:104B00000F94000200E414E0D8018D918D018823F8
:104B100019F00E942F4EF8CF81E09AE5909353153B
:104B2000809352158EE290E0AFC08230910509F07B
:104B3000C5C081E0809334020E94ECE08FEF96E0E4
:104B400090934709809346098BE090E0909353152A
:104B50008093521505E00093461512E8109349150D
:104B600080E092E1A0E0B0E080934A1590934B156D
:104B7000A0934C15B0934D150E948DF910925315CA
:104B80001092521500934615109349158EE090E14E
:104B9000A0E0B0E080934A1590934B15A0934C157C
:104BA000B0934D150E948DF9109253151092521525
:104BB00000934615109349158FE090E1A0E0B0E016
:104BC00080934A1590934B15A0934C15B0934D15B7
:104BD0000E948DF9109253151092521500934615AC
:104BE0001093491586E190E1A0E0B0E080934A156A
:104BF00090934B15A0934C15B0934D150E948DF9D1
:104C000062E070E080E090E00E94A9AE109253153F
:104C100010925215009346151093491580E190E1CA
:104C2000A0E0B0E080934A1590934B15A0934C15EB
:104C3000B0934D150E948DF9109253151092521594
:104C4000009346151093491582E190E1A0E0B0E091
:104C500080934A1590934B15A0934C15B0934D1526
:104C60000E948DF90AE614E0F80181918F018823F2
:104C700019F00E942F4EF8CF81E09AE590935315DA
:104C8000809352158DE290E09093551580935415C2
:104C900087E08093461582E88093491584E890E088
:104CA000A0E0B0E080934A1590934B15A0934C156B
:104CB000B0934D150E948DF90C9402338330910509
:104CC00049F581E08093340204E914E0D8018D9124
:104CD0008D018823C9F00E942F4EF8CF8091FA14DD
:104CE0009091FB14A091FC14B091FD148233F0E17B
:104CF0009F07A105B10509F05BC480910215909151
:104D00000315009709F023C480910502882309F454
:104D10000DC31DC3049711F00C940233109234029A
:104D20000C94023380910215909103158130910506
:104D3000D1F41092340280910502882319F082E0A8
:104D400090E002C083E090E0909353158093521559
:104D500085E08093461582E8809349158EE190E1C5
:104D6000A0E0B0E09FCF8230910519F50EEB14E082
:104D7000F80181918F01882319F00E942F4EF8CFFE
:104D800081E0809334028091CD11843049F081E03C
:104D90009AE5909353158093521585E390E074CF74
:104DA00081E09AE5909353158093521586E390E045
:104DB0006BCF8330910509F04CC02091050222236E
:104DC00019F1909353158093521585E08093461501
:104DD00082E8809349158EE190E1A0E0B0E08093F5
:104DE0004A1590934B15A0934C15B0934D150E9406
:104DF0008DF940E060E070E088EC92E40E9453E1BD
:104E0000109205020C94023382E090E090935315C7
:104E10008093521585E08093461582E8809349156A
:104E20008EE190E1A0E0B0E080934A1590934B159D
:104E3000A0934C15B0934D150E948DF940E060E0B1
:104E400070E0CB010E9453E181E0809305020C9455
:104E50000233049711F00C940233809120098823C7
:104E6000F1F082E090E0909353158093521585E025
:104E70008093461582E8809349158FE190E1A0E088
:104E8000B0E080934A1590934B15A0934C15B093C6
:104E90004D150E948DF9109220090C94023383E085
:104EA00090E0909353158093521585E080934615BA
:104EB00082E8809349158FE190E1A0E0B0E0809313
:104EC0004A1590934B15A0934C15B0934D150E9425
:104ED0008DF981E0809320090C94023360910215D2
:104EE0007091031580E090E00F9438156B017C0100
:104EF00020E030E04AEF53E40F94331587FF11C0F0
:104F000020E030E040E251E4C701B6010F947D1E7D
:104F100018166CF0C12CD12C70E2E72E71E4F72E3C
:104F200006C0C12CD12CEAEFEE2EE3E4FE2EC70121
:104F3000B6010F94891D70935602609355020C942C
:104F400002338091FA149091FB14A091FC14B0915B
:104F5000FD148830F0E19F07A105B10509F050C0AC
:104F600081E09AE590935315809352158DE290E07D
:104F7000909355158093541587E08093461512E859
:104F80001093491584E890E0A0E0B0E080934A15C2
:104F900090934B15A0934C15B0934D150E948DF92D
:104FA000109253151092521505E000934615109378
:104FB000491580E190E1A0E0B0E080934A1590931C
:104FC0004B15A0934C15B0934D150E948DF910927E
:104FD000531510925215009346151093491582E10E
:104FE00090E1A0E0B0E080934A1590934B15A09318
:104FF0004C15B0934D150E948DF90E94ECE08FC0C6
:105000008A3020E19207A105B105E1F580910215F2
:1050100090910315813F910511F00C94023381E0CA
:105020009AE5909353158093521586E390E0909300
:1050300055158093541587E08093461582E8809338
:10504000491584E890E0A0E0B0E080934A15909381
:105050004B15A0934C15B0934D150E948DF94EE75A
:1050600055E065E875E084E00E94AAA960E081E768
:1050700095E00E94ADE087E695E090934709809324
:1050800046094DC08C309041A105B10509F047C0DB
:105090008091021590910315019709F040C00F947B
:1050A0002D0F1092CD1181E0809334028CE090E0BE
:1050B000909353158093521585E08093461512E81E
:1050C0001093491584E190E1A0E0B0E080934A1587
:1050D00090934B15A0934C15B0934D150E948DF9EC
:1050E00081E09AE5909353158093521585E390E003
:1050F000909355158093541587E08093461510932F
:10510000491584E890E0A0E0B0E080934A159093C0
:105110004B15A0934C15B0934D150E948DF98091BD
:10512000FA149091FB14A091FC14B091FD148C30F2
:105130009041A105B10511F00C9402338091021544
:1051400090910315029711F00C9402330F942D0FD8
:1051500081E0809359081092CD118093340210920F
:105160005C0810925B0881E09AE590935315809358
:10517000521582E590E088CD2091021530910315FB
:10518000B90180E090E037FF09C00F94381520E0A6
:1051900030E040E857E40F941C1C02C00F9438150F
:1051A00020E030E048EC52E40F94171D6B017C01C5
:1051B00020E030E040EA51EC0F947D1E87FD31C0C5
:1051C00020E030E040EA51E4C701B6010F94331506
:1051D00018163CF1A70196016091361370913713B0
:1051E00080913813909139130F941C1C20E030E00B
:1051F00048EC53E40F94991590580F94891DCB01F6
:105200000E9482FCC0923613D0923713E09238137A
:10521000F09239138AEF96E09093470980934609FC
:1052200028C020E030E048EC52E4609136137091E1
:10523000371380913813909139130F9499150F9467
:10524000891D709353156093521585E08093461520
:1052500082E88093491586E290E1A0E0B0E0809377
:105260004A1590934B15A0934C15B0934D150E9481
:105270008DF96091361370913713809138139091A6
:1052800039138E010B5E1F4F23E041E00F940B108A
:105290009F938F938CEE96E09F938F930451110907
:1052A0001F930F930F94CB14C8010E9483AF0F90EC
:1052B0000F900F900F900F900F900C9402338091ED
:1052C000021590910315009729F481E08093340230
:1052D0000C94023381309105B1F48091050288234A
:1052E00049F081E09AE590935315809352158CE331
:1052F00090E0CACC81E09AE59093531580935215C3
:105300008BE390E0C1CC82309105F9F283309105B6
:1053100039F58091050240E0882389F060E070E073
:1053200088EC92E40E9453E11092050281E09AE534
:10533000909353158093521589E390E0A5CC60E0DB
:1053400070E0CB010E9453E181E08093050281E08F
:105350009AE590935315809352158AE390E094CC8C
:105360008530910559F540E060E070E084E393E416
:105370000E942CAD46E060E070E08CE892E40E9470
:105380002CAD84EB90E0909353158093521505E07B
:105390000093461512E81093491584E390E1A0E0CC
:1053A000B0E080934A1590934B15A0934C15B093A1
:1053B0004D150E948DF986E490E02DC08630910550
:1053C00099F540E060E070E080E793E40E942CAD46
:1053D00046E060E070E08CED92E40E942CAD80EF3E
:1053E00090E0909353158093521505E00093461575
:1053F00012E81093491584E390E1A0E0B0E08093B7
:105400004A1590934B15A0934C15B0934D150E94DF
:105410008DF98EE690E0909353158093521500938A
:10542000461510934915BFC0813F910511F00C94AA
:10543000023340E060E070E0CB010E9453E141E0C4
:1054400060E070E0CB010E9453E11092050240E061
:1054500060E070E0CB010E942CAD46E060E070E0BF
:10546000CB010E942CAD109253151092521505E0FD
:105470000093461512E81093491584E390E1A0E0EB
:10548000B0E080934A1590934B15A0934C15B093C0
:105490004D150E948DF961E070E080E090E00E947F
:1054A000A9AE109253151092521500934615109301
:1054B00049158AE390E1A0E0B0E080934A1590930B
:1054C0004B15A0934C15B0934D150E948DF961E0DA
:1054D00070E080E090E00E94A9AE84E190E09093BB
:1054E000531580935215009346151093491584E186
:1054F00090E1A0E0B0E080934A1590934B15A09303
:105500004C15B0934D150E948DF981E09AE590936A
:1055100053158093521589E390E09093551580932D
:10552000541587E0809346151093491584E890E060
:10553000A0E0B0E080934A1590934B15A0934C15D2
:10554000B0934D150E948DF982E00C94FB328130AE
:105550009105A9F440E060E070E0CB010E942CAD21
:10556000109253151092521585E08093461582E8EB
:105570008093491584E390E1A0E0B0E093CB0297DB
:1055800011F00C94023346E060E070E0CB010E9421
:105590002CAD109253151092521585E0809346154C
:1055A00082E8809349158AE390E1A0E0B0E07ACBED
:1055B000843320E19207A105B10551F460910215F1
:1055C0007091031580E090E00F94381540E010C012
:1055D0008A339041A105B10511F00C94023360911A
:1055E00002157091031580E090E00F94381546E0A5
:1055F0000E942CAD0C9402338091021590910315FA
:10560000009709F462CE8130910509F04CC0809179
:105610005B17882319F083E090E002C082E090E0FD
:10562000909353158093521585E08093461582E838
:105630008093491585E490E1A0E0B0E080934A159D
:1056400090934B15A0934C15B0934D150E948DF976
:105650008AE090E0909353158093521585E08093F3
:10566000461582E88093491580E092E1A0E0B0E021
:1056700080934A1590934B15A0934C15B0934D15FC
:105680000E948DF90E9499AD811103C08CED96E0C6
:1056900002C080ED96E0909347098093460982E02E
:1056A0008093CE1171C18230910509F0A8C081E0CC
:1056B0008093340288E0EFE4F8E0DF011D928A95E0
:1056C000E9F780E090E0A0E2B1E480934F08909386
:1056D0005008A0935108B0935208809353089093B8
:1056E0005408A0935508B093560884E690E0909330
:1056F00053158093521505E00093461512E8109358
:10570000491584E590E1A0E0B0E080934A159093BC
:105710004B15A0934C15B0934D150E948DF920E0C8
:1057200030E040E251E46091530870915408809158
:105730005508909156080F9499150F94891D7093F0
:10574000531560935215009346151093491588E53B
:1057500090E1A0E0B0E080934A1590934B15A093A0
:105760004C15B0934D150E948DF96091B20B70915C
:10577000B30B8091B40B9091B50B0F94891D70936E
:10578000531560935215009346151093491586E3FF
:1057900090E1A0E0B0E080934A1590934B15A09360
:1057A0004C15B0934D150E948DF98091B60B9091D8
:1057B000B70B909353158093521500934615109391
:1057C000491584E390E1A0E0B0E080934A159093FE
:1057D0004B15A0934C15B0934D150E948DF962E0C6
:1057E00070E080E090E00E94A9AE81E09AE590939D
:1057F00053158093521581E490E00C943E3483302D
:10580000910509F076C010925D0880E00E9495AE87
:1058100020E030E040E251E40F9499150F94891D87
:10582000709353156093521505E00093461512E8E6
:105830001093491588E490E1A0E0B0E080934A1508
:1058400090934B15A0934C15B0934D150E948DF974
:1058500081E00E9495AE20E030E040E251E40F94F8
:1058600099150F94891D70935315609352150093E9
:105870004615109349158AE490E1A0E0B0E08093CA
:105880004A1590934B15A0934C15B0934D150E945B
:105890008DF982E00E9495AE20E030E040E251E4D4
:1058A0000F9499150F94891D709353156093521599
:1058B00000934615109349158CE490E1A0E0B0E008
:1058C00080934A1590934B15A0934C15B0934D15AA
:1058D0000E948DF962E070E080E090E00E94A9AE45
:1058E00081E09AE5909353158093521587E490E0F8
:1058F000C5C78430910509F485C68530910549F402
:105900004EE750E160E070E085EE94E00E943CF9E3
:1059100079C6069709F076C68CEC96E09093470915
:10592000809346098BE090E02BC280910215909104
:105930000315019711F51092340281E09AE59093D6
:105940005315809352158FE390E0909355158093F3
:10595000541587E08093461582E88093491584E8C2
:1059600090E0A0E0B0E080934A1590934B15A0938F
:105970004C15B0934D150E948DF9809102159091B0
:105980000315029709F03EC681E09AE590935315FE
:105990008093521580E490E077C9E0910215F09170
:1059A00003153197EB30F10508F0E4C18827ED5677
:1059B000FF4F8F4F0D94141C8091BA1380FF5CC66B
:1059C000869580FD5CC658C62DEC3CEC4CEC5DE346
:1059D0006091361370913713809138139091391379
:1059E0000F941D1C6B017C0120E030E040EA51EC7B
:1059F0000F947D1E87FDC2C120E030E040EA51E4F3
:105A0000C701B6010F94331518160CF03FC6B6C186
:105A10002DEC3CEC4CEC5DE3609136137091371348
:105A200080913813909139130F941C1C6B017C01E9
:105A300020E030E040EA51EC0F947D1E87FD9EC1CE
:105A400020E030E040EA51E4C701B6010F9433157D
:105A500018160CF092C692C180E00E948DAC0E9494
:105A600099AD811103C083E796E002C085E696E018
:105A7000909347098093460982E08093CE1181E09C
:105A80009AE5909353158093521584E590E0909396
:105A900055158093541587E08093461582E88093CE
:105AA000491584E890E0A0E0B0E080934A15909317
:105AB0004B15A0934C15B0934D150E948DF95EC106
:105AC00083E08093CE1183E090E090935315809310
:105AD000521585E08093461582E8809349158DE83C
:105AE00090E1A0E0B0E080934A1590934B15A0930D
:105AF0004C15B0934D150E948DF9E12CF12C00E06E
:105B0000DD24D394AA24A39445E0942E55E0852E59
:105B100062E8762EDD2031F0CC24C39435E0B32E3C
:105B200010E005C0CC24CA94BB24BA9414E0DA2453
:105B3000B116D1F1802F90E04897A4F50F5FF701DF
:105B4000919EE00DF11D1124EE0FFF1FEE0FFF1FC0
:105B5000E45BFC4E20E030E04AE754E46081718170
:105B6000828193810F9499150F94891D7093531519
:105B7000609352158092461570924915802F90E0DF
:105B80008158974F880F991F092E000CAA0BBB0B49
:105B900080934A1590934B15A0934C15B0934D15D7
:105BA0000E948DF91C0DC4CFBFEFEB1AFB0AE5E094
:105BB000EE16F10409F0AECF81E09AE5909353150B
:105BC0008093521585E590E0909355158093541578
:105BD00087E08093461582E88093491584E890E039
:105BE000A0E0B0E080934A1590934B15A0934C151C
:105BF000B0934D150E948DF987E096E09093470988
:105C000080934609BBC042E060E070E080E890E429
:105C10000E94B7AD40E060E070E08DE193E40E9447
:105C2000B7AD41E060E070E08BE193E413C042E087
:105C300060E070E080E890E40E94B7AD40E060E092
:105C400070E080E292E40E94B7AD41E060E070E075
:105C500080E292E40E94B7AD86E08093CE118EC0C0
:105C600042E060E070E080E890E40E94B7AD40E080
:105C700060E070E089E893E4E6CF42E060E070E045
:105C800080E890E40E94B7AD40E060E070E089E811
:105C900093E40CC042E060E070E080E890E40E9491
:105CA000B7AD40E060E070E080E292E40E94B7AD02
:105CB00041E060E070E087E893E4CCCF80915B172F
:105CC00081111CC083E090E090935315809352158E
:105CD00085E08093461582E88093491585E490E13C
:105CE000A0E0B0E080934A1590934B15A0934C151B
:105CF000B0934D150E948DF981E01BC082E090E0C9
:105D0000909353158093521585E08093461582E851
:105D10008093491585E490E1A0E0B0E080934A15B6
:105D200090934B15A0934C15B0934D150E948DF98F
:105D300080E00E948DAC20E030E048EC52E46091BD
:105D400036137091371380913813909139130F9453
:105D500099150F94891D709353156093521585E022
:105D60008093461582E88093491586E290E1A0E091
:105D7000B0E09BCE8BEE95E00E943A4F8AE090E037
:105D8000909353158093521585E08093461582E8D1
:105D9000809349154BC184E08093CE118091FA1411
:105DA0009091FB14A091FC14B091FD146091021528
:105DB000709103158834F0E19F07A105B10509F43E
:105DC00053C08A3420E19207A105B10509F456C0F9
:105DD0008C3430E19307A105B10509F45AC086342B
:105DE0009041A105B10509F05EC063307105B9F5B8
:105DF0008AED95E0909347098093460981E080936E
:105E00005E088093340210924E0881E09AE59093E8
:105E10005315809352158AE490E090935515809322
:105E2000541587E08093461512E81093491584E8CD
:105E300090E0A0E0B0E080934A1590934B15A093BA
:105E40004C15B0934D150E948DF98AE090E0909327
:105E500053158093521585E080934615E5C06093F5
:105E60005D081092CE11CEC380E090E8ADE9B3E4B6
:105E70008CA39DA3AEA3BFA3312C15C080E090E0FE
:105E8000ABE9B3E48CA39DA3AEA3BFA333243394A7
:105E90000AC080E090E0A8ECB3E48CA39DA3AEA37D
:105EA000BFA382E0382E80E090E00F94381520E008
:105EB00030E040E251E40F94171D6B017C0120E0BB
:105EC00030E0A9010F94331587FF09C010924808EC
:105ED0001092490810924A0810924B081FC02CA13A
:105EE0003DA14EA15FA1C701B6010F947D1E1816FA
:105EF0004CF0C0924808D0924908E0924A08F092CB
:105F00004B080CC08CA19DA1AEA1BFA180934808F5
:105F100090934908A0934A08B0934B0860914808B1
:105F20007091490880914A0890914B08432D0E9436
:105F3000B7AD61E070E080E090E00E94A9AE80E043
:105F40000E9495AE20E030E040E251E40F949915B4
:105F50000F94891D709353156093521505E00093BB
:105F6000461512E81093491588E490E1A0E0B0E0EE
:105F700080934A1590934B15A0934C15B0934D15F3
:105F80000E948DF981E00E9495AE20E030E040E271
:105F900051E40F9499150F94891D709353156093D4
:105FA000521500934615109349158AE490E1A0E03C
:105FB000B0E080934A1590934B15A0934C15B09385
:105FC0004D150E948DF982E00E9495AE20E030E0F0
:105FD00040E251E40F9499150F94891D7093531565
:105FE0006093521500934615109349158CE490E187
:105FF000A0E0B0E080934A1590934B15A0934C1508
:10600000B0934D150E948DF961E070E080E090E062
:106010000E94A9AE1092CE118AE090E090935315A1
:1060200080935215009346151093491580E092E134
:10603000A0E0B0E00C9452268091FA149091FB14E9
:10604000A091FC14B091FD148635E0E19E07A105F6
:10605000B10509F041C020E030E040E253E4609136
:10606000B20B7091B30B8091B40B9091B50B0F9460
:106070003315209102153091031587FF0AC425308E
:10608000310508F006C480EA90E0909353158093A0
:10609000521585E08093461512E81093491580E269
:1060A00090E1A0E0B0E080934A1590934B15A09347
:1060B0004C15B0934D150E948DF965E070E080E0BD
:1060C00090E00E94A9AE81E09AE5909353158093E9
:1060D000521582E490E0D2C38435F0E19F07A10518
:1060E000B105B9F4609102157091031580E090E05C
:1060F0000F94381520E030E040E251E40F94171D72
:1061000060934F0870935008809351089093520801
:1061100079C288359041A105B10509F073C260913B
:1061200002157091031580E090E00F94381520E07F
:1061300030E040E251E40F94171D609353087093D0
:10614000540880935508909356085CC260910215DC
:106150007091031584EC95E00F94BA0180910215BB
:106160009091031582309105A1F038F4009771F0F9
:106170000197E1F48EE095E043C28430910579F017
:1061800058F0059799F489E995E00BC088EF94E001
:1061900037C286EB95E005C08CEA95E002C087EA3D
:1061A00095E090934709809346092CC282E295E0DE
:1061B00027C281E395E00E943A4F809102159091A9
:1061C00003158130910519F46499C3C41BC2892B4E
:1061D00009F018C28FE395E00E943A4F809144087D
:1061E000813039F585E595E00E943A4F81E09AE5E6
:1061F00090935315809352158EE290E0909355152D
:106200008093541587E08093461582E88093491562
:1062100084E890E0A0E0B0E080934A1590934B159D
:10622000A0934C15B0934D150E948DF91092CC118E
:1062300035C0823069F489E695E00E943A4F81E0EA
:106240009AE5909353158093521586E390E00EC023
:10625000833031F58DE795E00E943A4F81E09AE571
:10626000909353158093521581E490E090935515C7
:106270008093541587E08093461582E880934915F2
:1062800084E890E0A0E0B0E080934A1590934B152D
:10629000A0934C15B0934D150E948DF91092EA12FF
:1062A000109244080E94ECE0ADC1809102159091DB
:1062B00003158F3F910531F028F08FEF90E0A0E0BB
:1062C000B0E002C0A0E0B0E0809306029093070225
:1062D000A0930802B09309028091060290910702F0
:1062E000A0910802B09109020097A105B10509F536
:1062F000109253151092521505E00093461512E8BE
:10630000109349158AE890E1A0E0B0E080934A1527
:1063100090934B15A0934C15B0934D150E948DF999
:1063200089E090E0909353158093521500934615A1
:106330003DC00196A11DB11D05E0B695A7959795A5
:1063400087950A95D1F70197A109B109009731E026
:10635000A307B10550F0B0935315A0935215909335
:1063600055158093541587E005C09093531580937D
:10637000521585E08093461512E8109349158AE876
:1063800090E1A0E0B0E080934A1590934B15A09364
:106390004C15B0934D150E948DF988E090E09093D4
:1063A00053158093521585E0809346151093491537
:1063B0008CE890E1A0E0B0E080934A1590934B15F3
:1063C000A0934C15B0934D150E948DF98091060253
:1063D00090910702A0910802B0910902BA2FA92F4B
:1063E000982F88270097E1E0AE07B10550F0B093F1
:1063F0005315A0935215909355158093541587E02B
:1064000005C0909353158093521585E080934615EF
:1064100082E88093491581EA90E0A0E0B0E00C9416
:10642000522681E995E00E943A4F0E9420AD4091AA
:10643000FA145091FB146091FC147091FD148823A0
:1064400039F0433DF0E25F076105710509F4C7C308
:10645000423D50426105710509F0D4C0809102159A
:1064600090910315019709F00CC50E9420AD882377
:1064700009F407C58091BA1987FDC4C0A2E18A0258
:10648000C00111248B58944E0E947559C12C90E282
:10649000D92EE12CF12C05E012E810925315109240
:1064A00052150093461510934915C0924A15D09283
:1064B0004B15E0924C15F0924D150E948DF9BFEFEF
:1064C000CB1ADB0AEB0AFB0AEAE0CE16E0E2DE06B4
:1064D000E104F10411F70091BA19F2E10F02800111
:1064E0001124035F154EF80101900020E9F7C8015F
:1064F0008E1B9F0B439697FD01967C01F594E794C4
:106500001E141F040CF0C6C49E012F5F3F4F69018B
:1065100084E1D9011D928A95E9F7A70162EA75E045
:10652000C9010F94901FB801C6018E0D9F1D0F94D5
:106530007B1F40E050E260E070E0C6010E943CF941
:1065400062E070E080E090E00E94A9AE40E060E090
:1065500070E08FE793E40E9453E141E060E070E077
:106560008FE793E40E9453E1109205028DE090E0E2
:10657000909353158093521585E08093461512E849
:106580001093491584E190E1A0E0B0E080934A15B2
:1065900090934B15A0934C15B0934D150E948DF917
:1065A00062E070E080E090E00E94A9AE81E09AE5B0
:1065B000909353158093521585E390E09093551571
:1065C0008093541587E0809346151093491584E80D
:1065D00090E0A0E0B0E080934A1590934B15A09313
:1065E0004C15B0934D150E948DF981E080933402D3
:1065F0008093CC1183E08093CD1104C08EE895E0A8
:106600000E943A4F80E5E6EFF4E1DF011D928A95A2
:10661000E9F78AE58093F71485EA8093F8140C94DF
:106620004B1F8CEB93E10E948357F701EA56FA4E19
:106630008083809196158A3581F01E141F0414F012
:106640000C946A20D601E02F1D92EA95E9F710928A
:106650004D0810924C080C946A2062E070E080E0D3
:1066600090E00E94A9AEFFEFEF1AFF0AF0924D08EA
:10667000E0924C080C946A208CEB96E002C08BEA06
:1066800096E0909347098093460955CB88E290E0C5
:106690000E9482FC2DEC3CEC4CEC5DE360913613E7
:1066A0007091371380913813909139130F941D1CFA
:1066B0006B017C0120E030E040EA51EC0F947D1E3C
:1066C00087FD12C020E030E040EA51E4C701B60186
:1066D0000F943315181644F0C0923613D092371326
:1066E000E0923813F092391320E030E048EC52E4A5
:1066F000609136137091371380913813909139134C
:106700000F9499150F94891D70935315609352152A
:1067100085E08093461582E88093491586E290E1F2
:10672000A0E0B0E080934A1590934B15A0934C15D0
:10673000B0934D150E948DF9609136137091371307
:1067400080913813909139138E010B5E1F4F23E017
:1067500041E00F940B109F938F938DE996E09F93E8
:106760008F93045111091F930F930F94CB14C801F9
:106770000E9483AF88E996E076C088ED9FEF0E9483
:1067800082FC2DEC3CEC4CEC5DE360913613709197
:10679000371380913813909139130F941C1C6B019F
:1067A0007C0120E030E040EA51EC0F947D1E87FD33
:1067B00012C020E030E040EA51E4C701B6010F9476
:1067C0003315181644F0C0923613D0923713E09266
:1067D0003813F092391320E030E048EC52E4609135
:1067E00036137091371380913813909139130F94A9
:1067F00099150F94891D709353156093521585E078
:106800008093461582E88093491586E290E1A0E0E6
:10681000B0E080934A1590934B15A0934C15B0931C
:106820004D150E948DF96091361370913713809148
:106830003813909139138E010B5E1F4F23E041E016
:106840000F940B109F938F938AE896E09F938F93FA
:10685000045111091F930F930F94CB14C8010E9488
:1068600083AF85E896E090934709809346090F909F
:106870000F900F900F900F900F9080CA9093551526
:106880008093541587E080934615109349150C9416
:106890004E262430310589F481E00F94170F2091A2
:1068A00053083091540840915508509156080F9460
:1068B0001D1C41E00F94EE0EB2C02530310508F4E6
:1068C000F4C02630310509F431C108F023C181E05C
:1068D0008093570840E060E070E08EE393E40E940C
:1068E0002CAD20E030E048EC52E46091B20B7091A6
:1068F000B30B8091B40B9091B50B0F9499156B016C
:106900007C016091B60B7091B70B072E000C880BC1
:10691000990B0F943A159B01AC01C701B6010F9476
:10692000171D0F94901D6436710510F064E670E039
:10693000709353156093521505E00093461512E8C5
:106940001093491584E290E1A0E0B0E080934A15ED
:1069500090934B15A0934C15B0934D150E948DF953
:106960006091B20B7091B30B8091B40B9091B50B09
:106970000F94891D7093531560935215009346151B
:106980001093491586E390E1A0E0B0E080934A15AA
:1069900090934B15A0934C15B0934D150E948DF913
:1069A0008091B60B9091B70B90935315809352152D
:1069B000009346151093491584E390E1A0E0B0E000
:1069C00080934A1590934B15A0934C15B0934D1599
:1069D0000E948DF965E070E080E090E00E94A9AE31
:1069E00081E09AE5909353158093521584E490E0EA
:1069F000909355158093541587E080934615109316
:106A0000491584E890E0A0E0B0E080934A159093A7
:106A10004B15A0934C15B0934D150E948DF920E0B5
:106A200030E040E251E460914F087091500880914D
:106A30005108909152080F9499150F94891D7093E5
:106A400053156093521505E00093461512E8109314
:106A5000491584E590E1A0E0B0E080934A15909359
:106A60004B15A0934C15B0934D150E948DF920E065
:106A700030E040E251E460915308709154088091F5
:106A80005508909156080F9499150F94891D70938D
:106A9000531560935215009346151093491588E5D8
:106AA00090E1A0E0B0E00C9452262230310579F458
:106AB00080E00F94170F20914F08309150084091BB
:106AC0005108509152080F941D1C40E0F3CE233022
:106AD000310570F081E00F94170F20915308309129
:106AE000540840915508509156080F941C1CE1CE53
:106AF0002130310509F093CF80E00F94170F2091DA
:106B00004F083091500840915108509152080F940D
:106B10001C1CDBCF213F310509F081CF10925708B3
:106B200061E070E080E090E00E94A9AE81E09AE52B
:106B3000909353158093521581E490E090935515EE
:106B40008093541587E08093461582E88093491519
:106B500058CF8FEE95E00E943A4F81E00E9493A8B3
:106B60008DE090E0909353158093521585E08093CB
:106B7000461512E81093491584E190E1A0E0B0E0D9
:106B800080934A1590934B15A0934C15B0934D15D7
:106B90000E948DF983E08093CD1181E09AE5909376
:106BA00053158093521585E390E09093551580938B
:106BB000541587E0809346151093491584E890E0BA
:106BC000A0E0B0E080934A1590934B15A0934C152C
:106BD000B0934D150E948DF91092440813CD87E0B3
:106BE00096E00E943A4F8091BB199091BC19992769
:106BF00020910215309103158217930708F402CDF6
:106C00008AE995E00E943A4F809102158150809365
:106C1000BA19A4ED8A2EA0E29A2EA12CB12C05E07F
:106C200012E81092531510925215009346151093C6
:106C3000491580924A1590924B15A0924C15B0922E
:106C40004D150E948DF92FEF821A920AA20AB20AFC
:106C50003EED831630E29306A104B10411F7809152
:106C6000BA19A2E18A02C0011124FC01E35FF54ECA
:106C70007F0101900020E9F7C7018E1B9F0B43960F
:106C800097FD01968C011595079510161106FCF4D9
:106C90009E012F5F3F4F690184E1D9011D928A95C2
:106CA000E9F7A80162EA75E0C9010F94901FB701E6
:106CB000C601800F911F0F947B1F44ED50E260E0EE
:106CC00070E0C6010E943CF905E012E806C044ED00
:106CD00050E260E070E0C701F5CF109253151092BA
:106CE0005215009346151093491580924A159092BB
:106CF0004B15A0924C15B0924D150E948DF9BFEF27
:106D00008B1A9B0AAB0ABB0AE6EE8E16E0E29E06E1
:106D1000A104B10411F78E010F5F1F4F84E1D80168
:106D20001D928A95E9F78091BC198F938091BB19C8
:106D30008F93809103158F93809102158F938CEA26
:106D400095E09F938F931F930F930F94AA1F4EED7F
:106D500050E260E070E0C8010E943CF962E070E03F
:106D600080E090E00E94A9AE0FB6F894DEBF0FBE9F
:106D7000CDBF31E2C32E32E1D32EE12CF12C43E121
:106D8000442E40E6542E612C712C88248394912C3F
:106D9000AA24AA94BA2C75E0272EE2E83E2E0AE037
:106DA00010E08091BB199091BC198815990594F158
:106DB000B0925315A0925215209246153092491563
:106DC00040924A1550924B1560924C1570924D1599
:106DD0000E948DF910935315009352152092461579
:106DE00030924915C0924A15D0924B15E0924C153D
:106DF000F0924D150E948DF9FFEF8F1A9F0A20E146
:106E0000420E511C611C711C3FEFC31AD30AE30AE6
:106E1000F30AC7CF809102159091031524E0880FE3
:106E2000991F2A95E1F78D5F9F49A0E0B0E020EF20
:106E300037E8309353152093521505E0009346151B
:106E400012E81093491580934A1590934B15A0931F
:106E50004C15B0934D150E948DF9809102159091BB
:106E60000315805E9D4EA0E0B0E026E030E0309358
:106E700053152093521500934615109349150C9401
:106E800052268091021590910315892B11F40C94D0
:106E90006529B8CB40E050E260E070E0C8014ECB1D
:106EA000E3960FB6F894DEBF0FBECDBFDF91CF9152
:106EB0001F910F91FF90EF90DF90CF90BF90AF9018
:106EC0009F908F907F906F905F904F903F902F900A
:106ED00008952F923F924F925F926F927F928F927E
:106EE0009F92AF92BF92CF92DF92EF92FF920F9359
:106EF0001F93CF93DF93CDB7DEB7C154D1090FB63F
:106F0000F894DEBF0FBECDBF22968FAF229720919F
:106F100078082CAF21E0209378088091BE128D3440
:106F200009F4B3C4843511F40C943849873411F052
:106F30000C943F498091BC129091BD128B31910508
:106F400009F420C2B4F48430910534F48230910500
:106F5000E4F597FF2EC095C48531910511F40C948A
:106F600041498A31910509F409C2049709F089C49D
:106F7000C6C18A32910509F4B5C34CF48D3191052F
:106F8000B1F00CF429C24E9709F465C27AC48B356E
:106F9000910509F425C38C35910509F425C38A357B
:106FA000910509F06EC4109277080C94414914E0E1
:106FB0003FC280912002882311F40C9441490E9421
:106FC00032C30E9478D30C9441492091200222239D
:106FD00011F40C94414911E0029709F010E00E946D
:106FE00032C319821A821B821C821D821E821F825A
:106FF000188682E50E9415A8882309F438C10E94EA
:1070000095A74B015C0120E030E0A9010F943315F6
:10701000882309F442C18091431790914417A091AD
:107020004517B09146178CA39DA3AEA3BFA3809133
:10703000471790914817A0914917B0914A1788A710
:1070400099A7AAA7BBA78091111390911213A091A1
:107050001313B09114138CA79DA7AEA7BFA780915F
:10706000151390911613A0911713B091181388ABB4
:1070700099ABAAABBBAB2CA53DA54EA55FA56CA15A
:107080007DA18EA19FA10F94331581110DC028A958
:1070900039A94AA95BA968A579A58AA59BA50F94DA
:1070A0003315882309F4F9C020E030E0A901C501B7
:1070B000B4010F943315881F8827881F181729F0EB
:1070C00080E090E0A0E8BFEB04C080E090E0A0E8A2
:1070D000BFE388AF99AFAAAFBBAF2CA13DA14EA132
:1070E0005FA16CA57DA58EA59FA50F941C1C6CAB04
:1070F0007DAB8EAB9FAB28A539A54AA55BA568A93A
:1071000079A98AA99BA90F941C1C6B017C012CA94D
:107110003DA94EA95FA9CA01B9010F9499152B0188
:107120003C01A7019601C701B6010F9499159B0177
:10713000AC01C301B2010F941D1C0F94CB1E2B0197
:107140003C019B01AC0160E070E080E89FE30F949C
:10715000171D21966CAF7DAF8EAF9FAF219720E0BA
:1071600030E040E05FE3C301B2010F9499152B01B9
:107170003C01A5019401C501B4010F9499154B017F
:107180005C01A3019201C301B2010F9499159B0107
:10719000AC01C501B4010F941C1C0F94CB1E28AD8B
:1071A00039AD4AAD5BAD0F9499154B015C01C70138
:1071B000B601905821962CAD3DAD4EAD5FAD2197F7
:1071C0000F949915A50194010F9499156B017C01F9
:1071D0002CA53DA54EA55FA56CA17DA18EA19FA16B
:1071E0000F941D1C20E030E040E05FE30F94991500
:1071F0009B01AC01C701B6010F941D1C2CA13DA140
:107200004EA15FA10F941C1C69837A838B839C839E
:1072100028A939A94AA95BA968A579A58AA59BA52A
:107220000F941D1C20E030E040E05FE30F949915BF
:107230006B017C0121962CAD3DAD4EAD5FAD21972C
:107240006CA97DA98EA99FA90F949915A5019401F8
:107250000F9499159B01AC01C701B6010F941D1C39
:1072600028A539A54AA55BA50F941C1C12C089E46A
:107270000E9415A8882331F00E9495A769837A831C
:107280008B839C838AE40E9415A8882331F00E9496
:1072900095A76D837E838F83988720E030E0A901D6
:1072A00069817A818B819C810F94331581110BC088
:1072B00020E030E0A9016D817E818F8198850F9457
:1072C00033158823A1F0412FBE016F5F7F4F81E10D
:1072D00093E10E9474CB0E9481EE6093B21370938D
:1072E000B3138093B4139093B5130C9441490F9446
:1072F000F8018CE797E00F9413010C94414980E565
:107300000E9415A8882329F00E940FF96B017C01C7
:1073100003C0C12CD12C760183E50E9415A88823D7
:1073200061F00E9495A720E030E04AE754E40F9412
:1073300099150F94901D6B017C010E948AA0809189
:107340003F0B811105C060E082E997E00E94ADE04B
:107350000E9481EEC60ED71EE81EF91E0E9481EE25
:10736000DC01CB018C199D09AE09BF09B7FD02C034
:107370000C94414980E00E945B4FF0CF0E94C19382
:107380000C9441490E94CF8281110C94414980E0C4
:1073900090E0A8E4B2E489839A83AB83BC8380E065
:1073A00090E0A0E2B1E48D839E83AF83B8878987A4
:1073B0009A87AB87BC8780E50E9415A8882321F0B7
:1073C0000E945DA7862F01C080E0BE016F5F7F4FE6
:1073D0000E94E5DF0C94414980913E0B8770873015
:1073E00011F00C94654960E08FE40E9422A881119D
:1073F0000C9441490C94654980915B1781111DC023
:107400000E94BB6C8823F9F0115011F40C944C4B82
:1074100040E050E060E078E085E00E94F1A861E0A3
:1074200083EF97E00E9437A88BED97E00E94C6D0CB
:107430000E94CF82882301F306C060E08FE40E949F
:1074400022A88823E9F20E945BA88EE998E00E94B6
:10745000C6D00C94414920912E1330912F134091A6
:1074600030135091311360914317709144178091FC
:107470004517909146170F941D1CAB01BC0188E580
:107480000E94F2AF6C8F7D8F8E8F9F8F2091321371
:107490003091331340913413509135136091471755
:1074A000709148178091491790914A170F941D1CAD
:1074B000AB01BC0189E50E94F2AF69837A838B83BB
:1074C0009C83BE016F5F7F4FCE014C960E94B08FB0
:1074D000882311F40C94414980E00E948DAC0E94F5
:1074E0005CD661E085E40E9422A8182F21E0482F95
:1074F000BE016F5F7F4FCE014C960E94ABE86B01DF
:107500007C019B01AC010F940F1F81115FC08C8C1B
:107510009D8CAE8CBF8C20E030E0A901C501B40188
:107520000F94331587FF05C027E137EB41E558EB92
:1075300004C027E137EB41E558E3C501B4010F94DE
:107540001D1CAB01BC0180EC98E00F94C701898041
:107550009A80AB80BC8020E030E0A901C501B40175
:107560000F94331587FF05C027E137EB41E558EB52
:1075700004C027E137EB41E558E3C501B4010F949E
:107580001D1CAB01BC018BEB98E00F94C70120E000
:1075900030E0A901C701B6010F94331587FF05C07C
:1075A00027E137EB41E558EB04C027E137EB41E534
:1075B00058E3C701B6010F941D1CAB01BC0186EB5B
:1075C00098E00F94C7018AE00E942F4E0E9443D694
:1075D000113011F40E94999D0E9433D90C944149B5
:1075E000209377080C9441491DED212E12E0312E95
:1075F0000BECE02E02E1F02E23E437E13DA32CA3B7
:1076000082E2C82E83E1D82E00E010E0D1018D91F6
:107610001D010E9415A8882309F44BC00E9495A75C
:107620002B013C01133049F0F60120813181428168
:1076300053810F941C1C2B013C01ACA1BDA12D91C9
:107640003D914D915C91C301B2010F941C1C4B0103
:107650005C012DEB37E346E855EB0F947D1E87FD6B
:107660000AC02DEB37E346E855E3C501B4010F949A
:1076700033151816F4F4133051F440924F1750920A
:107680005017609251177092521701E012C0A50175
:107690009401F70160817181828193810F941D1C97
:1076A000D7016D937D938D939C931397812F0E94A7
:1076B000C1D21F5FB4E0EB0EF11CECA1FDA134962A
:1076C000FDA3ECA3F4E0CF0ED11C143009F09ECF43
:1076D000002321F08FE497E10E949BA00E9433D900
:1076E0000C94414980912002882311F40C94414963
:1076F00089E40E9415A8082F882321F00E9491A7F1
:10770000E82E01C0E12C8AE40E9415A8182F8823D6
:1077100021F00E9491A7F82E01C0F12C002319F04E
:1077200024E02E1528F0112349F034E03F1530F401
:1077300088EC98E00F9413010C9441490E9453A7E0
:107740000023F1F020914013309141134E2D42035C
:10775000B001439F700D11248091F8129091F9129D
:10776000680F791F072E000C880B990B0F943A15A0
:107770006093111370931213809313139093141347
:107780001123F1F020914213309143134F2D420306
:10779000B001439F700D11248091FA129091FB1259
:1077A000680F791F072E000C880B990B0F943A1560
:1077B00060931513709316138093171390931813F7
:1077C00060E080E50E9422A88823C1F10023D1F067
:1077D00020912E1330912F1340913013509131137B
:1077E00060911113709112138091131390911413DF
:1077F0000F941C1C60931113709312138093131336
:10780000909314131123D1F020913213309133133C
:1078100040913413509135136091151370911613E4
:1078200080911713909118130F941C1C60931513DB
:1078300070931613809317139093181340E050E041
:10784000BA0186E40E94F2AF6B017C0120E030E0D7
:10785000A9010F947D1E181684F420E030E040E763
:1078600052E4C701B6010F94171D60935F02709335
:10787000600280936102909362020E9478D30C941C
:1078800041490E94A7820C9441498091BC12909179
:10789000BD128337910509F4ABC70CF0E1C0893400
:1078A000910509F49CC40CF069C08A31910509F472
:1078B00021C39CF58431910509F496C27CF4813191
:1078C000910509F470C22CF4029708F4E9C10C94F4
:1078D0003549429709F4BDC60C9435498731910565
:1078E00009F4ACC28CF48531910509F4A3C2469722
:1078F00011F00C9435490E945C598091CE16877F17
:107900008093CE160C9441498831910509F4AEC29A
:10791000499709F4E4C20C9435498F31910509F473
:1079200017C47CF48C31910509F45CC30CF4F0C2EB
:107930008D31910509F460C34E9709F464C30C942A
:1079400035498A32910509F423C464F480329105E3
:1079500009F4B8C3819711F00C9435490E9461B6BF
:107960000C9441498B32910509F435C4C09711F04C
:107970000C9435490E9421680C9441498836910540
:1079800009F4D5C4D4F58135910509F450C6C4F481
:107990008C34910509F432C44CF48B34910511F008
:1079A0000C9435490E94859E0C9441498D34910573
:1079B00009F428C48E34910509F428C40C9435497F
:1079C0008435910509F445C674F48235910509F4AE
:1079D0003DC68335910511F00C94354981E08093C3
:1079E00071080C9441498535910509F45EC68C35C2
:1079F000910509F473C60C9435498D36910509F447
:107A0000B5C48CF48A36910509F4D9C50CF4A1C526
:107A10008B36910509F4FBC58C36910511F40C9455
:107A200041490C9435498037910511F40C94414932
:107A300054F48E36910509F4F0C48F36910509F49B
:107A4000FDC40C9435498137910509F43CC5823752
:107A5000910511F00C9435490E9454CF0C94414982
:107A60008E32A1E09A0711F40C9423470CF081C0E8
:107A7000893C910509F4C7C7DCF58937910509F4FC
:107A80006EC7ECF48637910509F42CC734F48537BA
:107A9000910509F416C70C9435498737910509F407
:107AA0005BC78837910511F00C94354981E08093CC
:107AB0003509809334090E9474DA0C9441498B395A
:107AC000910509F456C554F48D37910509F4ACC5F8
:107AD0008C38910509F419C50C9435498E3B9105F4
:107AE00009F425C5883C910509F440C70C94354933
:107AF000833D910511F40C947345F4F48C3C91058D
:107B000009F4C6C734F48B3C910509F4A2C70C9460
:107B100035498D3C910509F4BEC78E3C910511F0A5
:107B20000C9435494DEDC42E42E0D42E59E3E52E98
:107B300059E0F52E10E0C5C7823E910511F40C9472
:107B4000D94554F48C3D910509F4D0C78D3D91057C
:107B500009F4D9C70C9435498232E1E09E0711F44B
:107B60000C9425468D32914011F40C9430460C94BF
:107B70003549843F21E0920711F40C9483480CF0BE
:107B800043C0823941E0940711F40C946D47DCF452
:107B90008033B1E09B0711F40C94B04614F40C94BC
:107BA00067478039F1E09F0711F40C946A478139E7
:107BB000914011F00C94354981E00E94E19D0E94B2
:107BC00033D90C944149843A31E0930711F40C9471
:107BD00080476CF48A39A1E09A0711F40C9441496A
:107BE0008C39914011F40C9475470C943549853AC1
:107BF000E1E09E0711F40C9483478C3A914011F414
:107C00000C94F3470C943549883522E0920711F41F
:107C10000C94AB481CF5873F41E0940711F40C9499
:107C200089487CF4853FB1E09B0711F40C948648A9
:107C3000863F914011F00C9435490E9498EE0C94C7
:107C40004149883FF1E09F0711F40C9492488C3031
:107C5000924011F40C94A3480C9435498C3633E0CF
:107C6000930711F40C9441497CF48B35A2E09A07F8
:107C700011F40C94AE488335934011F00C943549BF
:107C80000E9450C90C944149803AE3E09E0709F4F0
:107C90004FC2873E934011F40C9427490C94354908
:107CA000009174121091751280E50E9415A8882326
:107CB00061F00E940FF96B017C01BB24B394672B28
:107CC000682B692B31F4B12C04C0B12CC12CD12C00
:107CD000760183E50E9415A8882311F40C945E4B6D
:107CE0000E9495A720E030E04AE754E40F949915EC
:107CF0000F94901D6B017C01B1100BC0672B682B9A
:107D0000692B39F40115110521F0D8018C918111ED
:107D100002C0B12C02C0BB24B3940E948AA0B1104F
:107D200003C086E196E001C0C8010E94C8AF10916F
:107D3000780883E08093780881E08093EA1249EF25
:107D400058E062E079E082E00E94F1A887EE98E0D6
:107D50000E94C8AFC114D104E104F104B1F00E9443
:107D600081EEC60ED71EE81EF91E0E9481EEDC01D0
:107D7000CB018C199D09AE09BF09B7FF0EC08091D8
:107D8000EA1281110C94634B08C08091EA12882397
:107D900021F080E00E945B4FF8CF1092EA1210931E
:107DA00078080C9441498091B81284FF02C00C9469
:107DB000684B8091BA1287FF02C00C94684B809187
:107DC000BB12837011F00C94684B60E084E199E081
:107DD0000E94ADE05F988A9880910801817080933D
:107DE000060112980C9441498CE299E00F9413011A
:107DF0001092390B82EB94E10E9402628BE1E2EB7C
:107E0000F4E1DE01119601900D928A95E1F740E0D0
:107E100050E0BE016F5F7F4F80E090E00E94E25A29
:107E2000CE0101960E9438638DE199E00F94130111
:107E30000C9441490E94CD590C944149E09174122F
:107E4000F09175128081882329F0803209F4108224
:107E50003196F8CF40E061E08091741290917512F4
:107E60000E94B85C1092EB120C9441498091CB0AAD
:107E70008823E9F080E090E0A0EAB1E488A399A328
:107E8000AAA3BBA31C8E1D8E1E8E1F8E19821A8262
:107E90001B821C8220E0AE01405E5F4FBE01645E2B
:107EA0007F4FCE0101960E94B1A90C9441490E94D6
:107EB0003EB7882321F00E946D590E94859E40E0C4
:107EC00050E06DE379E085E00E94AAA961E08DECC5
:107ED0009EE20E9437A80E9431E10C9441498091B2
:107EE000CE1682FF03C08B7F8093CE160E9411C5F1
:107EF0000C9441498091CE1683FD02C00C944149F7
:107F000083E50E9415A881110C94844B0C9441497F
:107F100083E40E94CCA78823D9F181E599E00F94EE
:107F2000130180915C14882351F1BE016F5F7F4F74
:107F300089E594E10E94C9608E010F5F1F4FF8012F
:107F400081918F01882319F00E942F4EF8CFBE0136
:107F50006F5F7F4F80E090E00E94805C80916B19A2
:107F6000882389F080E20E942F4E0BE619E1D801A8
:107F70008D918D01882339F00E942F4EF8CF87E430
:107F800099E00F9413018AE00E942F4E0C9441490E
:107F900083E50E9415A8882309F10E946DA7182F78
:107FA00090E0CD970CF01CE3109368080E9481EEDE
:107FB0006B017C01212F30E0A8EEB3E00F94DD1BB4
:107FC000C60ED71EE81EF91EC0926408D09265083E
:107FD000E0926608F09267080C9441490E94355976
:107FE0000C94414940E060E08091741290917512C8
:107FF0000E94B85C0C9441498091CE168E7F80938C
:10800000CE160C9441498091CE1683FD02C00C948B
:1080100041490E94BBEA8091CE1683FD02C00C94B8
:1080200041496091741270917512CE014C960E9474
:108030009AFB8C01009711F40C9441496C8D7D8D55
:1080400019821C8222E0AC01CE0101960E941B67BE
:10805000811102C0F12C14C0CE0101960E9408FBD0
:108060008823C1F361E0CE0101960E94AD600097C4
:1080700089F325EEFC0120831C820E94BC62F82E4D
:10808000CE0101960E943863B801FF2089F08BE78A
:1080900099E00F94E5018AE00E942F4E1092CA16D3
:1080A0001092CB161092CC161092CD160C9441491A
:1080B00083E699E00F94E50180E699E00F941301BF
:1080C0000C9441498091CE1682FD0E948AA0809135
:1080D000CE1683FD02C00C94414960E080E50E9409
:1080E00022A8182F482F61E0809174129091751288
:1080F0000E94B85C83E50E9415A8882381F00E9445
:108100005DA7AB01BC014093CA165093CB16609398
:10811000CC167093CD1689E594E10E94C35F0E944E
:108120006D5911110C9441490E94859E0C9441494E
:1081300020917412309175129091CE1692609093A6
:10814000CE1640E060E0C9010E94B85C0C94414941
:108150000E945DDF6C8F7D8F8E8F9F8FBE016F5F62
:108160007F4FCE014C960E9485B560E0CE0101960E
:108170000E9408E10F94FC01BE016F5F7F4F89E808
:1081800099E00F94E5018AE00E942F4E0C9441493A
:1081900083E50E9415A8882311F40C9441490E949C
:1081A0006DA7F82E6DE070E080E50E94E7908C01ED
:1081B00097FF02C00C944149E82E60E089E40E94D8
:1081C00022A881110C94954B802F0E94574D81114C
:1081D0000DC50C94954B0E94CFC60C94414980E587
:1081E0000E94CCA7882311F40C9441498091CE16AB
:1081F00082FF02C00C9441490C94AE4B0E94ACDF4C
:108200000C9441490E94359F0C94414960E070E014
:1082100083E50E94E7908E34910531F40E94F09F2F
:108220000E9431E10C94414984EF99E00F941301CD
:1082300060912409709125098BEE99E00F94BA01A1
:1082400060912609709127098EED99E00F94BA018B
:108250006091240970912509809126099091270940
:10826000681B790B8091D311815021E030E082307E
:1082700010F020E030E0621B730B83ED99E00F9467
:10828000BA018AE00E942F4E8BEC99E00F94130103
:108290008091280990912909A0912A09B0912B0970
:1082A0008C8F9D8FAE8FBF8FBE016F5F7F4FCE01D2
:1082B0004C960E9485B5BE016F5F7F4F8EEB99E0B3
:1082C0000F94E50180912C0990912D09A0912E0920
:1082D000B0912F098C8F9D8FAE8FBF8FBE016F5FC6
:1082E0007F4FCE014C960E9485B5BE016F5F7F4FD8
:1082F0008EEA99E00F94E50120E030E04AE754E48B
:10830000609130097091310980913209909133095F
:108310000F94171DAB01BC0186E999E00F94C701CA
:108320008DE60E942F4E8AE00E942F4EAAC78091B0
:10833000471083FDA6C70E94E1C387FDA2C783E55E
:108340000E9415A8882379F00E9495A70F94891D93
:108350008B01CB010E94A6BF0135110524F40E94B8
:10836000359F0E9431E10F94BE0E8BC7809147105C
:1083700083FD87C70E94E1C3F82E87FD82C783E58E
:108380000E9415A8082F811106C082E50E9415A839
:10839000182F8823C1F10E9495A70F94891DCB0146
:1083A0000E94A6BF0E9495A720E030E040EA52E478
:1083B0000F943315181614F40C94B94B0E94359F82
:1083C0000E9431E16091B60B7091B70B072E000C43
:1083D000880B990B0F943A154B015C014090B20B3E
:1083E0005090B30B6090B40B7090B50BA301920149
:1083F0000F947D1E181614F40C94CC4B002311F42A
:108400000C94BD4B11E00F94BE0E112309F439C733
:10841000602F8F2D0E94B2B934C78EE40E9415A838
:10842000882309F42EC70E945DA760937012709391
:108430007112809372129093731223C783E50E9486
:10844000CCA7882331F060E083E50E94F69080930A
:1084500047100F94FC0184E29AE00F94130180917D
:108460004710882369F1BAE1EB2EBAE0FB2E00E059
:1084700010E020E08091471090E0A0E0B0E0002EF6
:1084800004C0B695A795979587950A94D2F780FF73
:108490000EC0DD24D394D20E222319F08CE20E9468
:1084A0002F4EF701859194910F9413012D2D0F5F9D
:1084B0001F4FF2E0EF0EF11C05301105D9F663CD28
:1084C00086E19AE05ECD83E50E9415A8882371F0CD
:1084D0000E946DA7282F30E02D3331051CF48093C6
:1084E0000002CFC68CE380930002CBC60F94FC0140
:1084F0004091000250E060E070E08BE29AE00F945F
:10850000A9018AE00E942F4EBCC68091471083FDCE
:10851000B8C683E50E9415A8882309F4B2C60E9454
:1085200095A70F94891DCB010E9445A7AAC68091EB
:10853000471083FDA6C683E50E9415A8182F811158
:108540000C94CF4B82E50E9415A881110C94CF4B5F
:1085500098C60E94E1C3182F87FD9AC680E59AE06D
:108560000F941301812F0E94C2B78AE00E942F4E00
:108570008FC683E50E9415A8882309F482C60E944D
:108580006DA7182F90E0CD970CF01CE310936D08A9
:108590000E9481EE6B017C01212F30E0A8EEB3E058
:1085A0000F94DD1BC60ED71EE81EF91EC092690887
:1085B000D0926A08E0926B08F0926C0862C660E0A4
:1085C00080E50E94F690F82E31E0381708F459C67D
:1085D00081E40E94CCA7882321F060919B0B062F99
:1085E00002C00FEF10E083E50E9415A8882349F030
:1085F0000E945DA78B016F3F710519F010F00FEF1E
:1086000010E0EF2DF0E0E556F44F00833AC660E04D
:1086100080E50E94F690823008F033C6E82FF0E043
:10862000E556F44F10822DC60E9411C52AC60E943D
:10863000B7BF0E94359F0E94CBA10E94994D68EE62
:1086400073E080E090E00F94E4001BC61092710884
:1086500018C683E50E9415A8882399F00E9495A763
:1086600020E030E04AE754E40F9499150F94901DF0
:1086700060930102709302028093030290930402BC
:1086800000C68091B81284FF02C00C94044C809103
:10869000BA1287FF02C00C94044C8091BB12837005
:1086A00011F00C94044C0C94354C83E50E94CCA73B
:1086B000882309F4E6C50E9495A720E030E04AE748
:1086C00054E40F9499150F94901D60937208709361
:1086D00073088093740890937508D3C50E94E1C312
:1086E00087FDCFC59091B81294FD04C09091BA1245
:1086F00097FF0AC0FDEDCF2EF2E0DF2EA8E4EA2EB0
:10870000A0E1FA2E10E009C09091BB12937091F78E
:10871000682F81E00E9494C6B4C5D6018D916D0189
:108720000E9415A8882309F459C0133009F04FC0DE
:108730000E9495A74B015C0120E030E040EA51E443
:108740000F94331587FF3AC0A5019401609168101A
:108750007091691080916A1090916B100F94171DA1
:108760002B013C019B01AC01609178107091791054
:1087700080917A1090917B100F94991560937810E6
:108780007093791080937A1090937B106091930B83
:108790007091940B8091950B9091960B0F943815D6
:1087A000A30192010F9499150F94901D6093930B60
:1087B0007093940B8093950B9093960B8092681016
:1087C00090926910A0926A10B0926B1007C00E943C
:1087D00095A7F701648B758B868B978B1F5FF4E0F1
:1087E000EF0EF11C143009F098CF0E9466A049C525
:1087F00087E79BE00F94130160E087E69BE00E940F
:108800003ACF60E082E59BE00E943ACF61E08BE4E2
:108810009BE00E943ACF61E080E49BE00E943ACF67
:1088200061E080E39BE00E943ACF60E087E29BE05A
:108830000E943ACF61E08DE19BE00E943ACF61E077
:1088400083E19BE00E943ACF61E08BE09BE00E94D5
:108850003ACF61E08DEF9AE00E943ACF61E08FEE6F
:108860009AE00E943ACF60E080EE9AE00E943ACF10
:1088700060E082ED9AE00E943ACF60E08CEB9AE0F3
:108880000E943ACF61E08BEA9AE00E943ACF61E021
:108890008CE99AE00E943ACF61E087E89AE00E9472
:1088A0003ACF61E084E79AE00E943ACF60E087E641
:1088B0009AE00E943ACF60E083E59AE00E943ACFC6
:1088C000E0C48091741290917512009741F0DC0120
:1088D0002C91222321F060E00E9408E1D2C40E9482
:1088E00031E1CFC4009174121091751294E0F12C13
:1088F00040E0915021F1F8018081282F2B7F213415
:1089000021F421812133D9F407C08035C1F481815C
:1089100080538A3048F013C0813421F0853421F42B
:1089200041E002C0FF24F39498012E5F3F4F89017C
:108930002F5F3F4FF80180818032C9F3DACF4111B8
:108940000F94FC01FF2021F082E69CE00F941301BC
:10895000C8010E943A4F95C40E9451DA92C4109205
:108960003509109234090E9474DA8BC40E94E1C365
:10897000182F87FD86C484E40E94CCA7882309F4BD
:108980003FC00E9495A76B017C0101E020E030E030
:10899000A9010F943315811101C000E00093B811B3
:1089A00020E030E0A901C701B6010F9433158823F8
:1089B00039F10E9495A724E01202F0011124E3543A
:1089C000FE4E608371838283938320E030E0A901AF
:1089D0006091BD117091BE118091BF119091C01135
:1089E0000F94331581110CC080E090E0A0EEBFE33E
:1089F0008093BD119093BE11A093BF11B093C0118D
:108A00000E94F5A23EC40E94E1C387FD3AC47DEDF9
:108A1000E72E72E0F72E08E410E1E8E5CE2EE0E163
:108A2000DE2ED7018D917D010E94CCA7882349F0CD
:108A30000E9495A70F94901DF80160837183828333
:108A400093830C5F1F4FC016D10659F70E941FA0D9
:108A500018C40E94E1C387FD14C46DEDE62E62E0E8
:108A6000F62E08E410E1D7018D917D010E94CCA77C
:108A7000882339F00E9495A7F80164A375A386A303
:108A800097A30C5F1F4FF0E108351F0761F7F9C38B
:108A90000E9499F8F6C38091B81281FDE9C68091D1
:108AA000B91281FDE5C68091BA128C7009F0E0C65A
:108AB000E8C31F5FF4E0EF0EF11C133011F40C94C7
:108AC0006E3BD6018D916D010E94CCA7882389F35E
:108AD0000E9495A7F7016083718382839383812F1E
:108AE0000E94C1D2E6CF0E94DFC5CBC383E50E94BE
:108AF00015A8882309F4C5C30E9491A79093560234
:108B000080935502BEC30E94E1C3F82E87FDB9C30E
:108B100083E50E9415A80F2D0F2C000C110B882344
:108B200069F10E9491A7F801EE0FFF1FEA5DFD4F6A
:108B300091838083000F111F000F111F98012B5E7E
:108B40003D4F7901BC01990F880B990B0F943A1591
:108B50002AE037ED43E25CE30F949915F801E754FE
:108B6000FE4E20813181428153810F949915D701A6
:108B70006D937D938D939C93139783C30F94FC0106
:108B800085E40E942F4E80E38F0D0E942F4EF80146
:108B9000EE0FFF1FEA5DFD4F6081718185E89CE06B
:108BA0000F94D80185E20E942F4E8AE00E942F4E3A
:108BB00068C380E50E94CCA7882309F462C360E003
:108BC00070E080E50E94E790F82E6FEF7FEF83E57D
:108BD0000E94E7908C010196039708F052C3F7FCBE
:108BE00050C38F2D0E94574D882339F00F94F80100
:108BF0008DE89CE00F94130144C30E948AA060E0BA
:108C00008F2D0E9423ED0F3FBFEF1B0731F0013086
:108C1000110571F000E010E00DC08F2D0E94CBEC2B
:108C200031E020E0892B09F030E0032F122F02C041
:108C300001E010E08F2D0E94CBEC8017910709F422
:108C400020C380E00E945B4FF5CF8AE50E9415A803
:108C5000811167C683E50E9415A8811162C611C300
:108C600060E085E40E94F690811173C080E50E9467
:108C7000CCA7882351F00E9495A76093B90B7093FD
:108C8000BA0B8093BB0B9093BC0B89E40E94CCA7DA
:108C9000882381F00E9495A72CEA35EC47E25EE339
:108CA0000F9499156093BD0B7093BE0B8093BF0B0F
:108CB0009093C00B84E40E94CCA7882381F00E948B
:108CC00095A72CEA35EC47E25EE30F94171D6093FD
:108CD000C10B7093C20B8093C30B9093C40B0F9482
:108CE000FC014091B90B5091BA0B6091BB0B709194
:108CF000BC0B87EC9CE00F94C7012CEA35EC47E2F3
:108D00005EE36091BD0B7091BE0B8091BF0B9091A3
:108D1000C00B0F94171DAB01BC0183EC9CE00F94BA
:108D2000C7012CEA35EC47E25EE36091C10B70911C
:108D3000C20B8091C30B9091C40B0F949915AB019A
:108D4000BC018FEB9CE00F94C7018AE00E942F4E7C
:108D500098C20F94F8018DEA9CE00F94130191C220
:108D600080E50E94CCA7882351F00E9495A76093CC
:108D7000140970931509809316099093170989E4D3
:108D80000E94CCA7882381F00E9495A72CEA35EC9D
:108D900047E25EE30F9499156093180970931909DF
:108DA00080931A0990931B0984E40E94CCA788231E
:108DB00081F00E9495A72CEA35EC47E25EE30F9420
:108DC000171D60931C0970931D0980931E099093D1
:108DD0001F090F94FC0140911409509115096091ED
:108DE00016097091170983ED9CE00F94C7012CEAD6
:108DF00035EC47E25EE360911809709119098091A2
:108E00001A0990911B090F94171DAB01BC018FEC3F
:108E10009CE00F94C7012CEA35EC47E25EE36091D9
:108E20001C0970911D0980911E0990911F090F94D2
:108E30009915AB01BC018BEC9CE00F94C7018AE053
:108E40000E942F4E1EC283E50E94CCA7182F8823B4
:108E500071F00E9495A70F94891D70931A02609378
:108E6000190221E0672B09F020E02093AD0B80E58B
:108E70000E94CCA7882359F02091190230911A0240
:108E8000232B11F00E9481A78093AD0BFAC1111121
:108E9000F8C10F94FC0183EF9CE00F9413018091C3
:108EA000AD0B882319F08BED9CE002C087ED9CE0B0
:108EB0000F9413016091190270911A0282EE9CE0E6
:108EC0000F94D8018EED9CE00F941301DAC10E943B
:108ED00009B0D7C10E948AA0D4C180E00E94E19D60
:108EE0000E94999D0E9433D9CCC18091B812887894
:108EF00009F07CC58091BA12867009F077C5A6C5C5
:108F00000E940291BEC16FEF7FEF89E40E94E7905B
:108F1000F82E6FEF7FEF8AE40E94E790E82E8AE553
:108F20000E94CCA7182F811105C081E50E94CCA713
:108F3000B82E01C0B12CF7FC06C0E7FC04C011112B
:108F400009C0B11007C00F94F8018DE59DE00F94A2
:108F5000130197C1E4E0EF1510F0EE1538F40F940B
:108F6000F8018EE39DE00F9413018BC1CF2C0F2CE1
:108F7000000CDD080E2D0E2C000C110B0E9495A785
:108F8000BB2099F025E02C9DF0012D9DF00D1124C2
:108F9000E00FF11FEE0FFF1FEE0FFF1FE45BFC4E13
:108FA000208131814281538103C020E030E0A9015A
:108FB0000F941D1C9B01AC0185E08C9DF0018D9DE3
:108FC000F00D1124E00FF11FEE0FFF1FEE0FFF1F3A
:108FD000E45BFC4E20833183428353836E2D8F2DBF
:108FE0000E94C4AE4EC10E94CF8281114AC10AE2E2
:108FF0001EE223E437E13DA32CA3CE0101965C01E0
:109000004FE7842E4EE2942E1C01F8016591759174
:1090100085919491ACA1BDA1CD90DD90ED90FD9096
:10902000BDA3ACA3A70196010F941C1C2B013C010E
:10903000F101608371838283938320E030E040EA12
:1090400051EC0F947D1E87FD0AC020E030E040EA1D
:1090500051E4C301B2010F94331518162CF4F40136
:10906000849118160CF416C5D101CD90DD90ED90C9
:10907000FD901D0120E030E040EA51ECC701B6014F
:109080000F947D1E87FD0AC020E030E040EA51E4E5
:10909000C701B6010F943315181664F40F94F80144
:1090A0008BE99DE00F94130161E08DE89DE00E9443
:1090B000ADE0E7C00C5F1F4FBFEF8B1A9B0AEEE2DB
:1090C00006331E0709F0A1CF39E3E32E39E0F32E72
:1090D00010E0F50181919191A191B1915F01F701AA
:1090E00081939193A193B1937F01812F0E94C1D26B
:1090F0001F5F133071F70E9433D960E08DE79DE068
:109100000E94ADE0BEC00E9483DABBC00E94E2F2C2
:10911000B8C061E083E50E9422A891E089270E94FF
:10912000D9EFAFC081E080933B130E94A6E110927B
:109130003B13882309F4A5C00F94FC0189EB9DE043
:109140000F9413019EC08091CE1682FF9AC0806258
:109150008093CE1696C00E940AC493C00E94E1C3B9
:10916000082F87FD8EC085E50E94CCA78823B1F12A
:10917000E02E002E000CFF080E9495A74B015C0119
:1091800020E030E0A9010F947D1E87FF04C0B7FAEC
:10919000B094B7F8B094C70123E0880F991F2A95BF
:1091A000E1F79C012C5B3C4E7901D9018D929D9297
:1091B000AD92BC92139720E030E04AEF53E4C50132
:1091C000B4010F947D1E18164CF480E090E0AAEFD5
:1091D000B3E4F70180839183A283B3838CE40E947C
:1091E000CCA7882309F44DC0002E000C110B0E945F
:1091F00095A76B017C0120E030E0A9010F947D1E52
:1092000087FF04C0F7FAF094F7F8F09420E030E01C
:109210004AEF53E4C701B6010F947D1E980193E015
:10922000220F331F9A95E1F7F901EC5BFC4E1816FB
:109230002CF0C482D582E682F78223C080E090E0E1
:10924000AAEFB3E484839583A683B7831AC081E031
:109250008093200210927F0B60E083E50E9422A899
:1092600081110FC00E944CB70CC00E94A78209C098
:109270008091BC12882329F00E940C6802C00E94D1
:10928000A7822296FFAD2297F11102C00E9459C811
:109290002CAD20937808CF5BDF4F0FB6F894DEBF7C
:1092A0000FBECDBFDF91CF911F910F91FF90EF9037
:1092B000DF90CF90BF90AF909F908F907F906F90F6
:1092C0005F904F903F902F9008950E948AA0309118
:1092D0005B173CAB80E00E948DAC0E945CD681E0C5
:1092E000809335090E9474DA88E50E94CCA7182F74
:1092F00089E50E94CCA7082F8AE50E94CCA710130D
:10930000BDC1181711F0012FB9C101E011E091E0C2
:109310009CA70E9453A782E50E9415A8882361F0AC
:109320000E9495A76B017C0120E030E0A9010F9419
:109330003315882369F106C0C12CD12C90E8E92EA1
:1093400090E4F92E111103C0002309F4FCC0C0926F
:109350001913D0921A13E0921B13F0921C13A70159
:10936000960160914B1770914C1780914D17909119
:109370004E170F94331587FF0BC019821A821B8278
:109380001C82BE016F5F7F4F89E193E10E945ED72F
:10939000112309F4D3C0002309F4CDC0109247175C
:1093A000109248171092491710924A1710924317BB
:1093B0001092441710924517109246170E9407D832
:1093C000EFE7FEE2A491A8AFE3E7FEE2C590D590F7
:1093D000E590F490E7E7FEE285909590A590B49033
:1093E000A5019401C701B6010F947D1E18162CF437
:1093F000A7019601C501B40104C0A5019401C701EC
:10940000B6010F94171D2B013C01EAE3FEE28591A2
:109410009591A591B4918CA39DA3AEA3BFA3E6E3C0
:10942000FEE285919591A591B49188A799A7AAA7E5
:10943000BBA79C01AD016CA17DA18EA19FA10F9442
:109440007D1E181634F428A439A49AA598AB1BA540
:1094500005C02CA03DA0AEA1A8AB1FA1A301920105
:10946000C301B2010F94991520E030E040E85FE3BA
:109470000F941D1C0F94CB1E910148A9512F0F94DE
:10948000991568A379A38AA39BA3E0E8FEE214914F
:1094900020E030E040EC5FE3C501B4010F94991582
:1094A0004B015C01612F110F770B880B990B0F9407
:1094B0003A159B01AC01C501B4010F94991569835C
:1094C0007A838B839C8320E030E040EC5FE3C7012C
:1094D000B6010F9499156B017C01B8AD6B2FBB0FD2
:1094E000770B880B990B0F943A159B01AC01C701C0
:1094F000B6010F9499156C8F7D8F8E8F9F8FAE0163
:10950000405E5F4FBE016F5F7F4FCE014C960E9461
:109510003CD70E948DEE1092471710924817109278
:10952000491710924A17109243171092441710923D
:1095300045171092461780E00E9409D8002319F0C1
:1095400081E00E9409D8ECA5EE2309F489C080913E
:10955000BA138370833051F060E08DEC97E00E9485
:10956000ADE00F94FC018EEB97E093C00E9407D80A
:1095700080914B1790914C17A0914D17B0914E17B9
:109580008093191390931A13A0931B13B0931C1379
:1095900020912E1330912F1340913013509131139D
:1095A00060E070E088E492E40F941C1C6B017C0185
:1095B00060931113709312138093131390931413E9
:1095C000209132133091331340913413509135135D
:1095D00060E070E088E492E40F941C1C4B015C0195
:1095E00060931513709316138093171390931813A9
:1095F00027E137EB41ED58EB0F947D1E87FD40C00E
:1096000023E030E04BE953E4C501B4010F94331576
:109610001816B4F127E137EB41ED58EBC701B6015D
:109620000F947D1E87FD2CC023E030E84DE953E404
:10963000C701B6010F943315181614F119821A8256
:109640001B821C82AE014F5F5F4F65E173E181E1D8
:1096500093E10E943CD782E00E9409D80E94999D24
:109660000E9407D880913409809335098CA90E9403
:109670008DAC0E9443D60E9433D903CE8CA749CE2D
:1096800060E08DEA97E00E94ADE00F94FC018BE969
:1096900097E00F941301E2CF61E081E998E00E9426
:1096A00037A88CE198E00E94C6D061E08FEA9EE284
:1096B0000E9437A88DE098E00E9433FAB1100C9414
:1096C000893E0C94823E80E00E945B4F0C94B53E34
:1096D00088E50E94CCA781115F9889E50E94CCA7FC
:1096E00081118A988AE50E94CCA7882329F080916D
:1096F000080181708093060185E40E94CCA788232D
:1097000009F4BFCD1298BDCD0E945DA7AB01BC018D
:109710004093CA165093CB166093CC167093CD1617
:1097200089E594E10E94C35FACCD61E0802F0E9487
:1097300023ED6F2D802F0E94F4EC6F2D70E0802FB1
:109740000E945FED47E0E41203C0F0929C0B99CDBC
:1097500089E0E81296CDF0929B0B93CD0E946DA705
:1097600090E08536910514F084E690E08093EB124A
:1097700088CD0E94859E0C94E241A3019201C5010F
:10978000B4010F947D1E18163CF08CEF99E060E058
:109790000E94ADE00C94024289E09AE0F8CF0E946A
:1097A00095A70F94891DCB010E9445A70E9495A7FC
:1097B00020E030E040EA50E40F947D1E181614F4C7
:1097C0000E94859E6091110970911209072E000C6C
:1097D000880B990B0F943A1520910D0930910E09C1
:1097E00040910F09509110090F947D1E18161CF41A
:1097F00081E49AE002C082E39AE060E00E94ADE07A
:10980000812F0E9434B83DCD0E948AA088E50E9435
:10981000CCA7882331F05F9A8091BA138E7F809312
:10982000BA1389E50E94CCA7882331F08A9A8091E7
:10983000BA138D7F8093BA138AE50E94CCA7882340
:1098400059F0809108018095817080930601809184
:10985000BA138B7F8093BA1385E40E94CCA7882328
:1098600009F40FCD0E94554D0CCD0E94CBA109CD1E
:1098700082E40E94CCA7882351F00E940FF96093E4
:1098800058107093591080935A1090935B1083E591
:109890000E94CCA7882351F00E9495A7609388105E
:1098A0007093891080938A1090938B1084E50E94A6
:1098B000CCA7882351F00E9495A760938C107093D9
:1098C0008D1080938E1090938F108AE40E94CCA705
:1098D000882309F4D6CC0E9495A76B017C012AE06D
:1098E00037ED43E25CE30F947D1E87FD13C02AE948
:1098F00039E949E95EE3C701B6010F94331518163B
:109900004CF0C092830BD092840BE092850BF092C6
:10991000860BB7CC0F94F80186E69CE00F941301F8
:10992000B0CC0E9495A720E030E040E050EC0F94CE
:10993000331587FD15C00E9495A720E030E040E078
:1099400050E40F947D1E18162CF00E9495A76B0111
:109950007C010BC0C12CD12CE12C10E4F12E05C0F0
:10996000C12CD12CE12CB0ECFB2E20916410309155
:1099700065104091661050916710C701B6010F94B1
:1099800099150F94891DCB010E9482FC80E50E94ED
:10999000CCA7882329F00E9481A7882309F471CCE1
:1099A000A701960160913613709137138091381397
:1099B000909139130F941D1C6093361370933713D5
:1099C00080933813909339130F94FC014091361310
:1099D0005091371360913813709139138CE99CE0E2
:1099E0000F94C7018AE00E942F4E4BCC88E40E945E
:1099F000CCA7882321F00E9481A78093760882E576
:109A00000E94CCA7082F83E50E94CCA7182F011134
:109A100002C0882351F0109207090E947C4D112347
:109A200021F00E9481A780931B0284E40E94CCA7AE
:109A3000882309F426CC0E9495A760936302709353
:109A4000640280936502909366021BCC0F94FC0124
:109A50008DE29DE00F94130180911B02811117C0CC
:109A600086E09DE00F9413018AE00E942F4E409102
:109A700063025091640260916502709166028DE00C
:109A80009DE00F94C7018AE00E942F4EFACB8AE036
:109A90009DE0E8CFF7FAF094F7F8F094D101CD9279
:109AA000DD92ED92FC921397DFCA129A0895FF920D
:109AB0000F931F93CF93DF931F92CDB7DEB7F82E8E
:109AC0000EED1DE041E050E0B801CE0101960F948B
:109AD0006D1489818F1102C081E007C00F5F1F4F95
:109AE0008DE0073F180771F780E00F90DF91CF916D
:109AF0001F910F91FF9008958091630290916402ED
:109B0000A0916502B09166028093A5109093A61073
:109B1000A093A710B093A810089580917E0881119A
:109B200007C00E94E2F2882319F081E080937E084A
:109B30000895EBE9FBE01082118208958F929F92C5
:109B4000AF92BF92CF92DF92EF92FF920F93CF939B
:109B5000DF931F92CDB7DEB75C016B017A0149013B
:109B6000F501808191810F94631B8983002311F09B
:109B7000F6018083BE016F5F7F4FC4010E9424F90C
:109B8000F50180819181019691838083FFEFCF1A47
:109B9000DF0A81E0E81AF10819F780E00F90DF9101
:109BA000CF910F91FF90EF90DF90CF90BF90AF904B
:109BB0009F908F9008957F928F929F92AF92BF92C5
:109BC000CF92DF92EF92FF920F931F93CF93DF9389
:109BD0001F92CDB7DEB77C0159018B016B01C40E1A
:109BE000D51E0C151D0559F1F70180809180F801F3
:109BF00071908F017982C4010F94631B781691F0E4
:109C0000672DC4010F946B1BC4010F94631B9981D2
:109C1000891741F00F94FC0184EC9DE00F9413012F
:109C200081E00EC0BE016F5F7F4FC5010E9424F925
:109C3000F70180819181019691838083D2CF80E06A
:109C40000F90DF91CF911F910F91FF90EF90DF90D8
:109C5000CF90BF90AF909F908F907F9008959091FC
:109C6000C00095FFFCCF8093C60008958F929F920D
:109C7000AF92BF92EF92FF920F931F93CF93DF9318
:109C8000CDB7DEB7A0970FB6F894DEBF0FBECDBF3D
:109C9000611571058105910591F100E0842E912CEB
:109CA000A12CB12C102FEE24E394F12CEC0EFD1E10
:109CB000E00EF11C07FDFA94A50194010F94891B95
:109CC000F7016083B901CA010F5F61157105810554
:109CD000910541F71F3F31F1E1E0F0E0EC0FFD1F8E
:109CE000E10FF11D17FDFA9580818A3010F097E39E
:109CF00001C090E3890F0E942F4E1150EBCF80E3FB
:109D0000A0960FB6F894DEBF0FBECDBFDF91CF9106
:109D10001F910F91FF90EF90BF90AF909F908F9009
:109D20000C942F4EA0960FB6F894DEBF0FBECDBF99
:109D3000DF91CF911F910F91FF90EF90BF90AF9067
:109D40009F908F900895CF92DF92EF92FF926B01D8
:109D50007C0197FF0BC08DE20E942F4EF094E0949F
:109D6000D094C094C11CD11CE11CF11C4AE0C70175
:109D7000B601FF90EF90DF90CF900C94364E8F920B
:109D80009F92AF92BF92CF92DF92EF92FF92CF93CA
:109D90006B017C01B42E20E030E0A9010F94331553
:109DA00087FF07C08DE20E942F4EF7FAF094F7F874
:109DB000F094C0E060E070E080E09FE3CB1541F0FC
:109DC0002DEC3CEC4CEC5DE30F949915CF5FF6CF96
:109DD0009B01AC01C701B6010F941D1C6B017C01F6
:109DE0000F94901D4B015C014AE00E94364ECC233B
:109DF00089F1C501B4010F9438159B01AC01C7016D
:109E0000B6010F941C1C6B017C018EE20E942F4E48
:109E100020E030E040E251E4C701B6010F9499150B
:109E20004B015C010F94891D6B01770FEE08FF0851
:109E3000C701B6010E94A34EC701B6010F943A159F
:109E40009B01AC01C501B4010F941C1C6B017C018A
:109E5000C150F1F6CF91FF90EF90DF90CF90BF907F
:109E6000AF909F908F9008958DE00E942F4E8AE0D2
:109E70000C942F4ECF93DF93EC018991882319F036
:109E80000E942F4EFACFDF91CF910C94344F8091E6
:109E9000EC119091ED11981759F0E92FF0E0E45191
:109EA000FE4E82819F5F9F779093ED1190E0089521
:109EB0008FEF9FEF08952F923F924F925F926F9294
:109EC0007F928F929F92AF92BF92CF92DF92EF924A
:109ED000FF920F931F93CF93DF93CDB7DEB72897F1
:109EE0000FB6F894DEBF0FBECDBFE82E0E946D1BEB
:109EF0000E9481EE4B015C0180910002882359F1A0
:109F000080917808882339F140917F08509180082A
:109F1000609181087091820895018401041B150BE2
:109F2000260B370B37FD2AC0833079F03CF48130A3
:109F300094F00F94FC0186E29EE00BC0843059F44B
:109F40000F94FC0187EF9DE004C00F94FC018FE0AB
:109F50009EE00F9413012091000230E0A8EEB3E0E0
:109F60000F94DD1B860E971EA81EB91E80927F08D7
:109F700090928008A0928108B092820880911B0282
:109F8000882319F18091070981111FC08091CE1695
:109F900082FD08C08091D311813021F08091CB0ADD
:109FA000882399F0F894649919C66091A51070916E
:109FB000A6108091A7109091A810789420E030E02E
:109FC000A9010F94331587FD99C58091C90A843082
:109FD00008F07EC20E9481EE4B015C018091C90AAB
:109FE00081111DC08091EC119091ED11891B8F772B
:109FF000B1F48091E8089091E908A091EA08B09145
:10A00000EB08A5019401281B390B4A0B5B0BDA0105
:10A01000C901885E9340A109B109B7FFF0C570E698
:10A02000F72E8091C90A843008F035C18091EC1177
:10A030009091ED11891B8F7709F42DC10E94474F34
:10A04000AC0197FDEECF20916E1230916F128A30E5
:10A0500019F08D3009F0ECC01092E7082115310598
:10A0600019F40E94FB83DDCFF901E957F74F108205
:10A0700010926F1210926E1207E818E0F8018191A9
:10A08000803211F48F01FACF8E3409F07AC00115B5
:10A09000110509F476C068EA7FE0C8010F94B11495
:10A0A0006C01892B41F06EE470E0C80104960F94B6
:10A0B000701F009709F4C8014AE050E060E070E0CA
:10A0C00001960F94291260938308709384088093FB
:10A0D000850890938608409070125090711260909D
:10A0E0007212709073123FEF431A530A630A730A95
:10A0F000641575058605970531F0CD2821F460E0DB
:10A1000085E79FE051C06AE270E0C8010F949F1F8D
:10A110009C01009709F1982F901BD12C992339F0BD
:10A120009150F801E90FF11D8081D826F7CF4AE060
:10A1300050E060E070E0C90101960F9429124D2CA7
:10A14000512C612C712C641575058605970541F01D
:10A1500060E086E59FE028C060E08CE29FE024C0DC
:10A160008091830890918408A0918508B091860819
:10A170008093701290937112A0937212B093731225
:10A1800016C08091CE1680FF12C064E271E1C80152
:10A190000F94B114009729F0FC01838180538A3019
:10A1A00030F460E082E09FE00E9468B774C0809164
:10A1B000200281111CC067E470E0C8010F94701F79
:10A1C0000097A9F04AE050E060E070E001960F943B
:10A1D0002912643071058105910548F48BE89EE0F1
:10A1E0000F94130160E081E89EE00E94ADE0809250
:10A1F000E8089092E908A092EA08B092EB088091F2
:10A2000087088B3309F40DCF8091C90A843008F098
:10A2100008CF80914509F89EC001112467E878E0D5
:10A22000885B964F0F947B1F81E00E94AEC8F9CEE9
:10A230002F3531050CF0F5CE8C35C1F40E94474F17
:10A2400097FDEFCE2091E7082111EBCE20916E1201
:10A2500030916F12A9014F5F5F4F50936F1240937F
:10A260006E12F901E957F74F8083DBCE8B3321F46F
:10A2700081E08093E708D5CE8091E7088111D1CEA7
:10A28000C901019690936F1280936E12F901E957FC
:10A29000F74F4083C6CE8091CE1682FF19C18091C0
:10A2A000C90A811102C01092ED08DD24D3944091B7
:10A2B000CA165091CB166091CC167091CD16809134
:10A2C000C6169091C716A091C816B091C916481726
:10A2D00059076A077B0708F4D12C00E010E0CC2472
:10A2E000C39440E6B42E54E6A52E69E6962E8091DE
:10A2F000C90A843008F0ECC0D110EAC08091ED08A2
:10A300008111E6C08091611490916214A091631450
:10A31000B09164148093CA169093CB16A093CC1678
:10A32000B093CD1641E050E0BE016F5F7F4F89E5ED
:10A3300094E10E94A863019719F4898190E002C01A
:10A340008FEF9FEFF82E4090CA165090CB1660907A
:10A35000CC167090CD164091C6165091C7166091DC
:10A36000C8167091C916DD24D394441655066606A6
:10A37000770608F4D12C4416550666067706B0F425
:10A38000019609F461C02AE0F21609F46EC03DE0BE
:10A39000F31609F46AC043E2F41619F05AE3F51211
:10A3A0007CC08091EC08811178C054C00E948AA0C2
:10A3B00089E594E10E942F638091C516882339F1C5
:10A3C00081508093C516989EC001112441E061E040
:10A3D0008053954F0E94B85CE091C51664E0E69FFB
:10A3E000F0011124E453F54F408151816281738162
:10A3F0004093CA165093CB166093CC167093CD162B
:10A4000089E594E10E94C35F0E946D5916C00E94C5
:10A410005C590E94CBA10E94359F0E945DDF6D3385
:10A4200071058105910518F483EB9FE002C088EB6C
:10A430009FE00E94F5C8A092EB128091CE1682FD9B
:10A440000DC08BEC9FE004C00F94F8018CEB9FE0F3
:10A450000F94130173E2F71208C005C053E2F5121E
:10A46000DBC300E010E0C092ED081092EC0801158B
:10A47000110519F40E94FB830DC080914509B89E17
:10A48000000D111D1124F801E85BF64F108280E0E9
:10A490000E94AEC800E010E02ACF0F35110508F089
:10A4A00026CF8BE3F81203C0C092EC0820CF809136
:10A4B000EC0881111CCF80914509F801B89EE00D90
:10A4C000F11D1124E85BF64FF0820F5F1F4F0FCF95
:10A4D0000E9481EE4B015C0140917208509173081B
:10A4E00060917408709175084115510561057105F9
:10A4F00029F18091B2139091B313A091B413B0914C
:10A50000B513840F951FA61FB71F95018401081B63
:10A51000190B2A0B3B0B37FD11C00F94F80160910A
:10A52000810B7091820B8FED9FE00F94E5018AE023
:10A530000E942F4E80E090E00E9433FA4091010289
:10A54000509102026091030270910402411551057D
:10A550006105710509F44EC09091D0148091D11419
:10A56000981759F00E9481EE6093B2137093B31361
:10A570008093B4139093B5133DC08091CB0A8111A1
:10A5800037C0E11035C08091B2139091B313A09100
:10A59000B413B091B513840F951FA61FB71FA50163
:10A5A0009401281B390B4A0B5B0B57FD21C080918E
:10A5B000FE0881111FC081E08093FE085F9A8091A0
:10A5C000BA138E7F8093BA138A9A8091BA138D7FC3
:10A5D0008093BA1380910801809581708093060161
:10A5E0008091BA138B7F8093BA130E94554D02C09D
:10A5F0001092FE088091FA089091FB08A091FC0847
:10A60000B091FD08B501A401481B590B6A0B7B0BE7
:10A6100077FDBCC12091D0149091D1148091350266
:10A6200010913602291317C060919B0B869FB001D1
:10A630001124660F672F661F770B7195062F809187
:10A640009C0B189FB0011124660F672F661F770BB4
:10A650007195162F29C02091D11458E4259F90019F
:10A6600011242B53344FF901EA5BFF4F6081869F21
:10A67000B0011124660F672F661F770B7195062FA7
:10A6800031968081819FB0011124660F672F661F6C
:10A69000770B7195162F8091D1149091D014981743
:10A6A00019F08F5F8F70F9CF002331F10E9481EE96
:10A6B000C090F208D090F308E090F408F090F5080C
:10A6C000DC01CB01C114D104E104F10469F48C591B
:10A6D0009F4FAF4FBF4F8093F2089093F308A09322
:10A6E000F408B093F50806C08C199D09AE09BF099E
:10A6F000B7FF0AC00FEF08C01092F2081092F308DB
:10A700001092F4081092F508602F70E089E00E9422
:10A710005FED112331F10E9481EEC090F608D090D8
:10A72000F708E090F808F090F908DC01CB01C114BB
:10A73000D104E104F10469F48C599F4FAF4FBF4F2E
:10A740008093F6089093F708A093F808B093F9085F
:10A7500006C08C199D09AE09BF09B7FF0AC01FEFDB
:10A7600008C01092F6081092F7081092F80810929C
:10A77000F908612F70E087E00E945FED80918C12F4
:10A78000882309F4F6C0E0902C02F0902D0200918D
:10A790002E0210912F026091B60B7091B70B6E5F75
:10A7A0007F4F072E000C880B990B0F943A159701D9
:10A7B000A8010F94331587FDDCC03090D114212CF3
:10A7C0001A821B821C828091D014831509F467C001
:10A7D000832D90E068E4689FF001699FF00D1124DB
:10A7E000EB53F44F458956896789708D452B462B6D
:10A7F000472B89F4418D528D638D748D452B462BEB
:10A80000472B49F4458D568D678D70A1452B462BFE
:10A81000472B09F43FC078E4789F9001799F300D71
:10A820001124C9018B53944F6C01FC016181728129
:10A83000838194810F94CB1E2B013C01F60161A111
:10A8400072A183A194A10F9438156D837E838F83A9
:10A850009887F60165A176A187A190A50F94381578
:10A860009B01AC016D817E818F8198850F94171DAE
:10A87000A30192010F9499153B016C01222D3A819D
:10A880004B815C810F947D1E181624F4262C7A824D
:10A89000CB82DC8281E0830D8F70382E94CF2091A3
:10A8A0003002309131024091320250913302622DD8
:10A8B0007A818B819C810F9499159701A8010F943F
:10A8C0001D1C3B016C012090280230902902409011
:10A8D0002A0250902B029B01AC01B701C8010F94D2
:10A8E0007D1E18166CF09101A201B301C6010F94F0
:10A8F0007D1E18161CF47101820102C073018601CD
:10A900004090EE085090EF086090F0087090F108C9
:10A910009701A801C301B2010F947D1E1816C4F45B
:10A9200020E037ED43EA5CE3B701C8010F949915C5
:10A930006B017C0128E431EE4AE75FE3C301B20119
:10A940000F949915A70196010F941D1C7B018C0192
:10A95000C701D8018093EE089093EF08A093F00808
:10A96000B093F108B701C8010F94891DCB010E9473
:10A97000A6BFF4E68F0E911CA11CB11C8092FA08B0
:10A980009092FB08A092FC08B092FD080E94FB8305
:10A990008091D311813009F06EC00E9481EE6B016D
:10A9A0007C018091030990910409A0910509B0915F
:10A9B000060997018601081B190B2A0B3B0B37FD73
:10A9C0003AC08090D4119090D511A090D611B0903B
:10A9D000D7110E945DDF6093D4117093D5118093DD
:10A9E000D6119093D711009128091091290920912F
:10A9F0002A0930912B09081919092A093B09DC0198
:10AA0000CB01800F911FA21FB31F80932809909341
:10AA10002909A0932A09B0932B09D701C601805FA9
:10AA2000984DAF4FBF4F8093030990930409A093B3
:10AA30000509B09306098091FF0890910009A09143
:10AA40000109B0910209A7019601281B390B4A0B95
:10AA50005B0B57FD10C030E8C30E3EEED31EE11C69
:10AA6000F11CC092FF08D0920009E0920109F09217
:10AA700002090E940F9F80916D08882391F00E9427
:10AA800081EE0091690810916A0820916B0830915D
:10AA90006C08DC01CB01801B910BA20BB30BB7FF41
:10AAA000BEC00E9481EE6B017C01209168082223C8
:10AAB00009F4D3C08091640890916508A09166085C
:10AAC000B0916708B701A601481B590B6A0B7B0BB5
:10AAD00077FDC3C030E0A8EEB3E00F94DD1BC60ED7
:10AAE000D71EE81EF91EC0926408D0926508E09255
:10AAF0006608F09267080E943559AFC011E01093C4
:10AB000007098091CB0A811166C089E296E00E9414
:10AB10003A4F84E08093CD1182E08093440881E035
:10AB20009AE590935315809352158EE490E090939C
:10AB300055158093541587E08093461582E88093DD
:10AB4000491584E890E0A0E0B0E080934A15909326
:10AB50004B15A0934C15B0934D150E948DF9109391
:10AB6000D8110E945BA840E060E77EE08AE692E2AE
:10AB70000E9467A880E30E942F4E8AE00E942F4E19
:10AB80000E944FA88091760860E0182719F08AE4A7
:10AB900091E20DC08EE59EE00E9437A880E30E94FE
:10ABA0002F4E8AE00E942F4E60E088E39EE00E94D4
:10ABB00037A88CE49EE00F94130180E30E942F4E8F
:10ABC0008AE00E942F4E112331F08EE39EE0909395
:10ABD0004709809346090E948AA0F7C980916302C1
:10ABE00090916402A0916502B09166028093A510D5
:10ABF0009093A610A093A710B093A810D6C98DEA81
:10AC00009FE00F9413018092E8089092E908A092C7
:10AC1000EA08B092EB0803CA1092EC082BCC0E9411
:10AC200081EE6B017C0120916D0830E0A8EEB3E06D
:10AC30000F94DD1BC60ED71EE81EF91EC0926908D0
:10AC4000D0926A08E0926B08F0926C0880E00E9453
:10AC5000C2B78AE00E942F4E24CF28960FB6F894F0
:10AC6000DEBF0FBECDBFDF91CF911F910F91FF903F
:10AC7000EF90DF90CF90BF90AF909F908F907F909C
:10AC80006F905F904F903F902F9008951F920F927A
:10AC90000FB60F9211240F900FBE0F901F901895B2
:10ACA0001F920F920FB60F9211240BB60F920F93B3
:10ACB0001F932F933F934F935F936F937F938F9344
:10ACC0009F93AF93BF93CF93DF93EF93FF93009145
:10ACD000ED11D091EC1111E01D0F1F77C091C6004E
:10ACE00090917D08492F092E000C550B660B770BB0
:10ACF0004131510508F064C0FA018827E256FF4F40
:10AD00008F4F0D94141CCD3449F0CE34B9F481E04A
:10AD100006C0CA3338F0CD3409F043C082E08093D6
:10AD20007D0876C0C03308F073C0C03209F470C02B
:10AD3000CD32B9F56DC0C13351F018F4C03289F588
:10AD400067C0C43331F0C83361F58BE0E8CF83E0EE
:10AD5000E6CF88E0E4CFC03321F0C13311F586E0BF
:10AD6000DECF84E0DCCFC833E1F485E0D8CFC23356
:10AD7000C1F487E0D4CFC133A1F489E0D0CFC03390
:10AD800081F48AE0CCCFC73361F48CE0C8CFC633FE
:10AD900041F48DE0C4CFC032D9F1C33511F48EE057
:10ADA000BECF80E1BCCF80ED8C0F8A3088F59FE06C
:10ADB00090937D0880937C082BC0CA3049F526C04B
:10ADC000CA3031F58091B415882301F1973089F0AC
:10ADD0003CF49530D9F4109214021092EA1216C085
:10ADE0009A3059F09F3091F480917C080E9493A88A
:10ADF0000DC081E08093C71009C00E9421A20E946B
:10AE00008AA08EEF0E9499D70E9407D810927D08E1
:10AE1000011731F0ED2FF0E0E451FE4EC283D12F47
:10AE2000D093EC11FF91EF91DF91CF91BF91AF9152
:10AE30009F918F917F916F915F914F913F912F9152
:10AE40001F910F910F900BBE0F900FBE0F901F9090
:10AE500018958EBD0DB407FEFDCF08958FEF8EBD02
:10AE60000DB407FEFDCF8EB50895909164009B7FD1
:10AE700090936400982F906A96959CBD80FD03C0C6
:10AE800091E0863009F490E09DBD0895CF92DF9265
:10AE9000EF92FF920F931F93CF93DF936C017A0190
:10AEA0008B01C0E0D0E0CE15DF0581F0D8016D91B7
:10AEB0008D01D601ED91FC910190F081E02DC6014C
:10AEC0001995892B11F02196EECF7E01C701DF91F4
:10AED000CF911F910F91FF90EF90DF90CF90089549
:10AEE000089580E090E00895FC01538D448D252F56
:10AEF00030E0842F90E0821B930B541710F0CF9614
:10AF0000089501970895FC01918D828D981761F045
:10AF1000828DDF01A80FB11D5D968C91928D9F5F90
:10AF20009F73928F90E008958FEF9FEF0895FC013B
:10AF3000918D828D981731F0828DE80FF11D858DEE
:10AF400090E008958FEF9FEF0895FC01918D228D81
:10AF5000892F90E0805C9F4F821B91098F73992706
:10AF600008958CEB93E10E94A55721E0892B09F409
:10AF700020E0822F0895FC01848DDF01A80FB11D10
:10AF8000A35ABF4F2C91848D90E001968F7399271F
:10AF9000848FA689B7892C93A089B1898C918370FD
:10AFA00080648C93938D848D981306C00288F389F6
:10AFB000E02D80818F7D80830895EF92FF920F9323
:10AFC0001F93CF93DF93EC0181E0888F9B8D8C8D55
:10AFD000981305C0E889F989808185FD26C0F62E81
:10AFE0000B8D10E00F5F1F4F0F731127E02E8C8D1C
:10AFF000E8120CC00FB607FCFACFE889F989808106
:10B0000085FFF5CFCE010E94BB57F1CF8B8DFE019E
:10B01000E80FF11DE35AFF4FF0829FB7F8940B8FB2
:10B02000EA89FB89808180620AC09FB7F894EE8923
:10B03000FF896083E889F9898081837080648083D7
:10B040009FBF81E090E0DF91CF911F910F91FF9022
:10B05000EF900895CF93DF93EC01888D8823C9F09A
:10B06000EA89FB89808185FD05C0A889B9898C9111
:10B0700086FD0FC00FB607FCF5CF808185FFF2CFAC
:10B08000A889B9898C9185FFEDCFCE010E94BB576D
:10B09000E7CFDF91CF91089580E090E0892B41F0D8
:10B0A00080E090E0892B21F00E940000811121C0F6
:10B0B00080E090E0892B41F080E090E0892B21F046
:10B0C0000E940000811118C080E090E0892B21F0DF
:10B0D0000E94B157811113C080E090E0892BA1F04C
:10B0E00080E090E0892B81F00E94000081110AC06D
:10B0F00008950E940000DCCF0E940000E5CF0E946E
:10B100000000EACF0C9400000895FC0120E03EE22C
:10B11000DB014C91403241F0283011F430833196FC
:10B12000DB014C91408331962F5F6F5F7F4F2B3057
:10B1300079F7108208950F942F1F0F931F93CF93C9
:10B14000DF938B01EA01DB016D917C910E94C96064
:10B15000D801ED91FC91119790818881992349F054
:10B16000893638F43196ED93FC9388818F5F88831C
:10B17000EFCF893658F48FE28083F8018081918186
:10B1800001969183808388818F5F8883DF91CF913F
:10B190001F910F9108951F920F920FB60F921124D5
:10B1A0000BB60F922F933F934F935F936F937F93C1
:10B1B0008F939F93AF93BF93EF93FF938CEB93E1A8
:10B1C0000E94BB57FF91EF91BF91AF919F918F91DB
:10B1D0007F916F915F914F913F912F910F900BBE97
:10B1E0000F900FBE0F901F9018951F920F920FB6E1
:10B1F0000F9211240BB60F922F938F939F93EF937F
:10B20000FF93E091CC13F091CD138081E091D213A4
:10B21000F091D31382FD12C090818091D5138F5F7E
:10B220008F732091D613821751F0E091D513F0E07F
:10B23000E454FC4E958F8093D51301C08081FF911B
:10B24000EF919F918F912F910F900BBE0F900FBE9A
:10B250000F901F9018958BE1E2EBF4E1A7E9B4E1C0
:10B2600001900D928A95E1F708958091CE1682FFA4
:10B270001FC084EA92E10F9413016091CA16709185
:10B28000CB168091CC169091CD164AE00E94364E96
:10B290008FE20E942F4E6091C6167091C716809162
:10B2A000C8169091C9164AE00E94364E0C94344F4D
:10B2B00086EB92E10D9413011092CB0A8091CE1689
:10B2C0008F7D8B7F8093CE160E943EB7882321F01E
:10B2D00089E594E10C942F6308958091CE1683FF45
:10B2E00003C084608093CE160895CF92DF92EF92D0
:10B2F000FF920F931F93CF93DF93CDB7DEB7EDB6D9
:10B30000FEB6DC010D900020E9F79D01281B390BEA
:10B310002C5F3F4F4DB75EB7421B530B0FB6F894EF
:10B320005EBF0FBE4DBF0DB71EB70F5F1F4F9F9380
:10B330008F9380EA91E19F938F931F930F930F94C4
:10B34000CB14680154E0C50ED11C0F900F900F90E4
:10B350000F900F900F90F6018081882349F0082EFE
:10B36000000C990B0F94341FF60181936F01F3CFFA
:10B37000C8010E94C3C88CE991E10E94F5C80FB6CC
:10B38000F894FEBE0FBEEDBEDF91CF911F910F91DD
:10B39000FF90EF90DF90CF9008958F929F92AF92A1
:10B3A000BF92CF92DF92EF92FF92CF938091CE1611
:10B3B000877F8093CE168091B514882321F082EB8D
:10B3C00094E10E942F63109296141092931485E3D7
:10B3D000809392140E9481EE6B017C0120EDC20EDD
:10B3E00027E0D21EE11CF11CA89561E08091921427
:10B3F0000E94F4EC61E0809192140E9423ED209A67
:10B40000289A219A2398229A81E00E94355785E054
:10B41000809394140E943557CAE08FEF0E942957F9
:10B42000C150D9F7A89520E030E0A90160E082E999
:10B4300094E10E940F6280939514813061F00E9424
:10B4400081EEDC01CB018C199D09AE09BF09B7FD66
:10B45000EACF81E062C0A8952AEA31E040E050E0FE
:10B4600068E082E994E10E940F62853011F481E086
:10B470000AC0C4E00E942E5780939514C150D1F7A2
:10B480008A3A61F482E080939614A895809196148C
:10B49000823081F0812C912C540111C00E9481EEE8
:10B4A000DC01CB018C199D09AE09BF09B7FDD4CFD2
:10B4B00082E033C0812C912CA12C80E4B82E20E0B6
:10B4C00030E0A90167E382E994E10E940F62A501DF
:10B4D000940169E282E994E10E940F6280939514DD
:10B4E000882361F00E9481EEDC01CB018C199D095B
:10B4F000AE09BF09B7FDE3CF8AE00FC08091961473
:10B50000823021F520E030E0A9016AE382E994E18C
:10B510000E940F62882361F088E08093931482E98F
:10B5200094E10E9407620F94FC018EE891E122C031
:10B530000E942E57807C803C19F483E080939614FF
:10B540000E942E570E942E570E942E5782E994E1A6
:10B550000E9407621092941481E00F940C048111F0
:10B560000CC080E00F940C04811107C00F94F80107
:10B570008AE791E10F9413011AC064E774E182EB4A
:10B5800094E10E945A60811105C00F94F80189E688
:10B5900091E1F0CF8091CE1688608093CE160F9403
:10B5A000FC018DE591E10F9413010E948D4DCF9127
:10B5B000FF90EF90DF90CF90BF90AF909F908F90D3
:10B5C0000C942B592F923F925F926F927F928F92A1
:10B5D0009F92AF92BF92CF92DF92EF92FF920F9322
:10B5E0001F93CF93DF93CDB7DEB7C356D1090FB604
:10B5F000F894DEBF0FBECDBF8C016B014A012DB6A2
:10B600003EB6512C7E0187E5E80EF11CF6018381E0
:10B61000823008F41FC180859185A285B3858F7122
:10B620009927AA27BB27892B8A2B8B2B09F012C1BC
:10B6300010926B194BE659E1BE016F5F7F4FC60157
:10B640000E94C46418160CF005C18C85982F98715F
:10B65000903129F42091390B2150223078F429813E
:10B66000222309F4F7C0253E89F22E3279F2209187
:10B670006B192E3259F28A7049F67CC06DB67EB6CF
:10B68000BE016F5F7F4FC7010E94855801151105EC
:10B6900021F0F8018081811163C021E081E090E018
:10B6A000F70101900020E9F73197EE19FF09E80F43
:10B6B000F91F32968DB79EB78E1B9F0B0FB6F8946D
:10B6C0009EBF0FBE8DBFEDB7FEB731965F01211152
:10B6D00002C0B80102C063E876E0C5010F947B1F89
:10B6E000B701C5010F94651F63E876E0C5010F94AB
:10B6F000651F19A21CA221E0A701B601CE01819607
:10B700000E941B6781110DC08091390B811109C006
:10B710000F94FC0189E491E10F941301C7010E9489
:10B720003A4F8BE1FE01B196DE01DC9601900D925D
:10B730008A95E1F740E050E0BE01645C7F4FC501AF
:10B740000E94E25ACE01CC960E943863CE018196C7
:10B750000E9438630FB6F8947EBE0FBE6DBE56CF02
:10B76000F80101900020E9F73197CF01801B910B80
:10B7700020E096CF21E0903109F020E08091CE16B4
:10B7800020FB84F98093CE16903141F0898587346F
:10B7900009F03CCF8A858E3709F438CF8091390B78
:10B7A000813021F068F08230C1F130CF80913C0BC4
:10B7B00090913D0B019690933D0B80933C0B26CFCF
:10B7C000BE016F5F7F4F8DEA99E10E948558011598
:10B7D000110529F48DEAA82E89E1B82E09C0580177
:10B7E000F50181915F018823A9F30E942F4EF8CFC4
:10B7F000F50181915F01882319F00E942F4EF8CF47
:10B8000080E20E942F4E6D8D7E8D8F8D98A14AE033
:10B810000E94364E0E94344FF9CEBE016F5F7F4FBB
:10B820008DEA99E10E9485588114910441F06DEAF6
:10B8300079E1C4010F94521F892B51F40BC0852D5F
:10B8400090E020913A0B30913B0B8217930711F057
:10B850005394DCCE0FB6F8943EBE0FBE2DBECD592C
:10B86000DF4F0FB6F894DEBF0FBECDBFDF91CF9193
:10B870001F910F91FF90EF90DF90CF90BF90AF900E
:10B880009F908F907F906F905F903F902F90089542
:10B89000CF93DF93CDB7DEB76B970FB6F894DEBFCB
:10B8A0000FBECDBF81E08093390B10923D0B1092FB
:10B8B0003C0B87E994E10E9402628BE1E7E9F4E145
:10B8C000DE01119601900D928A95E1F740E050E07B
:10B8D000BE016F5F7F4F80E090E00E94E25ACE0190
:10B8E00001960E94386380913C0B90913D0B6B96C2
:10B8F0000FB6F894DEBF0FBECDBFDF91CF91089594
:10B900000F931F93CF93DF93CDB7DEB76B970FB62F
:10B91000F894DEBF0FBECDBF8B0122E02093390B20
:10B9200090933B0B80933A0B87E994E10E9402626B
:10B930008BE1E7E9F4E1DE01119601900D928A9521
:10B94000E1F7A801BE016F5F7F4F80E090E00E94A9
:10B95000E25ACE0101960E9438636B960FB6F894B6
:10B96000DEBF0FBECDBFDF91CF911F910F91089524
:10B97000DF92EF92FF920F931F93CF93DF9300D04C
:10B980001F92CDB7DEB72091CE1623FF3DC1F42E16
:10B99000E62E8C010E943EB7882309F481C0FF2067
:10B9A00009F48CC08091C516882351F00F94F801DA
:10B9B0008FE592E10F94130180E090E00E9433FA4A
:10B9C00081ED9AE09A8389838FE28093D00A81E0A7
:10B9D0008B83F12C9BE1D92E8091C416F81678F454
:10B9E000DF9CC0011124AE014D5F5F4FBE016F5F50
:10B9F0007F4F8A549A4E0E949D58F394EDCF8B81CD
:10BA00008B3578F4AE014D5F5F4FBE016F5F7F4FA6
:10BA100089E594E10E949D5889819A8101979A83D2
:10BA20008983E981FA811082E091C51684E0E89F5C
:10BA3000F0011124E453F54F8091CA169091CB1672
:10BA4000A091CC16B091CD1680839183A283B3834D
:10BA50000F94FC01B80186E492E10F94E501609136
:10BA6000C51689E6689FB00111246053754F8BE3BA
:10BA700092E10F94E5014091CA165091CB16609166
:10BA8000CC167091CD1685E392E10F94A9018AE05E
:10BA90000E942F4E8091C5168F5F8093C51626C0D9
:10BAA000FF2039F00F94FC0185E292E10F9413011D
:10BAB0001DC01092C51682E0F82E02C0FF24F39438
:10BAC0000F94FC0180E292E10F94130181E0F816DB
:10BAD00009F497C08CE092E10F941301B80188E15A
:10BAE00092E10F94E5018AE00E942F4E0E945C597A
:10BAF000B801CE0103960E949AFB8C01009709F4CD
:10BB000083C06B817C81EE2009F450C021E0AC0140
:10BB100089E594E10E941B67882309F43FC0809166
:10BB20006A1490916B14A0916C14B0916D14809371
:10BB3000C6169093C716A093C816B093C916109254
:10BB4000CA161092CB161092CC161092CD16B801D0
:10BB50008EEF91E10F94E5014091C6165091C71602
:10BB60006091C8167091C91686EF91E10F94A901F2
:10BB70008AE00E942F4E87EE91E10F941301B801E5
:10BB800080E090E00E94805C80916B19811102C07E
:10BB9000C80102C08BE699E160E030C0B80183EDD6
:10BBA00091E10F94E50180ED91E10FC026E5AC0134
:10BBB00089E594E10E941B6781110AC0B8018CEBF2
:10BBC00091E10F94E50189EB91E10F9413011CC001
:10BBD0008091CE1681608093CE16B80180E090E00F
:10BBE0000E94805C1092B415B80187EA91E10F942D
:10BBF000E5018AE00E942F4E60E0C8010E9408E142
:10BC000003C082E192E168CF0F900F900F900F90E8
:10BC1000DF91CF911F910F91FF90EF90DF900895EA
:10BC2000CF92DF92EF92FF92CF936B017C01C42FF2
:10BC30008091601990916119A0916219B091631976
:10BC40008C159D05AE05BF05D1F00E94BC62811127
:10BC500002C080E018C020E637E1B701A60180915C
:10BC6000691990916A190E943E63882391F3C092EA
:10BC70006019D0926119E0926219F092631981E023
:10BC8000C11180936819CF91FF90EF90DF90CF9012
:10BC900008954F925F926F927F928F929F92AF9290
:10BCA000BF92CF92DF92EF92FF920F931F93CF93A9
:10BCB000DF93EC01423051056105710510F480E01D
:10BCC00069C089859A85AB85BC850196A11DB11D8A
:10BCD00084179507A607B70790F38F89803149F439
:10BCE000852E962EA72EBB248B899C89AD89BE8973
:10BCF0000FC0803221F78B889C88AD88BE88DB011D
:10BD0000CA01E7E0B695A79597958795EA95D1F78B
:10BD1000880E991EAA1EBB1E280139016A017B01EB
:10BD200041E0C501B4010E94105E882341F29F8961
:10BD3000903161F4DD24EE24FF249601220F331F9D
:10BD4000F901E05AF84E5182408211C0E894C7F8D8
:10BD5000DD24EE24FF249601220F331F220F331F10
:10BD6000F901E05AF84E40825182628273829A89C8
:10BD7000923080F04D815E816F817885840E951EB2
:10BD8000A61EB71E8092641990926519A09266193A
:10BD9000B0926719DF91CF911F910F91FF90EF90B3
:10BDA000DF90CF90BF90AF909F908F907F906F90DB
:10BDB0005F904F900895CF92DF92EF92FF920F9392
:10BDC0001F93CF93DF93FC0181859285A385B48572
:10BDD0000196A11DB11D84179507A607B70710F49A
:10BDE00080E061C08789803149F4BB27A72F962F57
:10BDF000852FC388D488E588F6880FC0803281F704
:10BE000083899489A589B6896A017B01C7E0F69484
:10BE1000E794D794C794CA95D1F78C0D9D1DAE1D9C
:10BE2000BF1DE9016A017B018F01409160195091AA
:10BE30006119609162197091631984179507A607BB
:10BE4000B70739F040E0BC01CD010E94105E8823A5
:10BE500039F2F8018789803179F4B701A6015527B5
:10BE600066277727440F551FFA01E05AF84E808164
:10BE70009181A0E0B0E012C0B701A6014F7755272D
:10BE800066277727440F551F440F551FFA01E05AC4
:10BE9000F84E80819181A281B381BF70888399839C
:10BEA000AA83BB8381E0DF91CF911F910F91FF9017
:10BEB000EF90DF90CF9008954F925F926F927F92B4
:10BEC000AF92BF92CF92DF92EF92FF920F931F93A8
:10BED000CF93DF9300D01F92CDB7DEB78C0149839B
:10BEE0005A836B837C835901C12CD12C7601412C60
:10BEF00082E0582E612C712C49815A816B817C81A2
:10BF00009E012F5F3F4FC8010E94DB5E882341F1F5
:10BF1000D301C201F801058404C0880F991FAA1F2C
:10BF2000BB1F0A94D2F7C80ED91EEA1EFB1E498118
:10BF30005A816B817C818789803139F481E0483F67
:10BF40005F4F6105710538F4D7CF81E0483F5F4FFF
:10BF50006F4F7F4088F2F501C082D182E282F38286
:10BF60000F900F900F900F90DF91CF911F910F9135
:10BF7000FF90EF90DF90CF90BF90AF907F906F9049
:10BF80005F904F9008958F929F92AF92BF92CF9201
:10BF9000DF92EF92FF920F931F93CF93DF93EC0109
:10BFA0008B81811102C080E078C009891A892B89B0
:10BFB0003C890417150726073707A8F36A017B0198
:10BFC000823029F4C886D986EA86FB860DC0C11462
:10BFD000D104E104F10451F4188619861A861B86EF
:10BFE0001C821D821E821F8281E057C08884998432
:10BFF000AA84BB84E98DFA8D258530E0275F3F4F09
:10C00000B501A4014150510961097109022E04C012
:10C0100076956795579547950A94D2F7D701C6014B
:10C020000197A109B10904C0B695A7959795879581
:10C030002A95D2F784179507A607B70720F0892815
:10C040008A288B2871F44D895E896F89788D4C839D
:10C050005D836E837F834C015D018E010C5F1F4FFA
:10C0600016C0841B950BA60BB70BF5CF4C815D81D9
:10C070006E817F819801898D9A8D0E94DB5E91E0AF
:10C08000891A9108A108B108882309F48CCF81147A
:10C090009104A104B10451F795CFDF91CF911F9185
:10C0A0000F91FF90EF90DF90CF90BF90AF909F9057
:10C0B0008F9008950F931F93CF93DF93FC012381FB
:10C0C000222311F080E044C08B01EC01FB01878941
:10C0D000803139F18032B1F783E08B83F801428DF2
:10C0E000538D648D758D4D8B5E8B6F8B788F9E011C
:10C0F0002F5E3F4FC8010E945C5F882319F31A8F9F
:10C10000098F81E08983188619861A861B861C820E
:10C110001D821E821F82188A1C861D861E861F860F
:10C1200017C082E08B831D8A1E8A1F8A188EFB012E
:10C13000808D918DA0E0B0E025E0880F991FAA1FA7
:10C14000BB1F2A95D1F7898B9A8BAB8BBC8BD7CF32
:10C15000DF91CF911F910F910895CF93DF93EC0161
:10C1600041E0611101C040E06C857D858E859F8531
:10C170000E94105E882341F0888920E2829FC001DE
:10C180001124805A984E02C080E090E0DF91CF9158
:10C190000895CF93DF93EB01FC012381211102C0AD
:10C1A00080E028C02250223020F48FE28883198258
:10C1B00020C060E00E94AD60009791F3FC0190E028
:10C1C00080E02EE23081303269F0883029F4DE01DF
:10C1D000A90FB11D2C939F5FDE01A90FB11D308106
:10C1E0003C939F5F8F5F31968B3061F7C90FD11DF4
:10C1F000188281E0DF91CF9108953F924F925F9234
:10C200006F927F928F929F92AF92BF92CF92DF9266
:10C21000EF92FF920F931F93CF93DF93CDB7DEB7CB
:10C220002C970FB6F894DEBF0FBECDBF5C01DC01CA
:10C2300059968D909C905A97F40181859285A3859B
:10C24000B4859C01AD012F5F3F4F4F4F5F4F298752
:10C250003A874B875C87D5011496CD90DD90ED90A1
:10C26000FC901797C114D104E104F10439F0BFEF39
:10C27000CB1ADB0AEB0AFB0A312C07C0F401C080A1
:10C28000D180E280F38033243394260137011D826C
:10C290001E821F821886F40181859285A385B4854C
:10C2A0002D813E814F815885281739074A075B0742
:10C2B00008F064C089859A85AB85BC858C159D0581
:10C2C000AE05BF0550F482E0C82ED12CE12CF12C34
:10C2D00092E0492E512C612C712C9E012F5F3F4F13
:10C2E000B701A601C4010E94DB5E882309F446C0A1
:10C2F00089819A81AB81BC81892B8A2B8B2B41F060
:10C30000260137019FEF491A590A690A790A05C0BF
:10C31000C414D504E604F70491F02D813E814F81C9
:10C3200058852F5F3F4F4F4F5F4F2D833E834F8385
:10C3300058873FEFC31AD30AE30AF30AACCF0FEFD3
:10C340001FEF2FEF3FE0B301A201C4010E94495E3D
:10C35000F82E882399F0D50114964D915D916D9139
:10C360007C911797411551056105710549F09301BD
:10C370008201C4010E94495E811102C0F12C29C0D2
:10C38000D50114964D925D926D927C921797332051
:10C3900051F0D301C2010196A11DB11DF4018083AA
:10C3A0009183A283B383F50185899689A789B08D8E
:10C3B000892B8A2B8B2B69F4D50155964D925D9272
:10C3C0006D927C92589711968C9111978068119676
:10C3D0008C938F2D2C960FB6F894DEBF0FBECDBF79
:10C3E000DF91CF911F910F91FF90EF90DF90CF9051
:10C3F000BF90AF909F908F907F906F905F904F9085
:10C400003F90089540E050E0BA010C94C35F61E0B2
:10C41000FC0180810E94F4EC8FEF0C942957EF927D
:10C42000FF921F93CF93DF9300D01F92CDB7DEB75B
:10C430007C01162F29833A834B835C83FC01828124
:10C440000E94355760E0F70180810E94F4EC0E9461
:10C45000E4FA812F80640E9429578C810E94295719
:10C460008B810E9429578A810E94295789810E94C5
:10C470002957112311F087E801C085E90E94295747
:10C480001C3011F40E942E5710E00E942E57F70125
:10C49000838387FF04C01F3F11F01F5FF6CF0F900B
:10C4A0000F900F900F90DF91CF911F91FF90EF9021
:10C4B00008950F931F93CF93DF93EC0189018C8133
:10C4C000833039F089E0440F551F661F771F8A9526
:10C4D000D1F79A01AB0168E1CE010E940F62811190
:10C4E00028C08EEF8EBDF801C8019E5F0DB407FE17
:10C4F000FDCF20812EBD0DB407FEFDCF21812EBDC5
:10C5000032968E179F0791F70DB407FEFDCF8FEF80
:10C510000E9429578FEF0E9429570E942E578B8324
:10C520008F71853041F083E18983CE010E940762DB
:10C5300019C086E016C00E94E4FA882379F020E052
:10C5400030E0A9016DE0CE010E940F62811108C0A8
:10C550000E942E57811104C011E005C087E101C07F
:10C5600086E1898310E0CE010E940762812FDF916E
:10C57000CF911F910F910895CF93809168198823CF
:10C58000B9F14091601950916119609162197091EF
:10C59000631920E637E18091691990916A190E9428
:10C5A0005962C82F811102C0C0E023C040916419B4
:10C5B000509165196091661970916719411551057F
:10C5C0006105710591F020E637E18091691990913C
:10C5D0006A190E945962882339F3109264191092E3
:10C5E000651910926619109267191092681901C0A6
:10C5F000C1E08C2FCF910895CF93DF93EC018B8115
:10C60000882339F1898187FF20C061E0CE010E9433
:10C61000AD60FC01892BE9F08081853ED1F08B81F2
:10C62000823040F489899A89AB89BC89848F958F3F
:10C63000A68FB78F8D899E89AF89B88D938F828F92
:10C64000B58BA48B89818F778983DF91CF910C94EF
:10C65000BC6281E0888380E0DF91CF910895CF9321
:10C66000DF93EC010E94FC621B82DF91CF91089561
:10C67000FC01238121110C942F630895CF92DF9246
:10C68000EF92FF920F931F93CF93DF93EC018901F9
:10C690008C81833039F089E0440F551F661F771F66
:10C6A0008A95D1F79A01AB0161E1CE010E940F6238
:10C6B000882339F084E08983CE010E94076280E0FC
:10C6C0003EC00E9481EE6B017C012CE2C20E21E093
:10C6D000D21EE11CF11C0E942E578B838F3F61F408
:10C6E0000E9481EEDC01CB018C199D09AE09BF09C6
:10C6F000B7FDF1CF81E11DC08E3FD1F48FEF8EBD2C
:10C70000F801D801A150BE4F0DB407FEFDCF9EB574
:10C7100091938EBDEA17FB07B9F70DB407FEFDCF65
:10C720008EB58C930E942E570E942E5711E003C0A5
:10C730008FE0898310E0CE010E940762812FDF9194
:10C74000CF911F910F91FF90EF90DF90CF900895C0
:10C750002F923F924F925F926F927F928F929F9211
:10C76000AF92BF92CF92DF92EF92FF920F931F93FF
:10C77000CF93DF9300D01F92CDB7DEB79C838B831E
:10C780004B015A01DC0113968C91811103C08FEF8C
:10C790009FEFE3C0EB81FC81818180FFF8CFEB81CB
:10C7A000FC8181899289A389B489408551856285FC
:10C7B0007385841B950BA60BB70BA50160E070E099
:10C7C00084179507A607B70708F45C0175018B81EC
:10C7D0009C8104969A838983612C42E0742EE11433
:10C7E000F10409F48BC0AB81BC8118964D915D9129
:10C7F0006D917C911B976A01B1E0DB22EB81FC819A
:10C800002381818D928D1A012B0139E05694479432
:10C81000379427943A95D1F7223061F4FC01828D48
:10C82000938DA48DB58DBC01CD01620D731D841D4A
:10C83000951D4AC0DC0114961C9111501221C1149F
:10C84000D10401F511111EC0452B462B472B59F47D
:10C85000EB81FC8185899689A789B08D8483958336
:10C86000A683B7830FC0AB81BC8114964D915D91B7
:10C870006D917C91179729813A810E94DB5E882314
:10C8800009F485CFEB81FC81218D328D84819581E6
:10C89000A681B7810297A109B109F901058404C0F5
:10C8A000880F991FAA1FBB1F0A94D2F74685578588
:10C8B00060897189840F951FA61FB71FBC01CD0128
:10C8C000610F711D811D911D93012C193D09870177
:10C8D0002E153F0508F489010115F2E01F0779F5CF
:10C8E000209160193091611940916219509163193A
:10C8F000621773078407950719F421C0C5012DC07D
:10C900009401AB01BC018091691990916A190E9450
:10C910003E63882309F43BCF800E911EEB81FC819E
:10C9200080859185A285B385800F911FA11DB11DC2
:10C9300080879187A287B387E01AF10A50CF40E041
:10C940000E94105E882309F422CFB601605A784E07
:10C95000A801C4010F94491FDFCF0F900F900F90D3
:10C960000F90DF91CF911F910F91FF90EF90DF908B
:10C97000CF90BF90AF909F908F907F906F905F907F
:10C980004F903F902F900895DF92EF92FF920F9378
:10C990001F93CF93DF938C01EB017A018DE0D82EAA
:10C9A00040E250E0BE01C8010E94A86380329105B8
:10C9B00039F021E0892B09F420E0822F819544C0D1
:10C9C00028812223C9F1253E11F02E3231F4E114E1
:10C9D000F10431F3F7011082E3CFE114F10441F1E6
:10C9E0003B853F733F3021F54A8D5B8D452B01F52B
:10C9F0002F713FEF320F3530D8F430E0215031093C
:10CA0000D29EC001D39E900D1124D701A80FB91F4B
:10CA1000FE0120E0AD01253088F431813D932F5F88
:10CA200032962D30C1F7288126FF02C0FA01158603
:10CA30002B8523FDB5CF08C080E006C02B3010F455
:10CA40003481ECCF3681EACFDF91CF911F910F91E6
:10CA5000FF90EF90DF9008954F925F926F927F92D8
:10CA60009F92AF92BF92CF92DF92EF92FF920F937D
:10CA70001F93CF93DF931F92CDB7DEB78C017B015D
:10CA80005A01C22EDB0159968D919C915A97F8015B
:10CA9000928F818FCB010E940262912CF7018085D9
:10CAA0009185A285B38541895289638974898417E8
:10CAB0009507A607B70708F060C025E0B695A795CB
:10CAC000979587952A95D1F7F82FFF70DF2ED7011C
:10CAD00013968C91823008F460C041E050E0BE01B2
:10CAE0006F5F7F4FC7010E94A863019719F4898186
:10CAF00090E002C08FEF9FEF019609F44EC0F7015E
:10CB000080859185A285B3854F96A11DB11D808733
:10CB10009187A287B387F0E2DF9EB0011124605AAB
:10CB2000784E61157105C9F1DB018C91882319F0EC
:10CB3000853EC1F46CC191100EC080916019909136
:10CB40006119A0916219B0916319F80184879587E2
:10CB5000A687B787D08ADB018C91882361F099245E
:10CB600093949CCF4BE050E0C5010F943C1F892B60
:10CB700009F094CF14C0992493948C2D827482343C
:10CB800061F4992009F48BC0F801D08861E0C801F4
:10CB90000E94AD60009709F00DC180E03BC1C7FC69
:10CBA000FCCFF0E2DF9EA00111249A01205A384EFA
:10CBB000D9011B968C91817121F08C2D827109F025
:10CBC0006AC08091601990916119A0916219B09129
:10CBD0006319F80184879587A687B787D08ACA0129
:10CBE000805A984E7C01DC0154964D915C9155978A
:10CBF00060E070E0DA0199278827858B968BA78BF8
:10CC0000B08FF701428D538D60E070E0482B592BB7
:10CC10006A2B7B2BD80155964D935D936D937C9336
:10CC20005897F9018385887161F4F701848D958D9A
:10CC3000A68DB78DF801818B928BA38BB48B81E08D
:10CC400010C0803141F598012F5E3F4FD8015996B1
:10CC50008D919C915A970E945C5F8823E1F084E05B
:10CC6000F80183838C2D8F70D80111968C931197C6
:10CC7000F801148215821682178218961D921D9251
:10CC80001D921C921B97C4FEB5C0C8010E9408FBF0
:10CC90008111B0C082CFD80113961C927ECFD701EC
:10CCA00013968C911397823009F477CF51968D911A
:10CCB0009D910D90BC91A02D803E9F4FAF41B1053D
:10CCC00008F06BCFC7010E94FD60882309F465CF8F
:10CCD0000E94BC62882309F460CFD70159962D9138
:10CCE0003C915A9714968D919D910D90BC91A02DD9
:10CCF0000297A109B109F901058404C0880F991FA1
:10CD0000AA1FBB1F0A94D2F7468457846088718893
:10CD1000480E591E6A1E7B1E81E08093681940925E
:10CD2000601950926119609262197092631980E0E3
:10CD300092E0E0E6F7E1DF019C011D9221503040D6
:10CD4000E1F7DD24D394D7015996ED91FC915A97E0
:10CD50008481D81698F420E637E1B301A2014D0D85
:10CD6000511D611D711D8091691990916A190E9470
:10CD70005962882309F411CFD394E5CF80E092E083
:10CD8000A0E0B0E0058404C0880F991FAA1FBB1F54
:10CD90000A94D2F7F7014189528963897489840F13
:10CDA000951FA61FB71F818B928BA38BB48B80E638
:10CDB00097E1D12C20E2DC011D922A95E9F72BE0C6
:10CDC000F501DC0101900D922A95E1F721E238E2AC
:10CDD000FC01318B208B40E058E057874687338B2E
:10CDE000228B318F208F578B468B0E94BC62811122
:10CDF000D8CED3CEC5FE09C0F801418952896389D6
:10CE00007489C8010E94C35F05C081E003C091100E
:10CE1000A6CE93CE0F90DF91CF911F910F91FF90EF
:10CE2000EF90DF90CF90BF90AF909F907F906F90EA
:10CE30005F904F9008952F923F924F925F926F9222
:10CE40007F928F929F92AF92BF92CF92DF92EF929A
:10CE5000FF920F931F93CF93DF93CDB7DEB7C254EA
:10CE6000D1090FB6F894DEBF0FBECDBF4C015B01F8
:10CE70006A01322E19821C821C8E1F8E611571056B
:10CE800011F410E0A6C0FC0183818111FACFFA01F0
:10CE900080818F3209F09BC0F501838182508230FE
:10CEA00010F485010CC0F501618D728DCE014C9698
:10CEB0000E945A60882329F38E01045E1F4FC60129
:10CEC0006C010196F60120812F32D1F3CE0101963B
:10CED0007C013C012E019CE1490E511C2396EFAED2
:10CEE00023972F2C9BE09150E7E3F0E0EC0FFD1F20
:10CEF000E90FF11D80E280839111F5CF960147E0A3
:10CF0000D9018D91882369F18F3259F18E3239F42C
:10CF10004A3009F4B6CF98E04AE09D01F1CFE9ED3F
:10CF2000F2E12491222321F031968213FACFA9CF86
:10CF3000491708F4A6CF813208F4A3CF8F3709F43C
:10CF4000A0CF21E0290FE7E3F0E0EC0FFD1FE90F90
:10CF5000F11D9FE9980F9A3108F480528083922F37
:10CF6000DCCF8FA9803209F48CCF6901F90180816F
:10CF70002F5F3F4F8F32C9F38823F9F021E0AE01D4
:10CF8000495C5F4FB801C7010E942C65882309F4F2
:10CF900078CF0A151B0519F0C8010E942F636E1483
:10CFA0007F0441F023969FAD2397822D8701E92EC0
:10CFB000F82E98CF942D852DF9CF232DAE01495C05
:10CFC0005F4FB801C4010E942C65182F02C08B016D
:10CFD0007DCFCE014C960E943863CE0101960E940F
:10CFE0003863812FCE5BDF4F0FB6F894DEBF0FBEE4
:10CFF000CDBFDF91CF911F910F91FF90EF90DF9008
:10D00000CF90BF90AF909F908F907F906F905F90E8
:10D010004F903F902F900895CF93C82F0F94FC010D
:10D0200084E50E942F4E6C2F70E080E090E00E941B
:10D03000A34E80E20E942F4E87EC92E1CF910D9497
:10D0400013012F923F924F925F926F927F928F9235
:10D050009F92AF92BF92CF92DF92EF92FF920F9387
:10D060001F93CF93DF93CDB7DEB7C154D1090FB66D
:10D07000F894DEBF0FBECDBF2DB73EB73FA72EA79A
:10D080000E94CF8281114FC461E086E50E94F69034
:10D090008D8B853018F085E894E179C03D89332384
:10D0A00021F085E694E10F9413016AE080E50E9487
:10D0B000F690182F8CEF810F8F3218F081E494E1F5
:10D0C00066C060E085E40E9422A8811103C082E06E
:10D0D0008FA302C091E09FA3609143177091441702
:10D0E00080914517909146176D837E838F83988733
:10D0F000C0904717D0904817E0904917F0904A1712
:10D10000C986DA86EB86FC8620912E1330912F1388
:10D1100040913013509131130F941D1CAB01BC0191
:10D1200088E50E94F2AF6D877E878F87988B29856F
:10D130003A854B855C8560913213709133138091F1
:10D140003413909135130F941D1CAB01BC0189E57C
:10D150000E94F2AF698B7A8B8B8B9C8BBE016F5ECA
:10D160007F4FCE010D960E94B08F811103C089E2DE
:10D1700094E10DC08CE40E94CCA7082F882381F095
:10D180000E946DA78E8B803128F086EF93E10F947B
:10D190001301C9C3AE89A13021F4B2E0BE8B01C036
:10D1A0001E8A60E083E50E9422A88CAB882321F0D0
:10D1B000011102C0E7E0EE8BFD89F33020F08CED29
:10D1C00093E10F94130120915B172BAF80E00E9435
:10D1D0008DAC0E945CD6812F90E09EAB8DABADB73D
:10D1E000BEB7E4E01E9FA019B10911240FB6F89450
:10D1F000BEBF0FBEADBF2DB73EB72F5F3F4F3DA7A0
:10D200002CA72D894FA1BE016F5E7F4FCE010D96D9
:10D210000E94ABE89B01AC010F940F1F8111ECC27F
:10D220000E9481EE611571058105910511F00F9441
:10D23000C41033EF3F8B8FE4888F93EC998F37ECDA
:10D24000232EA3EFAA8FBFE4BB8FE3ECEC8FF7E4B0
:10D25000FD8F1EA233243394412C512C32014AA25B
:10D260005BA26CA27DA22E89822F90E0DC01119737
:10D270002296BFAFAEAF2297FEA1EF2FF0E0FF8F57
:10D28000EE8F2DA93EA9E217F3070CF0CDC23E891F
:10D29000332309F46EC10F9476102AE030E040E0A9
:10D2A00050E00F94AB1B0F943A1520E030E040EAB9
:10D2B00050E40F947D1E18161CF001E010E002C02F
:10D2C0000FEF1FEF0F94761028E631E040E050E0BA
:10D2D0000F94AB1B0F943A154B015C010F94761021
:10D2E00021E230E040E050E00F94AB1B6B5F7F4FDA
:10D2F0008F4F9F4F0F943A1568A779A78AA79BA7CE
:10D300008D898430E1F448A559A56AA57BA58EECEA
:10D3100093E10F94C701B501A40186EC93E10F944A
:10D32000C70180EC93E10F9413010130110519F44A
:10D3300083E40E942F4E8CEB93E10F941301312C68
:10D34000C801110FAA0BBB0B8FAB98AFA9AFBAAF37
:10D35000832D90E02296AEADBFAD22978A179B0732
:10D360000CF007C1BCA9BB2379F06FA978AD89ADDA
:10D370009AAD0F943A159B01AC010F941D1C20E04F
:10D3800030E040E952E41AC00F94761024E130E016
:10D3900040E050E00F94AB1B675E7F4F8F4F9F4F75
:10D3A0000F943A156B017C016FA978AD89AD9AADE8
:10D3B0000F943A159B01AC01C701B6010F94991562
:10D3C0009B01AC01C501B4010F941D1C4B015C0114
:10D3D00020E030E044EB53E40F947D1E18164CF42B
:10D3E00020E030E044EB53E4C501B4010F941C1C71
:10D3F000EDCF20E030E0A901C501B4010F94331551
:10D4000087FF0BC020E030E044EB53E4C501B401DA
:10D410000F941D1C4B015C01ECCF2BED3FE049E468
:10D4200050E4C501B4010F94991520E030E044E3C5
:10D4300053E40F94171D6B017C010F94121D68AB10
:10D4400079AB8AAB9BAB20912E1330912F13409177
:10D450003013509131136D857E858F8598890F9497
:10D460001C1C6CAF7DAF8EAF9FAF28A939A94AA90C
:10D470005BA968A579A58AA59BA50F9499159B0121
:10D48000AC016CAD7DAD8EAD9FAD0F941D1C6D8359
:10D490007E838F839887C701B6010F94BD1E68AB4A
:10D4A00079AB8AAB9BAB209132133091331340910F
:10D4B00034135091351369897A898B899C890F942B
:10D4C0001C1C6B017C0128A939A94AA95BA968A584
:10D4D00079A58AA59BA50F9499159B01AC01C7015D
:10D4E000B6010F941D1C69877A878B879C874BE355
:10D4F00051E060E070E0CE0105960E947E8346E335
:10D5000051E060E070E0CE0109960E947E83ED89D3
:10D51000E430F9F44D815E816F81788580EB93E191
:10D520000F94C70149855A856B857C858DEA93E107
:10D530000F94C70140914B1750914C1760914D17B4
:10D5400070914E178AEA93E10F94C7018AE00E9416
:10D550002F4E19821A821B821C82AE014F5F5F4FD1
:10D56000BE01675F7F4FCE0105960E943CD7339482
:10D57000EFCE20E04FA1BE016F5E7F4FCE010D9632
:10D580000E94ABE8D62EE72EF82E192FEE8DFF8DD8
:10D59000EE0FFF1FEE0FFF1F2CA53DA5E20FF31F9F
:10D5A000862F9E2DAF2DB12F80839183A283B383CD
:10D5B000312C2D2D3E2D4F2D512F6D2D7E2D8F2D4C
:10D5C000912F0F940F1F811102C0332433942D2DFE
:10D5D0003E2D4F2D512F6D2D7E2D8F2D912F0F9480
:10D5E0000F1F811121C100E0412C512C3201ECA50B
:10D5F000FDA534E0039FE00DF11D11242081318150
:10D6000042815381C301B2010F941D1C2B013C01C7
:10D610000F5F8EA1801758F78E8C9F8C9FEF891A11
:10D62000990A092C000CAA08BB08C501B4010F9483
:10D630003A156E8F7F8F88A399A39B01AC01C3011C
:10D64000B2010F94171D6AA37BA38CA39DA32A8DFF
:10D650003B8D4C8D5D8D6D2D7E2D8F2D912F0F94DB
:10D66000331587FF04C0DA8EEB8EFC8E1D8F2F8959
:10D67000388D498D522D6D2D7E2D8F2D912F0F942C
:10D680007D1E181624F4DF8AE88EF98E212EC12C17
:10D69000412C512C3201ECA5FDA5A4E0CA9EE00D61
:10D6A000F11D11242AA13BA14CA15DA160817181D2
:10D6B000828193810F941C1C9B01AC010F949915DE
:10D6C0009B01AC01C301B2010F941D1C2B013C0155
:10D6D000C394BEA1BC15F8F62E8D3F8D48A159A16B
:10D6E0000F94171D0F94CB1E2B013C018D89825086
:10D6F0008E3708F07DC0C501B4010E94A34E6DA90C
:10D700007EA985EA93E10F94D80195E8A92E96E0C9
:10D71000B92EF50181915F01882319F00E942F4EE7
:10D72000F8CF43E06D2D7E2D8F2D912F0E94BF4E9F
:10D73000FD89F23009F459C00BE816E0D8018D914B
:10D740008D01882319F00E942F4EF8CF44E06AA182
:10D750007BA18CA19DA10E94BF4E03E916E0F801B8
:10D7600081918F01882319F00E942F4EF8CF46E057
:10D77000C301B2010E94BF4E0CE916E0D8018D91A1
:10D780008D01882319F00E942F4EF8CF43E06A8D57
:10D790007B8D8C8D9D8D0E94BF4E03EA16E0F801B3
:10D7A00081918F01882319F00E942F4EF8CF43E01A
:10D7B0006F89788D898D922D0E94BF4E0AEA16E0FE
:10D7C000D8018D918D01882319F00E942F4EF8CF3A
:10D7D0002A8D3B8D4C8D5D8D6F89788D898D922D35
:10D7E0000F941C1C43E00E94BF4E8AE00E942F4E03
:10D7F000BEA1BF5FBEA340CDE3EFEF8BFFE4F88F88
:10D8000023EC298F87EC282E33EF3A8F8FE48B8F10
:10D8100093EC9C8FA7E4AD8F312C412C512C32011D
:10D820004AA25BA26CA27DA280E00E94E19D33200F
:10D8300009F46AC08AE993E10F941301BD89BB23FF
:10D8400009F44DC003EB16E0F80181918F018823A4
:10D8500019F00E942F4EF8CF46E06AA17BA18CA15F
:10D860009DA10E94BF4E0AEB16E0D8018D918D015B
:10D87000882319F00E942F4EF8CF43E06A8D7B8DEC
:10D880008C8D9D8D0E94BF4E01EC16E0F8018191B8
:10D890008F01882319F00E942F4EF8CF43E06F8943
:10D8A000788D898D922D0E94BF4E08EC16E0D8012C
:10D8B0008D918D01882319F00E942F4EF8CF2A8D6B
:10D8C0003B8D4C8D5D8D6F89788D898D922D0F9458
:10D8D0001C1C43E00E94BF4E8AE00E942F4E01EDC7
:10D8E00016E0F80181918F01882319F00E942F4ED4
:10D8F000F8CF46E0C301B2010E94BF4E8AE00E9409
:10D900002F4E8AE00E942F4E0E9443D68BAD0E947C
:10D910008DAC0E9433D92EA53FA50FB6F8943EBF1B
:10D920000FBE2DBF07C08EA59FA50FB6F8949EBF52
:10D930000FBE8DBFAEA5BFA50FB6F894BEBF0FBE7C
:10D94000ADBFCF5BDF4F0FB6F894DEBF0FBECDBFCC
:10D95000DF91CF911F910F91FF90EF90DF90CF90CB
:10D96000BF90AF909F908F907F906F905F904F90FF
:10D970003F902F9008952F923F924F925F926F9217
:10D980007F928F929F92AF92BF92CF92DF92EF924F
:10D99000FF920F931F93CF93DF93CDB7DEB7E59739
:10D9A0000FB6F894DEBF0FBECDBF30905B1787E592
:10D9B0000E94CCA7882309F4F9C08091401390916C
:10D9C0004113892B29F40F94F80188E893E134C0BE
:10D9D0008AE50E9415A8882379F00E9495A72091D6
:10D9E0002A1330912B1340912C1350912D130F9427
:10D9F0001C1C6B017C0108C0C0904B17D0904C17C9
:10DA0000E0904D17F0904E1720E030E040E251ECEE
:10DA1000C701B6010F947D1E87FD0AC020E030E0EB
:10DA200040E251E4C701B6010F94331518163CF4D7
:10DA30000F94F8018BE793E10F941301BFC040E00E
:10DA400050E060EC7FE788E50E94F2AF209122135E
:10DA50003091231340912413509125130F941C1CD3
:10DA60002B013C0140E050E060EC7FE789E50E943B
:10DA7000F2AF209126133091271340912813509133
:10DA800029130F941C1C4B015C016FEF89E40E9469
:10DA9000F690182F6FEF8AE40E94F690082FA301EA
:10DAA0009201C301B2010F940F1F811158C0A5014B
:10DAB0009401C501B4010F940F1F811150C06091F2
:10DAC000F8127091F912072E000C880B990B0F9425
:10DAD0003A159B01AC01C301B2010F941C1C20E05C
:10DAE00030E0A9010F941D1C20E030E0A9010F9443
:10DAF000171D0F94891D162F6091FA127091FB1259
:10DB0000072E000C880B990B0F943A159B01AC0162
:10DB1000C501B4010F941C1C20E030E0A9010F9452
:10DB20001D1C20E030E0A9010F94171D0F94891DE2
:10DB3000062F812F012E000C990B97FD04C005972D
:10DB40001CF014E001C010E0802F002E000C990B97
:10DB500097FD04C005971CF004E001C000E01530FB
:10DB600068F5063058F580E00E948DAC25E0120281
:10DB7000F0011124E00FF11D07FDFA95EE0FFF1FD4
:10DB8000EE0FFF1FE45BFC4EC082D182E282F38283
:10DB9000A7019601602F812F0E94C4AE832D0E94A1
:10DBA0008DAC332059F00E9433D908C08AE40E941A
:10DBB000CCA7182F882321F00E94D3AC10E0D8C442
:10DBC00060E070E086E50E94E7909A8F898F059764
:10DBD00018F083E593E1A3C260E084E40E9422A8E8
:10DBE000282E40E050E0BA018AE50E94F2AF6DA70E
:10DBF0007EA78FA798AB40E050E86BEB75E483E518
:10DC00000E94F2AF20E030E040E752E40F94171D8D
:10DC100060935B0270935C0280935D0290935E025E
:10DC200088E40E94CCA7882309F40BC10E9495A721
:10DC30000F94891D698B7A8B8B8B9C8B69887A8872
:10DC400080902E1390902F13A0903013B09031132A
:10DC500020E030E0A901C501B4010F941D1CD62EAF
:10DC6000E72EF82E092F20E030E040EA50E40F9430
:10DC7000331587FF05C0D12CE12CF0EAFF2E00E41C
:10DC800069897A8977FE02C06F5F7F4F75956795C6
:10DC900088279927861B970B9E8B8D8BBC0163561B
:10DCA0007F4F072E000C880B990B0F943A15562EB8
:10DCB000672E782EC92E2D2D3E2D4F2D502F0F94CF
:10DCC0007D1E18161CF4D52C73010C2D6D2D7E2D88
:10DCD0008F2D902F0F94891D6B017C012B0120E06B
:10DCE00030E84DE953E4C501B4010F941D1C962E94
:10DCF000A72EB82E092F20E030E84AE953E40F940C
:10DD00007D1E181634F4912C60E8A62E7AE9B72E01
:10DD100003E469897A896C0D7D1D072E000C880B40
:10DD2000990B0F943A156B017C01292D3A2D4B2D3F
:10DD3000502F0F94331587FF04C09C2CAD2CBE2CA4
:10DD40000F2D692D7A2D8B2D902F0F94891D788F93
:10DD50006F8B8090321390903313A0903413B09057
:10DD6000351320E030E0A901C501B4010F941D1C5A
:10DD7000D62EE72EF82E092F20E030E040EA50E4BE
:10DD80000F94331587FF05C0D12CE12C50EAF52EF6
:10DD900000E46D897E8965567F4F072E000C880B45
:10DDA000990B0F943A156D8B672E782EC92E2D2D59
:10DDB0003E2D4F2D502F0F947D1E18161CF4DD881C
:10DDC00073010C2D6D2D7E2D8F2D902F0F94891D9D
:10DDD0006B017C013B0120E030E04BE953E4C501DD
:10DDE000B4010F941D1C962EA72EB82E092F20E0EB
:10DDF00030E848E953E40F947D1E181634F4912C52
:10DE000030E8A32E48E9B42E03E469897A896C0DC1
:10DE10007D1D072E000C880B990B0F943A156B0192
:10DE20007C01292D3A2D4B2D502F0F94331587FF50
:10DE300004C09C2CAD2CBE2C0F2D692D7A2D8B2D62
:10DE400021C18CE40E9415A8882369F00E9495A73F
:10DE500020912213309123134091241350912513C4
:10DE60000F941C1C2CC020E030E0A90160912E13FF
:10DE700070912F1380913013909131130F941D1CCA
:10DE80006B017C0120E030E040EA50E40F94331550
:10DE900087FD0DC020E030E0A901C701B6010F9455
:10DEA000331587FF0AC0C12CD12C760106C0C12CC6
:10DEB000D12C20EAE22E20E4F22EC701B6010F9405
:10DEC000891D2B0182E50E9415A8882369F00E9414
:10DED00095A7209122133091231340912413509140
:10DEE00025130F941C1C3CC020E030E84DE953E49E
:10DEF00060912E1370912F138091301390913113F4
:10DF00000F941D1CD62EE72EF82E092F20E030E8A6
:10DF10004AE953E40F947D1E181634F4D12C80E89E
:10DF2000E82E9AE9F92E03E4B201655C7E4F072ED4
:10DF3000000C880B990B0F943A15962EA72EB82E2D
:10DF4000C92E2D2D3E2D4F2D502F0F94331587FFA9
:10DF500003C0D92C75010C2D6D2D7E2D8F2D902F8A
:10DF60000F94891D788F6F8B86E40E9415A88823F3
:10DF700069F00E9495A720912613309127134091B4
:10DF80002813509129130F941C1C2CC020E030E062
:10DF9000A9016091321370913313809134139091E1
:10DFA00035130F941D1C6B017C0120E030E040EA2A
:10DFB00050E40F94331587FD0DC020E030E0A90137
:10DFC000C701B6010F94331587FF0AC0C12CD12CAD
:10DFD000760106C0C12CD12C00EAE02E00E4F02E20
:10DFE000C701B6010F94891D3B0182E40E9415A868
:10DFF000882369F00E9495A720912613309127135A
:10E0000040912813509129130F941C1C3CC020E010
:10E0100030E04BE953E460913213709133138091F7
:10E020003413909135130F941D1CD62EE72EF82E25
:10E03000092F20E030E848E953E40F947D1E1816BC
:10E0400034F4D12CA0E8EA2EB8E9FB2E03E4B301A6
:10E050006A5C7E4F072E000C880B990B0F943A15C3
:10E06000962EA72EB82EC92E2D2D3E2D4F2D502F7A
:10E070000F94331587FF03C0D92C75010C2D6D2D1E
:10E080007E2D8F2D902F0F94891D7B01B301072CBE
:10E09000000C880B990B0F943A156C8F7D8F8E8F27
:10E0A0009F8F69837A838B839C83B201052C000C3C
:10E0B000880B990B0F943A1568A379A38AA39BA3A5
:10E0C0006D837E838F839887BE016F5F7F4FCE0104
:10E0D00005960E94B08F882301F1B7010F2C000C28
:10E0E000880B990B0F943A1569877A878B879C87E1
:10E0F000AF89B88DBD01BB0F880B990B0F943A15F2
:10E100006D877E878F87988BBE01675F7F4FCE01BB
:10E110000D960E94B08F813029F087E393E10F9430
:10E12000130126C2298D3A8D232B69F081E293E1F8
:10E130000F941301222021F087E193E10F94130142
:10E140008AE00E942F4E0E948AA080E00E948DAC3F
:10E1500081E00E94E19D882321F0832D0E948DACF7
:10E160002DCD0F89188D0419150917FF02C00D5FF9
:10E170001F4F1595079515950795B801012E000CB1
:10E18000880B990B0F943A156CA37DA38EA39FA3C4
:10E19000E618F708F7FE03C033E0E30EF11C570161
:10E1A000B594A794B594A794B5010B2C000C880BDB
:10E1B000990B0F943A1568A779A78AA79BA70E9485
:10E1C0005CD66091401370914113072E000C880BB0
:10E1D000990B0F943A159B01AC016CA17DA18EA106
:10E1E0009FA10F943315811122C060914213709149
:10E1F0004313072E000C880B990B0F943A159B01C3
:10E20000AC0168A579A58AA59BA50F94331581114A
:10E210000EC08091F8129091F9124816590639F4FF
:10E220008091FA129091FB126816790699F00E947B
:10E23000D3AC1093411300934013B0924313A092B8
:10E2400042135092F9124092F8127092FB126092AF
:10E25000FA12312C60E085E40E9422A8882319F08C
:10E2600061E06CA702C082E08CA791E09B8FE12C5B
:10E27000F12C812C912C5401A1E0A98BB1E0BD8B34
:10E2800025E02F8B10E07AEEC72E72E1D72EE9AA97
:10E29000A989B1E0AB27A98B0B8DC7010F2C000C0E
:10E2A000AA0BBB0B8AAB9BABACABBDAB9F899117E9
:10E2B00009F4BEC0612F012E000C770B880B990B5F
:10E2C0000F943A152CA13DA14EA15FA10F94991571
:10E2D00028A139A14AA15BA10F941D1C2B013C016F
:10E2E0006AA97BA98CA99DA90F943A1528A539A5DF
:10E2F0004AA55BA50F9499152C8D3D8D4E8D5F8D94
:10E300000F941D1C4B015C0120E030E0A901C3010A
:10E31000B2010F94331587FF04C020E030E0A9015B
:10E3200004C020E030E040E05FE3C301B2010F949D
:10E330001D1C0F94BF1D69837A838B839C8320E00F
:10E3400030E0A901C501B4010F94331587FF04C063
:10E3500020E030E0A90104C020E030E040E05FE3CD
:10E36000C501B4010F941D1C0F94BF1D6D837E83E6
:10E370008F839887A98DBA8DAB2B81F0602F70E0C9
:10E3800083E093E10F94D80169E170E081E093E1CB
:10E390000F94D8018EEF92E10F9413011F92B9E10F
:10E3A000BF931F920F93DF92CF921F920E94B5826C
:10E3B000298D4CA5BE016B5F7F4FCE0101960E9457
:10E3C000ABE84B015C010FB6F894DEBF0FBECDBFCA
:10E3D0009B01AC010F940F1F882321F0832D0E9415
:10E3E0008DAC33C0A50194016DA57EA58FA598A91C
:10E3F0000F941D1C9B01AC0165E01603F001112474
:10E40000EE0DFF1DEE0FFF1FEE0FFF1FE45BFC4E36
:10E41000208331834283538369A9812F0E94C4AE34
:10E4200080E00E945B4F0F5F8D89180F312C3ECF2B
:10E4300094E0E916F10449F0A5019401C501B40185
:10E440000F940F1F882309F47EC00E9431E180E001
:10E450000E94E19D882351F0832D0E948DAC812C78
:10E46000912C90ECA92E9FE7B92E52C0A5019401E2
:10E47000C501B4010F940F1F81114AC0222001F180
:10E480000F9422010E94CFFE21103FC083E497E148
:10E490000E94B6FC9B01AC0160914B1770914C1728
:10E4A00080914D1790914E170F941C1C60934B1741
:10E4B00070934C1780934D1790934E1781E026C0B0
:10E4C00012E084E0F82E02E0EF2CE11ADF2CD01AE3
:10E4D00021E041E0602F812F0E943CFF21E04FEFBF
:10E4E000602F8E2D0E943CFF2FEF41E06D2D812F7C
:10E4F0000E943CFF2FEF4FEF6D2D8E2D0E943CFFB1
:10E50000015020F71150F8F6BBCF832D80935B1795
:10E510000E9443D680915B1781110E9407D80E9408
:10E52000999D0E948AA089EE92E10E94C6D00E9425
:10E5300033D911E0A5019401C501B4010F940F1F57
:10E54000811116C03BCBA989AA2361F031E03D8B34
:10E5500065E06F8B10E08FEFE81AF80A9B8D9B5FE8
:10E560009B8F95CEBFEFBD8B2FEF2F8B14E0F3CF9A
:10E57000812FE5960FB6F894DEBF0FBECDBFDF91B9
:10E58000CF911F910F91FF90EF90DF90CF90BF90B0
:10E59000AF909F908F907F906F905F904F903F9043
:10E5A0002F9008952F923F924F925F926F927F9299
:10E5B0008F929F92AF92BF92CF92DF92EF92FF9293
:10E5C0000F931F93CF93DF93CDB7DEB7CD58D1090B
:10E5D0000FB6F894DEBF0FBECDBF5B016A01190113
:10E5E000E996FFAEEEAEE99720915C1030915D1098
:10E5F00040915E1050915F10DC016D917D918D9185
:10E600009C910F9499150F948A1E2B013C0125961D
:10E610006CAF7DAF8EAF9FAF25972091601030918A
:10E6200061104091621050916310F5016081718119
:10E63000828193810F9499150F948A1E4B015C017E
:10E6400029966CAF7DAF8EAF9FAF29972091641054
:10E65000309165104091661050916710D6016D9110
:10E660007D918D919C910F9499150F948A1E6B0149
:10E670007C012D966CAF7DAF8EAF9FAF2D97209113
:10E6800068103091691040916A1050916B10F1013F
:10E6900060817181828193810F9499150F948A1EF4
:10E6A00067966CAF7DAF8EAF9FAF679761966CAF8B
:10E6B0007DAF8EAF9FAF61978091471083FF0EC0F3
:10E6C00067962CAD3DAD4EAD5FAD67972093F214CC
:10E6D0003093F3144093F4145093F5148091451043
:10E6E00090914610892B11F00C94C280D801BC91F6
:10E6F000A896BFAFA897F801F181AC96FFAFAC9791
:10E70000D8011296BC91E096BFAFE097F801038163
:10E710008091D0149091D114891B8F708F3021F487
:10E7200080E00E945B4FF4CFF091D014C557DF4FCB
:10E73000F883CB58D0408091D014282E312C809172
:10E74000E6149091E714A091E814B091E914481AE6
:10E75000590A6A0A7B0A8091EA149091EB14A091FD
:10E76000EC14B091ED14A5019401281B390B4A0B50
:10E770005B0B6B962CAF3DAF4EAF5FAF6B9780914D
:10E78000EE149091EF14A091F014B091F114A70140
:10E790009601281B390B4A0B5B0B6F962CAF3DAFD4
:10E7A0004EAF5FAF6F978091F2149091F314A091E8
:10E7B000F414B091F5146796CCACDDACEEACFFACC4
:10E7C0006797C81AD90AEA0AFB0A09F472C080914D
:10E7D000AD0B811128C06091B20B7091B30B809189
:10E7E000B40B9091B50B0F94891D209119023091B3
:10E7F0001A0262177307BCF467968CAD9DADAEAD7F
:10E80000BFAD67978093F2149093F314A093F41420
:10E81000B093F5140F94FC0182E095E10F9413017D
:10E82000C12CD12C7601C701B6010F943A15209165
:10E8300015023091160240911702509118020F9460
:10E8400099154B015C0120E030E0A9010F947D1E79
:10E8500087FF04C0B7FAB094B7F8B09420E030E076
:10E860004AEF53E4609168107091691080916A10CA
:10E8700090916B100F949915A50194010F94331585
:10E8800087FF17C067962CAD3DAD4EAD5FAD679766
:10E890002093F2143093F3144093F4145093F5142E
:10E8A0000F94FC0183EE94E10F941301C12CD12C41
:10E8B0007601D301C2018827B7FD83959927AA273E
:10E8C000BB27182F6B962CAD3DAD4EAD5FAD6B9752
:10E8D00057FD12606F968CAD9DADAEADBFAD6F971D
:10E8E000B7FD1460F7FC1860C701B6010F943A1524
:10E8F0002091150230911602409117025091180292
:10E900000F9499156B017C0120E030E0A9010F9470
:10E910007D1E87FF04C0C701B601905802C0C70121
:10E92000B60120E030E040E05FE30F941D1C0F943F
:10E93000901DE7966CAF7DAF8EAF9FAFE79788E4F1
:10E94000829DF001839DF00D1124EB53F44F108252
:10E9500015AB5301420177FE07C088249924540166
:10E9600084189508A608B70888E4829DF001839D65
:10E97000F00D1124EB53F44F858A968AA78AB08E46
:10E980006B962CAD3DAD4EAD5FAD6B9767962CAFE2
:10E990003DAF4EAF5FAF679757FF0DC050954095A5
:10E9A000309521953F4F4F4F5F4F67962CAF3DAF4E
:10E9B0004EAF5FAF679788E4829DF001839DF00DB5
:10E9C0001124EB53F44F67968CAD9DADAEADBFAD4A
:10E9D0006797818F928FA38FB48F6F962CAD3DADCB
:10E9E0004EAD5FAD6F97A3962CAF3DAF4EAF5FAF0F
:10E9F000A39757FF0DC050954095309521953F4FF7
:10EA00004F4F5F4FA3962CAF3DAF4EAF5FAFA39775
:10EA100088E4829DF001839DF00D1124EB53F44FA7
:10EA2000A3968CAD9DADAEADBFADA397858F968FF0
:10EA3000A78FB0A3C301B2010F943A1520919D0B8B
:10EA400030919E0B40919F0B5091A00B0F94991504
:10EA5000A7966CAF7DAF8EAF9FAFA79769AB7AAB30
:10EA60008BAB9CAB6B966CAD7DAD8EAD9FAD6B975C
:10EA70000F943A152091A10B3091A20B4091A30B5A
:10EA80005091A40B0F9499152B013C016DAB7EABFB
:10EA90008FAB98AF6F966CAD7DAD8EAD9FAD6F9720
:10EAA0000F943A152091A50B3091A60B4091A70B1E
:10EAB0005091A80B0F9499156B966CAF7DAF8EAFEC
:10EAC0009FAF6B9769AF7AAF8BAF9CAF2091A90BCB
:10EAD0003091AA0B4091AB0B5091AC0BC701B60122
:10EAE0000F9499156B017C0121966CAF7DAF8EAFB1
:10EAF0009FAF219796E089169104A104B1041CF5FB
:10EB000067962CAD3DAD4EAD5FAD679726303105B4
:10EB100041055105C4F4A3968CAD9DADAEADBFAD1E
:10EB2000A3970697A105B10574F420E030E0A90190
:10EB3000C701B6010F947D1E87FF16C0F7FAF09447
:10EB4000F7F8F09411C0E996AEADBFADE997CD905E
:10EB5000DD90ED90FC9020E030E0A901C701B60106
:10EB60000F943315882369F088E4829DF001839D1A
:10EB7000F00D1124EB53F44FC586D686E786F08A54
:10EB800038C0A7962CAD3DAD4EAD5FADA797CA017D
:10EB9000B9010F9499156B017C01A3019201C30186
:10EBA000B2010F9499159B01AC01C701B6010F94F6
:10EBB0001D1C6B017C016B962CAD3DAD4EAD5FAD68
:10EBC0006B97CA01B9010F9499159B01AC01C7015C
:10EBD000B6010F941D1C0F94CB1E28E4229DF0015A
:10EBE000239DF00D1124EB53F44F658776878787BB
:10EBF000908B88E4829DF001839DF00D1124EB53EE
:10EC0000F44FE7962CAD3DAD4EAD5FADE79721A338
:10EC100032A343A354A3582D492D3A2D2B2D67968B
:10EC20008CAD9DADAEADBFAD679788169906AA06AF
:10EC3000BB0660F464965FAD649765964FAD6597CB
:10EC400066963FAD669767962FAD6797852F942F91
:10EC5000A32FB22FA3962CAD3DAD4EAD5FADA397C4
:10EC600082179307A407B50710F4DA01C901E796E4
:10EC70002CAD3DAD4EAD5FADE79782179307A4076E
:10EC8000B50710F4DA01C90128E4229DF001239DA3
:10EC9000F00D1124EB53F44F85A396A3A7A3B0A7BF
:10ECA0000697A105B10510F40C945081DF01AA5B11
:10ECB000BF4F80919B0B8C93E95BFF4F80919C0B26
:10ECC000808389288A288B2809F05F9888E4829DB0
:10ECD000F001839DF00D1124EB53F44F818D928D43
:10ECE000A38DB48D892B8A2B8B2B09F08A9888E40D
:10ECF000829DF001839DF00D1124EB53F44F858D1F
:10ED0000968DA78DB0A1892B8A2B8B2B29F0809112
:10ED10000801817080930601E7968CAD9DADAEAD84
:10ED2000BFADE797892B8A2B8B2B11F40C94C480F1
:10ED30008091A010882319F081508093A010129820
:10ED400080E28093A010D0908810E0908910F0901D
:10ED50008A1010918B102D2D3E2D4F2D512FA896DE
:10ED60006FADA897AC967FADAC97E0968FADE0976E
:10ED7000902F0F94331587FF0AC0A896DFAEA8978F
:10ED8000AC96EFAEAC97E096FFAEE097012F88E42B
:10ED9000829DF001839DF00D1124EB53F44F2585E6
:10EDA000368547855089EB962CAF3DAF4EAF5FAFB0
:10EDB000EB9760E070E080E89FE30F94171DA79643
:10EDC0006CAF7DAF8EAF9FAFA797A8962FADA897DA
:10EDD000AC963FADAC97E0964FADE097502F0F94B7
:10EDE00099154B015C018091D0149091CE14891B30
:10EDF0008F70EC968FAFEC97A501940160E074E200
:10EE000084E799E40F94171D0F948A1E6B017C010F
:10EE1000EC968FADEC9782508630C0F580915810FB
:10EE200090915910A0915A10B0915B10C816D90654
:10EE3000EA06FB0658F58C199D09AE09BF09BC010D
:10EE4000CD01660F771F881F991FEC964FADEC9789
:10EE5000042F10E020E030E0A90198010F94891BF5
:10EE6000CA01B9010F9438150F948A1E6C0D7D1DCF
:10EE70008E1D9F1D0F9438159B01AC0160E074E25C
:10EE800084E799E40F94171D4B015C01A5019401DF
:10EE9000EB966CAD7DAD8EAD9FADEB970F94991554
:10EEA0009B01AC010F949915C158DF4F688379839A
:10EEB0008A839B83CF57D04088E4829D8001839DC5
:10EEC000100D11240B53144FC158DF4F88819981C5
:10EED000AA81BB81CF57D040F80181839283A3835D
:10EEE000B48325A136A147A150A5AB962CAF3DAF69
:10EEF0004EAF5FAFAB97CA01B9010F943815AF960B
:10EF00006CAF7DAF8EAF9FAFAF979B01AC01C501DA
:10EF1000B4010F9499150F94FB1C0F94901DCD57BD
:10EF2000DF4F688379838A839B83C358D040F8017D
:10EF300066AB77AB80AF91AF8E010F5C1F4F9E0128
:10EF40002F5D3F4FE1963FAF2EAFE1974CE650E18A
:10EF5000C757DF4F59834883C958D040C8014096EE
:10EF6000C457DF4F99838883CC58D040C957DF4FAF
:10EF700039832883C758D04064961FAE649768963B
:10EF80001FAE689790E86C969FAF6C97AFE3A09622
:10EF9000AFAFA097F80121913191419151918F012B
:10EFA000C501B4010F9499156B017C01C957DF4F5E
:10EFB000A881B981C758D0406D937D938D939D935F
:10EFC000C957DF4FB983A883C758D04020E030E04D
:10EFD000A9010F947D1E87FF04C0F7FAF094F7F89B
:10EFE000F094C757DF4FE881F981C958D04041906C
:10EFF000519061907190C757DF4FF983E883C958EA
:10F00000D040A7019601C301B2010F94331587FFC9
:10F0100024C0A7019601C301B2010F94171D7B0103
:10F020006C0164962FAD649768963FAD68976C96B7
:10F030004FAD6C97A0965FADA0970F94331587FFE7
:10F040000CC06496EFAE64976896FFAE68976C96B6
:10F05000CFAE6C97A096DFAEA097C457DF4F288144
:10F060003981CC58D0402017310709F093CF20E0E8
:10F0700030E040E85FE364966FAD649768967FADDB
:10F0800068976C968FAD6C97A0969FADA0970F94E4
:10F09000331587FF7AC08E010F5C1F4F64962FAD2A
:10F0A000649768963FAD68976C964FAD6C97A09645
:10F0B0005FADA097E196AEADBFADE1976D917D914B
:10F0C0008D919C910F949915E196EEADFFADE1976E
:10F0D0006193719381939193E196FFAFEEAFE197C6
:10F0E0000E171F07D9F688E4829D8001839D100DBD
:10F0F00011240B53144FCD57DF4F688179818A81DA
:10F100009B81C358D0400F94381564962FAD6497F7
:10F1100068963FAD68976C964FAD6C97A0965FADC3
:10F12000A0970F9499150F94901DD801D6966D93C2
:10F130007D938D939C93D99764962FAD6497689631
:10F140003FAD68976C964FAD6C97A0965FADA0975A
:10F1500064966FAD649768967FAD68976C968FAD37
:10F160006C97A0969FADA0970F949915C158DF4F4B
:10F17000288139814A815B81CF57D0400F949915FE
:10F18000F8016183728383839483AF962CAD3DAD88
:10F190004EAD5FADAF97A7966CAD7DAD8EAD9FAD1B
:10F1A000A7970F94991567966CAF7DAF8EAF9FAF01
:10F1B000679788E4829DF001839DF00D1124EB5345
:10F1C000F44F85889688A788B08C81149104A10497
:10F1D000B10419F5818D928DA38DB48D892B8A2B65
:10F1E0008B2BD9F4858D968DA78DB0A1892B8A2B79
:10F1F0008B2B99F4209180103091811040918210D6
:10F200005091831067966CAD7DAD8EAD9FAD6797C5
:10F210000F9499150F94FB1C2BC2E7962CAD3DADB6
:10F220004EAD5FADE797232B242B252B49F0209182
:10F230007C1030917D1040917E1050917F1008C05D
:10F240002091841030918510409186105091871044
:10F2500067966CAD7DAD8EAD9FAD67970F94991598
:10F260000F94FB1C0F94901D6B017C018091970BF8
:10F270009091980BA091990BB0919A0BAB962CADF5
:10F280003DAD4EAD5FADAB9782179307A407B507B1
:10F2900008F4D6C081149104A104B10411F1609165
:10F2A000870B7091880B8091890B90918A0B6C155C
:10F2B0007D058E059F05A8F40F94791B2B013C0159
:10F2C000A5019401C701B6010F94791B4616570694
:10F2D0006806790630F4C301B2010F94891B6901F5
:10F2E0007A0188E4829DF001839DF00D1124EB5397
:10F2F000F44F818C928CA38CB48C81149104A10462
:10F30000B10441F160918B0B70918C0B80918D0B4E
:10F3100090918E0B6C157D058E059F05D8F4AB96EC
:10F320002CAD3DAD4EAD5FADAB970F94791B2B016E
:10F330003C01A5019401C701B6010F94791B461643
:10F3400057066806790630F4C301B2010F94891B91
:10F3500069017A0188E4829DF001839DF00D1124FA
:10F36000EB53F44F858C968CA78CB0A0811491043C
:10F37000A104B10441F160918F0B7091900B8091C9
:10F38000910B9091920B6C157D058E059F05D8F41D
:10F39000AB962CAD3DAD4EAD5FADAB970F94791BE9
:10F3A0002B013C01A5019401C701B6010F94791B03
:10F3B000461657066806790630F4C301B2010F9469
:10F3C000891B69017A0188E4829DF001839DF00D1B
:10F3D0001124EB53F44F81A092A0A3A0B4A08114F8
:10F3E0009104A104B10409F447C16091930B709199
:10F3F000940B8091950B9091960B6C157D058E0565
:10F400009F0508F039C1AB962CAD3DAD4EAD5FAD5B
:10F41000AB970F94791B2B013C01A5019401C70107
:10F42000B6010F94791B461657066806790608F050
:10F4300023C1C301B2010F94891B69017A011CC168
:10F4400081149104A104B104C9F16091870B7091FA
:10F45000880B8091890B90918A0B6C157D058E0528
:10F460009F0560F50F943815AF962CAD3DAD4EADB0
:10F470005FADAF970F9499152B013C01C501B40105
:10F480000F9438154B015C01C701B6010F94381574
:10F49000A50194010F9499159B01AC01C301B20120
:10F4A0000F94331587FF0AC0A5019401C301B2016F
:10F4B0000F94171D0F94901D6B017C0188E4829DB1
:10F4C000F001839DF00D1124EB53F44F418C528CCD
:10F4D000638C748C4114510461047104C9F160910E
:10F4E0008B0B70918C0B80918D0B90918E0B6C150A
:10F4F0007D058E059F0560F50F943815AF962CADF0
:10F500003DAD4EAD5FADAF970F9499154B015C01CA
:10F51000C301B2010F9438152B013C01C701B6019C
:10F520000F943815A30192010F9499159B01AC011A
:10F53000C501B4010F94331587FF0AC0A3019201DE
:10F54000C501B4010F94171D0F94901D6B017C0130
:10F5500088E4829DF001839DF00D1124EB53F44F5C
:10F56000458C568C678C70A0411451046104710461
:10F57000C9F160918F0B7091900B8091910B9091DC
:10F58000920B6C157D058E059F0560F50F9438155F
:10F59000AF962CAD3DAD4EAD5FADAF970F949915C5
:10F5A0004B015C01C301B2010F9438152B013C01E2
:10F5B000C701B6010F943815A30192010F94991554
:10F5C0009B01AC01C501B4010F94331587FF0AC03C
:10F5D000A3019201C501B4010F94171D0F94901D52
:10F5E0006B017C0188E4829DF001839DF00D112464
:10F5F000EB53F44F81A092A0A3A0B4A08114910476
:10F60000A104B104C9F16091930B7091940B8091A6
:10F61000950B9091960B6C157D058E059F0560F5F9
:10F620000F943815AF962CAD3DAD4EAD5FADAF9795
:10F630000F9499152B013C01C501B4010F943815A5
:10F640004B015C01C701B6010F943815A501940167
:10F650000F9499159B01AC01C301B2010F943315AE
:10F6600087FF0AC0A5019401C301B2010F94171DC1
:10F670000F94901D6B017C0188E4829D8001839D25
:10F68000100D11240B53144FF801EE5BFF4FC08295
:10F69000D182E282F382C701B6010F9438156B0163
:10F6A0007C0167962CAD3DAD4EAD5FAD67970F9475
:10F6B000171DAB966CAF7DAF8EAF9FAFAB97D801E8
:10F6C00051966D937D938D939C9354972DEB37E3D7
:10F6D00046E051E4C701B6010F9499150F94901DAF
:10F6E000F80161AB72AB83AB94AB29A93AA94BA9E2
:10F6F0005CA9A7966CAD7DAD8EAD9FADA7970F941D
:10F700009915AF966CAF7DAF8EAF9FAFAF97698BFA
:10F710007A8B8B8B9C8B2DA93EA94FA958ADA796B0
:10F720006CAD7DAD8EAD9FADA7970F9499154B0134
:10F730005C016D8B7E8B8F8B988F29AD3AAD4BAD75
:10F740005CADA7966CAD7DAD8EAD9FADA7970F94C8
:10F7500099156B017C01698F7A8F8B8F9C8F219615
:10F760002CAD3DAD4EAD5FAD2197A7966CAD7DAD97
:10F770008EAD9FADA7970F949915A7966CAF7DAFEF
:10F780008EAF9FAFA7976D8F7E8F8F8F98A3EC96CC
:10F79000FFADEC97FF2309F4BBC22091D21464960D
:10F7A0002FAF64973091D31468963FAF689740911C
:10F7B000D4146C964FAF6C975091D514A0965FAF50
:10F7C000A0972DEB37E346E855E364966FAD649759
:10F7D00068967FAD68976C968FAD6C97A0969FAD3D
:10F7E000A0970F94331587FD93C28091901090914C
:10F7F0009110A0919210B0919310E7968CAF9DAFAD
:10F80000AEAFBFAFE7972091941030919510409123
:10F81000961050919710E3962CAF3DAF4EAF5FAF6F
:10F82000E3978091981090919910A0919A10B091BF
:10F830009B10EF968CAF9DAFAEAFBFAFEF9720910F
:10F840009C1030919D1040919E1050919F10C15876
:10F85000DF4F288339834A835B83CF57D040E796B5
:10F860006CAD7DAD8EAD9FADE7979058AF962CAD4A
:10F870003DAD4EAD5FADAF970F9499152B013C0197
:10F88000E3962CAD3DAD4EAD5FADE397C501B40140
:10F890000F9499159B01AC01C301B2010F941C1C7C
:10F8A0002B013C01EF962CAD3DAD4EAD5FADEF971A
:10F8B000C701B6010F9499159B01AC01C301B201B8
:10F8C0000F941C1C2B013C01C158DF4F288139814A
:10F8D0004A815B81CF57D040A7966CAD7DAD8EAD90
:10F8E0009FADA7970F9499159B01AC01C301B2017D
:10F8F0000F941C1C2B013C012FEE3FEF4FE75FE301
:10F900000F947D1E18160CF4B2C12FEE3FEF4FE797
:10F910005FEBC301B2010F94331587FF08C0EFEE10
:10F920004E2E55245A94EFE76E2EEFEB7E2EE7967F
:10F930002CAD3DAD4EAD5FADE797AF966CAD7DADF7
:10F940008EAD9FADAF970F941C1C69837A838B8318
:10F950009C83E3962CAD3DAD4EAD5FADE397C50105
:10F96000B4010F941C1C6D837E838F839887EF9660
:10F970002CAD3DAD4EAD5FADEF97C701B6010F9415
:10F980001C1C69877A878B879C87C158DF4F288129
:10F9900039814A815B81CF57D040A7966CAD7DAD50
:10F9A0008EAD9FADA7970F941C1C6D877E878F87A8
:10F9B000988BAE014F5F5F4FA5965FAF4EAFA59797
:10F9C000CE01419663969FAF8EAF63978A01C12C9B
:10F9D000D12C7601D8018D909D90AD90BD908D0178
:10F9E00020E030E0A901C501B4010F94331588234C
:10F9F00071F0A5019401C501B4010F9499159B0103
:10FA0000AC01C701B6010F941D1C6B017C0163960C
:10FA1000EEADFFAD6397E017F107E1F6C701B60160
:10FA20000F94CB1E9B01AC0160E070E080E89FE387
:10FA30000F94171D6B017C01A5960EAD1FADA59708
:10FA4000A7019601D8016D917D918D919C910F94A4
:10FA50009915F80161937193819391938F01639646
:10FA60002EAD3FAD63972E173F0751F778E4A72ED1
:10FA700070E1B72EA8963FADA897AC963FAFAC9774
:10FA8000A9964FADA997E4964FAFE497AA960FAD0C
:10FA9000AA97AB961FADAB97A596AEADBFADA59798
:10FAA000CD90DD90ED90FD90A596BFAFAEAFA59740
:10FAB00020E030E0A901C701B6010F943315882377
:10FAC00061F1F50160817181828193810F94381514
:10FAD000A70196010F94171D6B017C0120E030E017
:10FAE000A9010F947D1E87FF04C0F7FAF094F7F880
:10FAF000F094AC962FADAC97E4963FADE497A80197
:10FB0000C701B6010F94331587FF07C0AC96CFAE7F
:10FB1000AC97E496DFAEE4978701F4E0AF0EB11C3A
:10FB200063962EAD3FAD6397A5964EAD5FADA5979D
:10FB30002417350709F0B0CFA301920160E070E00F
:10FB400080E89FE30F941C1C20E030E040E05FE37E
:10FB50000F9499150F94CB1E6B017C012091830BA0
:10FB60003091840B4091850B5091860BAC966FAD14
:10FB7000AC97E4967FADE497C8010F949915A7015F
:10FB800096010F9499154B015C01A701960160E065
:10FB900070E080E89FE30F941C1C9B01AC01C50141
:10FBA000B4010F94171D6B017C0120E030E040E8A8
:10FBB0005FE3EB966CAD7DAD8EAD9FADEB970F9493
:10FBC000331587FF5CC0A3019201C301B2010F94FA
:10FBD000991523EC38EB42E35FEB0F94991523EF73
:10FBE00036E64FE55FE30F941C1CA30192010F94CE
:10FBF00099152BED3FE049EC5FE30F941D1C2CEEB3
:10FC000031E548E35EE30F941C1C4B015C0124EEDC
:10FC10003BEC46E150E40F947D1E181684F5A501D7
:10FC200094016BED7FE089E490E40F941C1C9B0130
:10FC3000AC01EB966CAD7DAD8EAD9FADEB970F94A7
:10FC4000171DAC962FADAC97E4963FADE497A80195
:10FC50000F9499155B018C019B01AC01B601C701A2
:10FC60000F947D1E18165CF46501780108C03BE016
:10FC7000C32E47EDD42E53E2E52E6BE3F62E88E437
:10FC8000829DF001839DF00D1124EB53F44FA18070
:10FC9000B280038114819501A80164966FAD6497C9
:10FCA00068967FAD68976C968FAD6C97A0969FAD68
:10FCB000A0970F947D1E181664F46496AFAE6497F7
:10FCC0006896BFAE68976C960FAF6C97A0961FAF03
:10FCD000A0979601A70164966FAD649768967FAD73
:10FCE00068976C968FAD6C97A0969FADA0970F9478
:10FCF0007D1E1816CCF46496CFAE64976896DFAE7E
:10FD000068976C96EFAE6C97A096FFAEA0970CC06C
:10FD100064961FAE649768961FAE68976C961FAE88
:10FD20006C97A0961FAEA09780E1FE017196A0E9A6
:10FD3000B0E101900D928A95E1F788E4829D8001FF
:10FD4000839D100D11240B53144F64968FAD64974F
:10FD500068969FAD68976C96AFAD6C97A096BFAD57
:10FD6000A097F80181879287A387B487AB966CAD83
:10FD70007DAD8EAD9FADAB9790589B01AC010F94BC
:10FD80001D1CD8011D962D913D914D915C91509770
:10FD90000F9499159B01AC016BE077ED83E29BE337
:10FDA0000F941C1C2BE0C22E27EDD22E23E2E22E54
:10FDB0002BE3F22EF801C582D682E782F086B0806E
:10FDC000C180D280E380F480A70196010F947D1E4C
:10FDD00087FD02C083E001C081E08B2998E4929DF9
:10FDE000F001939DF00D1124EB53F44F808380E1DB
:10FDF000FE01B196A6EDB4E101900D928A95E1F76E
:10FE0000C092D214D092D314E092D414F092D514AC
:10FE100080E1FE01EF5BFF4FA6EEB4E101900D9291
:10FE20008A95E1F79091D0148091D114981303C072
:10FE300084E68093CD14C557DF4F8881CB58D040DE
:10FE40008F5F8F708093D0148091D0149091CF14D5
:10FE500081508F70891709F4ABC0F090D0148FEFE8
:10FE60008F0D8F7064968FAF6497E090CF14809160
:10FE7000D014E81609F46BC0C12CD12C6496FFADE8
:10FE80006497FE1509F463C08F2E912C28E4289DF9
:10FE90008001299D100D11240B53144FD8018C9112
:10FEA00083FD32C0A4960FAFA497A8961FAFA89762
:10FEB0001996BC916896BFAF6897F801F2856C9669
:10FEC000FFAF6C97D8011B96BC91A096BFAFA097CF
:10FED000F801F4842580368047805084A201910186
:10FEE00068966FAD68976C967FAD6C978B2F9F2D42
:10FEF0000F943315811152C1C114D10459F0D601A8
:10FF00008C9180FD4BC106C0A496CFAEA497A89655
:10FF1000DFAEA89764968FAD649781508F7064961A
:10FF20008FAF64978091CF148E1107C0A496CFAC89
:10FF3000A497A896DFACA897A1CF6496FFAD64976D
:10FF4000FE1529F081E08E0D8F70E82EEBCF209109
:10FF5000CF1464962FAF6497C12CD12C8091D0140C
:10FF600064963FAD6497831719F1832E912C48E472
:10FF7000489D8001499D100D11240B53144FD80149
:10FF80008C9183FD0AC05801C114D10439F0C60117
:10FF90000E944788811102C08AC1560164968FADC4
:10FFA00064978F5F8F7064968FAF64976501D6CF2B
:10FFB000D090D1148090D01428E4D81469F08FEF39
:10FFC000880D8F70289FF0011124EB53F44F90811E
:10FFD00093FF02C0882EF1CF212C312C412C512CC3
:10FFE00064961FAE649768961FAE6897712C612C5B
:10FFF00000E010E0E12CF12C8D1409F481C048E4FC
:020000021000EC
:100000004D9D800111240B53144FD8018C9183FD19
:1000100019C015966D917D918D919C9118970F94B3
:10002000CB1EC62EB72EA82E992EE114F10409F48A
:1000300055C0F701808180FD0EC0D8018C9180FDF4
:100040000AC04CC06496CFAC64976896BFAC689702
:10005000A72C962C48C0F701808181608083C7015E
:100060000E944788811136C0F701618172818381C6
:1000700094810F94CB1E9B01AC0160E070E080E89E
:100080009FE30F94171D1B012C019B01AC016C2DEC
:100090007B2D8A2D992D0F94991569837A838B83F3
:1000A0009C8364962FAD649768963FAD6897472D03
:1000B000562DC201B1010F949915698B7A8B8B8BE8
:1000C0009C8BAE014F5F5F4FBE016F5E7F4FC701DC
:1000D0000E945AA3D7018C918E7F8C932C2C3B2CA1
:1000E0004A2C592C780181E08D0D8F70D82E6496A2
:1000F000CFAE64976896BFAE68977A2C692C7CCF98
:100100000115110509F4CCC0F8018081816080835C
:10011000C7010E944788811130C0D80111966D91A6
:100120007D918D919C9114970F94CB1E9B01AC01F6
:1001300060E070E080E89FE30F94171D6B017C0185
:100140002DEC3CEC4CE45DE30F94991569837A83C4
:100150008B839C839101A201C701B6010F9499156D
:10016000698B7A8B8B8B9C8BAE014F5F5F4FBE018F
:100170006F5E7F4FC8010E945AA3F80180818E7F75
:1001800080838EC080E015C1D0908C10E0908D10DF
:10019000F0908E1010918F100C94AB7628E4289D6F
:1001A000F001299DF00D1124EB53F44F808181FD66
:1001B00045C0C114D10431F0F601A580B680C780D6
:1001C000D08408C08BE0A82E87EDB82E83E2C82E1D
:1001D0008BE3D82E28E4289DF001299DF00D1124F1
:1001E000EB53F44F81899289A389B489BC01CD0175
:1001F00090589B01AC010F941D1CD8011D962D91A8
:100200003D914D915C9150970F9499159B01AC01D4
:10021000C601B5010F941C1C3B015C019B01AC01A4
:1002200068966FAD68976C967FAD6C97A0968FAD12
:10023000A0979F2D0F94331587FF0AC068966FAC67
:1002400068976C967FAC6C97A096AFACA097BF2CCC
:100250009301A501C201B1010F943315882309F45C
:1002600059CEB8E4B89DC001B99D900D1124FC0190
:10027000EB53F44F6F01808181608083C8010E943D
:100280004788882329F0D6018C918E7F8C9342CEAB
:10029000C301D501F60185839683A783B0873ACE43
:1002A00080916F00826080936F0081E082C0D601F0
:1002B0008C9181FD58C0D60115962D913D914D919F
:1002C0005C9118976B962CAF3DAF4EAF5FAF6B97BD
:1002D0001501B5E02B0E311CF80145805680678072
:1002E0007084A30192016B966CAD7DAD8EAD9FAD18
:1002F0006B970F94331587FF36C0F6018189928979
:10030000A389B489BC01CD0190589B01AC010F9425
:100310001D1CD6011D962D913D914D915C915097DC
:100320000F9499159B01AC016B966CAD7DAD8EADB4
:100330009FAD6B970F941C1C6B017C019B01AC0162
:10034000C301B2010F947D1E18166CF4D8018C9174
:1003500081608C93C5010E9447888823F1F0F801E1
:1003600080818E7F808328E4289DF001299DF00DF7
:100370001124EB53F44F21853285438554856581E3
:100380007681878190850F943315811107CE64960D
:100390003FAD64973093CF1401CED101CD92DD9261
:1003A000ED92FC9213976496BFAD6497B093CF140F
:1003B000DACFC357DF4F0FB6F894DEBF0FBECDBF05
:1003C000DF91CF911F910F91FF90EF90DF90CF9031
:1003D000BF90AF909F908F907F906F905F904F9065
:1003E0003F902F900895CF92DF92EF92FF920F935C
:1003F0001F93CF93DF93CDB7DEB764970FB6F89412
:10040000DEBF0FBECDBFC98ADA8AEB8AFC8AFC0147
:1004100080819181A281B38189839A83AB83BC83DC
:10042000FB0180819181A281B3818D839E83AF8303
:10043000B887FA0180819181A281B38189879A87E7
:10044000AB87BC87F90180819181A281B3818D87BF
:100450009E87AF87B88BAE01475F5F4FBE016B5F72
:100460007F4FCE0101960E947FA28091451090910E
:100470004610892B81F4CE0141967C019E01235FB9
:100480003F4FAE01475F5F4FBE016B5F7F4F4097AD
:100490000E94D27201C080E064960FB6F894DEBF6D
:1004A0000FBECDBFDF91CF911F910F91FF90EF90C5
:1004B000DF90CF900895CF93DF93CDB7DEB76097ED
:1004C0000FB6F894DEBF0FBECDBFE3E4F7E1808145
:1004D0009181A281B38189839A83AB83BC83848118
:1004E0009581A681B7818D839E83AF83B8878085F0
:1004F0009185A285B38589879A87AB87BC878485D8
:100500009585A685B7858D879E87AF87B88BAE0109
:10051000475F5F4FBE016B5F7F4FCE0101960E9428
:100520007FA29E01235F3F4FAE01475F5F4FBE0139
:100530006B5F7F4FCE0101960E94E0A060960FB6E0
:10054000F894DEBF0FBECDBFDF91CF9108950F9419
:10055000FC016091810B7091820B80ED94E10F940E
:10056000E5018DEC94E10D941301CF93DF93CDB7AA
:10057000DEB780917F0B81110FC09E01275F3F4F37
:100580004F8158856FE370E08FE39BE00F94FA147E
:100590008FE39BE00E9483AFDF91CF9108951F937B
:1005A000CF93DF9380913E0BC82FC270D82FD470A9
:1005B000182F117080FF04C0CC2311F0D11145C059
:1005C0000F94FC0187EC94E10F941301111103C007
:1005D00088E50E942F4EC11103C089E50E942F4E6D
:1005E000D11103C08AE50E942F4E8FEB94E10F9446
:1005F0001301DD2319F04BEA55E002C043E058E057
:10060000CC2319F02BEA35E002C026EE36E01123A8
:1006100019F08BEA95E002C088EE96E05F934F9365
:100620003F932F939F938F938DEA94E19F938F93A2
:100630001F920E94B5828DB79EB709960FB6F894A7
:100640009EBF0FBE8DBF81E001C080E0DF91CF91E2
:100650001F910895AF92BF92CF92DF92EF92FF92D7
:100660000F931F93CF93DF93CDB7DEB72C970FB6C1
:10067000F894DEBF0FBECDBF2DEDC22E22E0D22EEC
:100680005C0170E0CB0183529D4F7C01CE14DF04EE
:1006900009F180E20E942F4EF60181916F010E94C4
:1006A0002F4E8AE30E942F4EF50161917191819145
:1006B00091915F018E010F5F1F4F23E041E00F9486
:1006C0000B108C01F80181918F018823F9F20E94AF
:1006D0002F4EF8CF8AE00E942F4E2C960FB6F8943A
:1006E000DEBF0FBECDBFDF91CF911F910F91FF9065
:1006F000EF90DF90CF90BF90AF9008958F929F9230
:10070000AF92BF92CF92DF92EF92FF920F931F931F
:10071000CF93DF93EC018A01C880D980EA80FB8007
:10072000072E000C880B990B0F943A154B015C01B6
:100730009B01AC01C701B6010F94331587FD10C0B2
:10074000B801110F880B990B0F943A154B015C01FE
:100750009B01AC01C701B6010F947D1E181624F44D
:1007600088829982AA82BB82DF91CF911F910F91DB
:10077000FF90EF90DF90CF90BF90AF909F908F90C1
:100780000895EF92FF920F931F93CF93C82F7B0191
:100790008A01809120028823D1F00F94F801C701CB
:1007A0000F94130181E49DE10F941301C7FD08C06C
:1007B0006C2FCC0F770B880B990B0E94A34E04C0B3
:1007C0008DE39DE10F9413018AE00E942F4E0E9459
:1007D000B7BF80910F11811108C081E080930F1184
:1007E00010922002C8010E9433FACF911F910F91FD
:1007F000FF90EF9008952F923F924F925F926F92E9
:100800007F928F929F92AF92BF92CF92DF92EF92A0
:10081000FF920F931F93CF93DF93CDB7DEB72F9740
:100820000FB6F894DEBF0FBECDBF8091C710811107
:100830001DC080918D1281111DC02F960FB6F894A6
:10084000DEBF0FBECDBFDF91CF911F910F91FF9003
:10085000EF90DF90CF90BF90AF909F908F907F9060
:100860006F905F904F903F902F90089580E090E0C0
:100870000E9433FA0E941CC10E9481EE4B015C0170
:100880006091120270911302072E000C880B990BD5
:100890000F943A159B01AC016091B20B7091B30BB0
:1008A0008091B40B9091B50B0F947D1E18163CF4FB
:1008B00046EC5DE169ED7DE180E00E94C1838091BD
:1008C0008B12882309F404C26091B60B7091B70BA8
:1008D000072E000C880B990B0F943A1569837A83C5
:1008E0008B839C833AE0E32EF12C0CE310E020E0B4
:1008F000AE014F5F5F4F62EB7BE08EE391E10E94C0
:1009000049BDC090B20BD090B30BE090B40BF09007
:10091000B50B6091100270911102072E000C880B2C
:10092000990B0F943A159B01AC01C701B6010F94C6
:100930007D1E18160CF4A0C060E06093B80B809187
:10094000781290917912A0917A12B0917B1200974F
:10095000A105B10529F1A5019401281B390B4A0B0A
:100960005B0B57FD1DC0609176127091771280E08D
:1009700090E00F9438159B01AC016091B20B70911F
:10098000B30B8091B40B9091B50B0F94331587FF87
:1009900008C345EA5DE167EB7DE180E00E94C18329
:1009A00020E030E046E153E460910D0970910E09BA
:1009B00080910F09909110090F947D1E18160CF468
:1009C000D7C180917E1290917F12A0918012B09138
:1009D00081120097A105B10529F1A5019401281BF9
:1009E000390B4A0B5B0B57FD1DC060917C12709157
:1009F0007D1280E090E00F9438159B01AC0160916E
:100A00000D0970910E0980910F09909110090F94B2
:100A1000331587FFB5C14FE55DE162E77DE18FEFFB
:100A20000E94C18380918612882309F48AC1609153
:100A3000110970911209072E000C880B990B0F9465
:100A40003A1569837A838B839C8392E0E92EF12C9B
:100A500002E310E02FEFAE014F5F5F4F6DE079E0F2
:100A600089E391E10E9449BD80918612882309F4AF
:100A700048C110921309E1CE6091120270911302E5
:100A8000072E000C880B990B0F943A159B01AC01B3
:100A9000C701B6010F94331587FF4ECF6091B60B97
:100AA0007091B70B6115710509F476C2072E000C21
:100AB000880B990B0F943A15A70196010F941C1CF3
:100AC0002B013C0120E030E040E251EC0F94331563
:100AD00087FD62C280918B1281115EC220E030E0FE
:100AE00040E251E4C301B2010F947D1E18160CF4CC
:100AF00065C280913811811166C280913011909148
:100B00003111A0913211B09133118D839E83AF8347
:100B1000B8872091341130913511409136115091A0
:100B2000371129873A874B875C87A7019601609127
:100B300024117091251180912611909127110F9405
:100B40001C1C2091C10B3091C20B4091C30B5091E2
:100B5000C40B0F9499152D813E814F8158850F94B8
:100B60001C1C20ED3CEC4CE45DE30F9499152D81A9
:100B70003E814F8158850F941D1C6B017C01609351
:100B80003011709331118093321190933311809111
:100B9000BD0B9091BE0BA091BF0BB091C00B8D838C
:100BA0009E83AF83B88729853A854B855C85C301D1
:100BB000B2010F941D1C162F072F382E292E20E06E
:100BC00030E0A9010F94331587FD12C22D813E81BB
:100BD0004F81588560E070E08FE793E40F94171D14
:100BE00069877D878E879F87212F302F432D522D38
:100BF0000F94331587FF04C019850D853E842F841B
:100C0000812F902FA32DB22D809334119093351105
:100C1000A0933611B09337112091B90B3091BA0BD4
:100C20004091BB0B5091BC0BC301B2010F949915BD
:100C30002B013C01609328117093291180932A1194
:100C400090932B11212F302F432D522D6D817E81BA
:100C50008F8198850F9499159B01AC0160932C119D
:100C600070932D1180932E1190932F11C301B20117
:100C70000F941D1CA70196010F941D1C20E030E06D
:100C8000A9010F941D1C69837A838B839C834FEF8A
:100C900050E060E070E0CE0101960E947E83C0903B
:100CA000B20BD090B30BE090B40BF090B50B698110
:100CB0007A818B819C810F94891D75956795C0926F
:100CC0002411D0922511E0922611F092271135CEF1
:100CD0008091871290918812A0918912B0918A1206
:100CE0000097A105B10509F4EFCDA5019401281BDA
:100CF000390B4A0B5B0B57FDE7CD81E080938B12DC
:100D0000E3CDC0900D09D0900E09E0900F09F0904E
:100D1000100920E030E040EA50E4C701B6010F942A
:100D20007D1E87FD0AC020E030E046E153E4C701A4
:100D3000B6010F943315181634F560E0609313096B
:100D40007CCD8091821290918312A0918412B091F7
:100D500085120097A105B10509F469CE881A990A90
:100D6000AA0ABB0AB7FC63CE81E0809386125FCEED
:100D700041E85DE165E97DE18FEF0E94C18321CE0D
:100D80000E9408BF4FCE6091110970911209611540
:100D9000710509F40AC1072E000C880B990B0F94FA
:100DA0003A15A70196010F941C1C4B015C0120E031
:100DB00030E040E251EC0F94331587FDF6C020E09F
:100DC00030E040E251E4C501B4010F947D1E1816D5
:100DD0000CF4EFC0409018095090190960901A095E
:100DE00070901B09809121028111F8C0209120117F
:100DF00030912111409122115091231180911C11A9
:100E000090911D11A0911E11B0911F118D839E8391
:100E1000AF83B887C501B4010F941D1C162F072F8F
:100E2000382E292E20E030E0A9010F94331587FDDC
:100E3000E4C0A301920160E070E08FE793E40F94B7
:100E4000171D69877D878E879F87212F302F432D20
:100E5000522D0F94331587FF04C019850D853E84EC
:100E60002F84812F902FA32DB22D8093201190934A
:100E70002111A0932211B0932311209114093091D4
:100E800015094091160950911709C501B4010F9435
:100E900099154B015C0160931411709315118093A7
:100EA000161190931711212F302F432D522DC3016E
:100EB000B2010F9499152B013C01609318117093A6
:100EC000191180931A1190931B11A701960160913B
:100ED00010117091111180911211909113110F94B2
:100EE0001C1C20911C0930911D0940911E09509134
:100EF0001F090F9499152D813E814F8158850F94BC
:100F00001C1C20ED3CEC4CE45DE30F9499152D8105
:100F10003E814F8158850F941D1C6D837E838F8386
:100F2000988760931C1170931D1180931E119093EC
:100F30001F11C0921011D0921111E0921211F09273
:100F40001311A3019201C501B4010F941D1C2D8141
:100F50003E814F8158850F941D1C20E030E0A9018F
:100F60000F941D1C6B017C0120E030E0A9010F945F
:100F7000331587FDE2CE20E030E04FE753E4C701B0
:100F8000B6010F947D1E1816BCF0C701B6010F9470
:100F9000891D75956795D2CE81E08093381160E008
:100FA0008ECE80E00E9457BFFBCC81E0809321026F
:100FB000C4CE81E0809321026FE7C0CE81E08093B0
:100FC00038116FE77CCE1092381119861A861B866D
:100FD0001C861D821E821F821886A7CD10922102B8
:100FE0001D821E821F82188620E030E0A90112CFE8
:100FF00010E000E0312C212C03CE10E000E0312C79
:10100000212C2FCF90916F00292F227091FF05C0C6
:1010100090916F009D7F90936F0034E0839FC0019B
:101020001124FC01E954FF4E40815181628173819A
:10103000FC01E555FF4E408351836283738381E059
:101040008093AA10222329F080916F008260809300
:101050006F00089590916F00292F227091FF05C0B5
:1010600090916F009D7F90936F0094E0899FF001B5
:101070001124E954FF4E6081718182819381222382
:1010800029F020916F00226020936F000895BC0129
:1010900020910D1130910E1140910D1150910E11B2
:1010A0002417350711F09A01F7CF81E0261737078B
:1010B00009F080E008952F923F924F925F926F92D5
:1010C0007F928F929F92AF92BF92CF92DF92EF92D8
:1010D000FF921F93CF93DF9300D01F92CDB7DEB75F
:1010E0008FEF9FEF90938900809388001AE01A8217
:1010F0001982B9E32B2EBDE13B2E78948091091122
:1011000090910A11A0910B11B0910C11892B8A2B8F
:101110008B2B09F0D7C18091AA108823D1F01092AF
:10112000AA1080910D1190910E11892B91F01092BF
:10113000A91010920E1110920D119091D01480915F
:10114000D114981731F08091D1148F5F8F708093F4
:10115000D11480910D1190910E11892B09F4B2C117
:101160008090051190900611A0900711B090081181
:10117000409101115091021160910311709104117D
:10118000C090F410D12CE12CF12CDB01CA0188199C
:101190009909AA09BB09C816D906EA06FB0610F484
:1011A000D701C601382F880D991DAA1DBB1D80933C
:1011B000051190930611A0930711B0930811809127
:1011C0008400909185004E96C090DC10D090DD1088
:1011D000E090DE10F090DF104091CC105091CD10D7
:1011E0006091CE107091CF104C0D5D1D6E1D7F1D56
:1011F0004093DC105093DD106093DE107093DF108D
:1012000077FD1CC0889AC090B710D090B810E090BD
:10121000B910F090BA104091A110042E000C550B9B
:10122000660B770B4C0D5D1D6E1D7F1D4093B71037
:101230005093B8106093B9107093BA10C090E0103A
:10124000D090E110E090E210F090E3104091D010C7
:101250005091D1106091D2107091D3104C0D5D1D42
:101260006E1D7F1D4093E0105093E1106093E210DB
:101270007093E31077FD1CC08E9AC090BB10D09085
:10128000BC10E090BD10F090BE104091A210042E52
:10129000000C550B660B770B4C0D5D1D6E1D7F1DF5
:1012A0004093BB105093BC106093BD107093BE1060
:1012B000C090E410D090E510E090E610F090E710B8
:1012C0004091D4105091D5106091D6107091D710E4
:1012D0004C0D5D1D6E1D7F1D4093E4105093E51075
:1012E0006093E6107093E71077FD21C020910B0109
:1012F0002095287020930901C090BF10D090C01095
:10130000E090C110F090C2104091A310042E000C88
:10131000550B660B770B4C0D5D1D6E1D7F1D4093AD
:10132000BF105093C0106093C1107093C210C09052
:10133000E810D090E910E090EA10F090EB104091A6
:10134000D8105091D9106091DA107091DB104C0DCB
:101350005D1D6E1D7F1D4093E8105093E910609352
:10136000EA107093EB1077FD1CC0149AC090C31064
:10137000D090C410E090C510F090C6104091A41019
:10138000042E000C550B660B770B4C0D5D1D6E1D6E
:101390007F1D4093C3105093C4106093C510709389
:1013A000C610409184005091850048175907C8F332
:1013B0004091DC105091DD106091DE107091DF10D3
:1013C00077FD15C0C090C810D090C910E090CA1029
:1013D000F090CB104C195D096E097F094093DC1029
:1013E0005093DD106093DE107093DF108898409169
:1013F000E0105091E1106091E2107091E31077FDE0
:1014000015C0C090C810D090C910E090CA10F090DC
:10141000CB104C195D096E097F094093E010509381
:10142000E1106093E2107093E3108E984091E41005
:101430005091E5106091E6107091E71077FD19C0AA
:10144000C090C810D090C910E090CA10F090CB1096
:101450004C195D096E097F094093E4105093E51023
:101460006093E6107093E71020910B012870209391
:1014700009014091E8105091E9106091EA107091D3
:10148000EB1077FD15C0C090C810D090C910E09047
:10149000CA10F090CB104C195D096E097F0940937A
:1014A000E8105093E9106093EA107093EB101498D1
:1014B000315041F040918400509185004817590700
:1014C000C8F381CE8091091190910A11A0910B115E
:1014D000B0910C11892B8A2B8B2B09F074C3E091EE
:1014E0000D11F0910E11309709F4F4C4809105119B
:1014F00090910611A0910711B0910811409101112E
:101500005091021160910311709104118417950795
:10151000A607B70708F46BC080911B02882309F463
:101520004CC085899689A789B08D892B8A2B8B2BF6
:10153000A1F4818D928DA38DB48D892B8A2B8B2B59
:1015400061F4858D968DA78DB0A1892B8A2B8B2B6D
:1015500021F48091CB0A882381F161A172A183A13A
:1015600094A1C090A510D090A610E090A710F09084
:10157000A81025A923FF07C09095809570956195C7
:101580007F4F8F4F9F4F0F943A152091A90B3091A9
:10159000AA0B4091AB0B5091AC0B0F9499159B018A
:1015A000AC01C701B6010F941C1C6093A510709389
:1015B000A6108093A7109093A8101092A9101092D3
:1015C0000E1110920D119091D0148091D114981792
:1015D00009F480C48091D1148F5F8F708093D114EF
:1015E000A0EDCA2EA7E0DA2EE12CF12C4EC14091DD
:1015F000FD105091FE106091FF107091001148177E
:1016000059076A077B0708F467C04091F9105091A9
:10161000FA106091FB107091FC1081A992A9A3A906
:10162000B4A9FF24499FE12C5A9F90016A9F300D75
:10163000699F200D311D4A9FE00C211D3F1D599FC0
:10164000E00C211D3F1D689FE00C211D3F1D589F90
:10165000E10C2F1D3F1DE6942F1D3F1DB49F200D53
:10166000311DB59F300D112482AD93ADA4ADB5AD44
:10167000820F931FA11DB11D8093F5109093F6105A
:10168000A093F710B093F810C6A8D7A8E0ACF1ACBF
:10169000C816D906EA06FB0640F4C092F510D092AF
:1016A000F610E092F710F092F8108090F5109090FC
:1016B000F610A090F710B090F8108DE19DE121E0B8
:1016C000FC01C590D590E590F490C814D904EA04C3
:1016D000FB0408F4C9C2D3C24091F0105091F1103C
:1016E0006091F2107091F310481759076A077B0751
:1016F00008F063C04091EC105091ED106091EE1035
:101700007091EF1081A992A9A3A9B4A9FF24499FC0
:10171000E12C5A9F90016A9F300D699F200D311D69
:101720004A9FE00C211D3F1D599FE00C211D3F1DCC
:10173000689FE00C211D3F1D589FE10C2F1D3F1D90
:10174000E6942F1D3F1DB49F200D311DB59F300D18
:101750001124C901A0E0B0E08090F5109090F6103F
:10176000A090F710B090F810FE9688159905AA057C
:10177000BB0580F4C080D180E280F380881A990A8A
:10178000AA0ABB0A8C149D04AE04BF0438F44601B7
:10179000570104C080809180A280B3808DE19DE1DB
:1017A00021E0FC01C590D590E590F490C814D904CF
:1017B000EA04FB0408F4CBC2D5C280911C029091CC
:1017C0001D02A0911E02B0911F02B7FF56C086A94C
:1017D00097A9A0ADB1AD2DE13DE141E0F901C59082
:1017E000D590E590F490C816D906EA06FB0658F4A1
:1017F000B695A79597958795440F2C5F3F4F5DE170
:101800002933350759F74093F41080329105A1052B
:10181000B10508F432C38097A109B109811528E008
:101820009207A105B10508F405C344E0949F900117
:101830001124235E364EF901329645915491EE27DC
:10184000859FB001849F610D7E1F06946E1F7E1FD1
:101850001124CB01A0E0B0E0F9014591549160E082
:1018600070E0481B590B6A0B7B0B40931C02509392
:101870001D0260931E0270931F02C0901C02D09044
:101880001D02E0901E02F0901F0280910D119091B8
:101890000E11892B09F08FC10E94649D90930E1147
:1018A00080930D11892B09F486C180910D119091BF
:1018B0000E119C838B83DC018C9183FF42C0559673
:1018C0008D919D910D90BC91A02D8093B710909318
:1018D000B810A093B910B093BA10EB81FC81818D40
:1018E000928DA38DB48D8093BB109093BC10A09368
:1018F000BD10B093BE10858D968DA78DB0A180933D
:10190000BF109093C010A093C110B093C21081A1DA
:1019100092A1A3A1B4A18093C3109093C410A093EB
:10192000C510B093C6109091D0148091D11498171F
:1019300009F4B2CF8091D1148F5F8F708093D1144E
:10194000ABCFAB81BC8155964D905D906D907C90F6
:10195000589781E0411451046104710409F480E056
:10196000EB81FC81C18CD28CE38CF48CC114D1044A
:10197000E104F10409F08260AB81BC815D964D9178
:101980005D916D917C9190974115510561057105AF
:1019900009F084608093A9101092EC101092ED1061
:1019A0001092EE101092EF101092F9101092FA109F
:1019B0001092FB101092FC10EB81FC8185A196A186
:1019C000A7A1B0A58093011190930211A0930311D8
:1019D000B0930411882499245401881A990AAA0AF8
:1019E000BB0A8092E8109092E910A092EA10B0929F
:1019F000EB108092E4109092E510A092E610B09265
:101A0000E7108092E0109092E110A092E210B09264
:101A1000E3108092DC109092DD10A092DE10B09264
:101A2000DF10440C551C661C771C4092CC10509261
:101A3000CD106092CE107092CF10CC0CDD1CEE1C3D
:101A4000FF1CC092D010D092D110E092D210F09230
:101A5000D310440F551F661F771F4093D410509327
:101A6000D5106093D6107093D71041A152A163A1F5
:101A700074A1440F551F661F771F4093D8105093D1
:101A8000D9106093DA107093DB10880F991FAA1F8A
:101A9000BB1F8093C8109093C910A093CA10B09335
:101AA000CB1010920511109206111092071110928E
:101AB000081181A592A5A3A5B4A58093FD109093CC
:101AC000FE10A093FF10B093001185A596A5A7A5C1
:101AD000B0A98093F0109093F110A093F210B093FE
:101AE000F31085A990913609891721F08093360962
:101AF0000E94259D0E94E4D92FEF3FEFA90120937A
:101B00001C0230931D0240931E0250931F02EB8172
:101B1000FC8182AD93ADA4ADB5AD8093F5109093EB
:101B2000F610A093F710B093F8102DE13DE141E0DD
:101B3000F901C590D590E590F490C816D906EA064B
:101B4000FB0650F4B695A79597958795440F2C5FA3
:101B50003F4F2216330661F74093F410803291050F
:101B6000A105B10508F4B1C18097A109B10981159A
:101B7000F8E09F07A105B10508F484C144E0949FF3
:101B800090011124235E364EF9013296459154910D
:101B9000EE27859FB001849F610D7E1F06946E1F06
:101BA0007E1F1124F901C590D490E12CF12CC61AA6
:101BB000D70AE108F108C0920911D0920A11E09207
:101BC0000B11F0920C118091091190910A11A091C2
:101BD0000B11B0910C11AC01BD010097E1E0AE0713
:101BE000B10520F04FEF5FEF60E070E0841B950BD4
:101BF000A60BB70B8093091190930A11A0930B11B8
:101C0000B0930C11F89480918400909185004096D7
